:100000000C94C80C0C94220D0C94220D0C94220D0F
:100010000C94220D0C94220D0C94220D0C94220DA4
:100020000C94220D0C94F9220C94220D0C94220DA8
:100030000C948E400C94220D0C94220D0C94220DE5
:100040000C94220D0C94220D0C94131F0C94220D71
:100050000C9458150C94220D0C9422150C94220D1E
:100060000C9428250C94220D0C94A53B0C94220D85
:100070000C9446AF0C94220D0C9477A40C94220D92
:100080000C94220D0C94220D0C94220D5125562512
:100090005B2564257B259225A225B225202678287C
:1000A00092253C274D27622781279E27E92735285F
:1000B000052BFB2BA42C1E2D572DF42D842E2B301D
:1000C000A830EB3067319531C23127328532EB32BF
:1000D0008F333C3405356635FE86128BBD8FA59275
:1000E0004094BC95B0971A9A1E9C0D87D7877A8842
:1000F000DE883C89D489CF9E698AEC8AEC8AEC8AB6
:10010000EC8AEC8AEC8AEC8AEC8AEC8A218BAE8B46
:100110004D8C868CE38C598DEB8D0A8F8D8F8D8F56
:100120008D8F8D8F8D8F8D8F8D8F8D8F8D8FCC8FB0
:10013000EC8F16909C90F290589192912692CF9EBF
:100140007592759275927592759275927592759277
:100150002D9C429C639C839CA59CBA9CCF9C209D1B
:10016000209D3B9D569D569D569D569D569D569D48
:10017000569D36AD39AD39AD39AD42AD45AD48AD21
:100180005AAD5DAD57AD0A0D3D3D3D3D3D3D3D3D5B
:100190003D3D3D3D3D3D3D3D3D3D3D3D3D3D3D3D8F
:1001A0003D3D3D3D3D3D3D3D3D3D3D000A0D4261F6
:1001B00074743A002025642043656C6C7320002021
:1001C0004C6F77207761726E696E673A2025642ED6
:1001D0002564560020204175746F2D43483A202530
:1001E000642E2564560020204175746F6C616E6426
:1001F000696E673A2025642E256456000A0D4F6CFF
:1002000064204643204861726477617265206E6F96
:100210007420737570706F727465642062792074D5
:10022000686973204669726D7761726521000A0DF5
:10023000466F756E6420424C2D4374726C3A2000F8
:100240002564000A0D0A0D2121204D495353494EC2
:100250004720424C2D4354524C3A20256420212102
:10026000000A0D424C2D4669726D7761726520253A
:10027000642E25303264003C2D2D207761726E692A
:100280006E67206F6C642056657273696F6E210013
:100290000A0D43616C6962726174696E67207072E5
:1002A0006573737572652073656E736F722E2E00A1
:1002B0004F4B0A0D000A0D466C696768742D74690E
:1002C0006D65202575206D696E20546F74616C3AE0
:1002D0002575206D696E00416E676C654E69636BB4
:1002E00020202020202020416E676C65526F6C6CAE
:1002F000202020202020204163634E69636B202052
:1003000020202020202020416363526F6C6C20202D
:10031000202020202020205961774779726F2020EB
:1003200020202020202020416C7469747564652091
:100330005B302E316D5D204163635A2020202020E8
:1003400020202020202020476173202020202020F2
:1003500020202020202020436F6D70617373205671
:10036000616C7565202020566F6C74616765205B39
:10037000302E31565D2020526563656976657220A6
:100380004C6576656C20204779726F20436F6D70E5
:10039000617373202020204D6F746F7220312020F4
:1003A000202020202020204D6F746F7220322020CA
:1003B000202020202020204D6F746F7220332020B9
:1003C000202020202020204D6F746F7220342020A8
:1003D00020202020202020313620202020202020F6
:1003E00020202020202020313720202020202020E5
:1003F00020202020202020313820202020202020D4
:1004000020202020202020313920202020202020C2
:1004100020202020202020536572766F202020206D
:1004200020202020202020486F766572676173208D
:100430002020202020202043757272656E74205B7E
:10044000302E31415D2020436170616369747920F1
:100450005B6D41685D20204865696768742053655D
:1004600074706F696E742032352020202020202087
:100470002020202020202032362020202020202054
:100480002020202020202032372020202020202043
:10049000202020202020204932432D4572726F7287
:1004A00020202020202020424C204C696D6974209F
:1004B000202020202020204750535F4E69636B206E
:1004C000202020202020204750535F526F6C6C204A
:1004D0002020202020202021212120494E434F4D43
:1004E00050415449424C4520212121002E005B25DA
:1004F000695D005B25695D002B204D696B726F4B58
:100500006F70746572202B0048573A5625642E256B
:10051000642053573A25642E253032642563200029
:100520005365743A256420257300424F4154004DB1
:1005300069786572204572726F72210045525225AA
:1005400032643A0048617264776172652045727264
:100550006F7220313A2564202121004D697373693F
:100560006E6720424C2D4374726C3A256420212121
:1005700000493243204552524F5221212100424C22
:100580002D53656C6674657374204572723A25321A
:1005900064004865696768743A202025356900530E
:1005A0006574706F696E743A2535690050726573B1
:1005B000737572653A253569004F66667365743ADE
:1005C00020202535690028412900256900616374D0
:1005D0002E2062656172696E67004E69636B3A2016
:1005E000202020202025356900526F6C6C3A202095
:1005F0002020202025356900436F6D706173733AA8
:10060000202020253569004B25693A2534692020B2
:100610004B25693A25346920004E693A2534692012
:1006200020526F3A253469200047733A25346920F7
:100630002047693A253469200050313A2534692031
:100640002050323A253469200050333A253469204D
:100650002050343A25346920004779726F202D20CC
:1006600053656E736F72004E69636B202534692089
:10067000282534692900526F6C6C202534692028A4
:1006800025346929005961772020253469202825DF
:1006900034692900414343202D2053656E736F72E6
:1006A000004E69636B2025346920282533692900B1
:1006B000526F6C6C20253469202825336929005A33
:1006C00020202020253469202825336929286361CA
:1006D0006C290043616C6962726174696F6E3A00E3
:1006E0004143433A2020204E3A25336920523A258F
:1006F00033692000537469636B3A202825692F25DC
:10070000692920212120006F6E20006C616E642019
:10071000746F20736176652020202000757365203A
:100720006B65797320746F207472696D2041434347
:10073000006F666600536176653F202020202028E8
:1007400079657329286E6F2900466C792077697462
:100750006820475053206F666600566F6C7461675F
:10076000653A2020202533692E25316956004375CE
:100770007272656E743A2020202533692E25316906
:100780004100506F7765723A20202020202534697F
:1007900057004469736368617267653A202535695B
:1007A0006D41680052656365697665720052432D3C
:1007B0005175616C6974793A202534690052432D72
:1007C0004368616E6E656C733A25346900556E64DA
:1007D0006572766F6C746167657320200057617273
:1007E0006E3A202532642E25645600486F6D653AB6
:1007F000202532642E256456004C616E643A202513
:1008000032642E25645600506F746925693A2020A1
:1008100025336900506F746925693A2020253369B2
:1008200000466C696768742D54696D65202000541A
:100830006F74616C3A2535756D696E004163743A69
:1008400020202535756D696E0028726573657429E1
:1008500000436F6D70617373004D61676E65743A2C
:10086000202020253569004779726F3A202020200A
:100870002025356900547275653A202020202025F6
:10088000356900536572766F202000536574706F70
:10089000696E74202025336900506F736974696F25
:1008A0006E3A202533690052616E67653A253369D7
:1008B0002D25336900424C2D4374726C20457272B1
:1008C0006F72732000253364202533642025336440
:1008D000202533642000253364202533642025330C
:1008E00064202533642000424C2D004572722E0096
:1008F000424C2D2054656D7065726174757265008F
:100900002533642025336420253364202533642077
:100910000025336420253364202533642025336487
:100920002000424C2D0054656D70004300424C2065
:1009300043757272656E740028696E20302E3141E5
:100940002900253364202533642025336420253392
:10095000642000253364202533642025336420255A
:1009600033642000424C2D004900424C2D437472E8
:100970006C20666F756E642000202000202532698F
:100980000020202D00424C2056657273696F6E73F3
:10099000002531642E25303264202531642E253027
:1009A0003264202531642E25303264202531642EB6
:1009B0002530326400202531642E25303264202514
:1009C00031642E25303264202531642E2530326486
:1009D000202531642E25303264000A0D2D2D3E2055
:1009E00048617264776172652056657273696F6ED3
:1009F0002042797465204368616E676564203C2DF0
:100A00002D000A0D47656E65726174696E6720641A
:100A1000656661756C7420506172616D6574657294
:100A200020536574202564000A0D5573696E672094
:100A3000506172616D657465722053657420256420
:100A4000000A0D47656E65726174696E67206465A2
:100A50006661756C74204D69786572205461626CB2
:100A600065000A0D4D697865722D436F6E66696782
:100A70003A202725732720282575204D6F746F7223
:100A80007329000A0D414343206E6F742063616C2B
:100A900069627261746564210D0A000A0D477972FA
:100AA0006F2063616C6962726174696F6E2064614A
:100AB0007461206E6F742076616C69640D0A0000A9
:100AC000008F001E01AD013B02CA025803E6037409
:100AD0000402058F051B06A7063307BE074808D288
:100AE000085B09E3096B0AF20A780BFD0B810C0421
:100AF0000D860D070E870E060F840F00107B10F574
:100B0000106E11E5115B12CF124213B3132314922E
:100B100014FE146A15D3153B16A11605176717C8DE
:100B20001727188318DE1837198E19E319361A8714
:100B30001AD61A231B6E1BB61BFD1B411C831CC33C
:100B40001C001D3C1D751DAB1DE01D121E421E6FBD
:100B50001E9A1EC31EE91E0D1F2E1F4D1F691F84E6
:100B60001F9B1FB01FC31FD31FE11FEC1FF51FFBEF
:100B70001FFF1F00204C6F61642073696E676C2E2D
:100B8000506F696E7400536176652073696E676C8F
:100B90002E506F696E74004143432063616C69623B
:100BA000726174696F6E004143432063616C6962D6
:100BB000726174696F6E0041434320204E3D2533BE
:100BC0006920523D25336900537469636B212028E5
:100BD00025692F256929006C616E6420746F20736C
:100BE0006176652020202000757365206B65797320
:100BF000206E6F772020202000466C792077697462
:100C00006820475053206F66660020202020202057
:100C10002073617665202D2D3E002076616C756510
:100C2000732073746F726564202000737769746336
:100C30006820475053206F66662020005361766518
:100C400020506F696E743A006E6F2053442D4361DB
:100C50007264006E6F204750532D4669780025322C
:100C600064002D2D004469723A25336420416C7470
:100C70003A2533646D002D3E002020004C6F6164E6
:100C800020506F696E74006E6F2053442D43617263
:100C90006400253264002D2D00446973743A2533B5
:100CA0006420416C743A25336420002020202020E9
:100CB0002020202020202020202020002D3E002049
:100CC00020000000050005000401060108000601DF
:100CD00002000400040007000700070007000700E7
:100CE0000700070003010301050017010F010600BB
:100CF00009010A0119010501050119011A010F0174
:100D000001000900060006000501050000000800BA
:100D10004E6F204572726F722020202020202020EC
:100D2000004E6F7420636F6D70617469626C652032
:100D300020004D4B334D6167206E6F7420636F6DE3
:100D40007061004E6F20464320636F6D6D756E6954
:100D500063617400436F6D7061737320636F6D6DB9
:100D6000756E69630047505320636F6D6D756E69D2
:100D7000636174696F00636F6D7061737320766176
:100D80006C7565202020005243205369676E616CAA
:100D9000206C6F73742020004643207370692072AA
:100DA00078206572726F7220004E6F204E43206370
:100DB0006F6D6D756E69636174004643204E6963A3
:100DC0006B204779726F2020202000464320526F0D
:100DD0006C6C204779726F202020200046432059F8
:100DE0006177204779726F20202020200046432021
:100DF0004E69636B2041434320202020200046435E
:100E000020526F6C6C20414343202020202000465C
:100E100043205A2D41434320202020202020200021
:100E200050726573737572652073656E736F72208F
:100E3000004932432046432D3E424C2D4374726C90
:100E40002000426C204D697373696E67202020205A
:100E50002020004D69786572204572726F722020E3
:100E600020202000436172656672656520457272BC
:100E70006F7220200047505320466978206C6F73B2
:100E80007420202020004D61676E657420457272C9
:100E90006F7220202020004D6F746F722072657376
:100EA0007461727420202000424C204C696D69747A
:100EB0006174696F6E202020004750532052616E8C
:100EC000676520202020202020004E6F2053442DD5
:100ED000436172642020202020200053442D4C6F59
:100EE0006767696E67206572726F7200466C796918
:100EF0006E672072616E676521202020004D617849
:100F000020416C74697475646521202020004E6F47
:100F1000204750532066697820202020202000633D
:100F20006F6D70617373206E6F742063616C2E003F
:100F3000424C2D53656C667465737420202020200C
:100F4000006E6F206578742E20636F6D706173730F
:100F50002000636F6D706173732073656E736F72C1
:100F60002020004661696C7361666520706F737440
:100F7000696F6E004E6F20526564756E64616E63BA
:100F80007921202000526564756E64616E6379205A
:100F90007465737420004750532055706461746504
:100FA0002052617465200053657420203A00204C63
:100FB0006F616420506F736974696F6E2053503194
:100FC000202020002053746F726520506F73697465
:100FD000696F6E20535031202000204D696B726F75
:100FE0004B6F707465722028426F61742920200055
:100FF000202053494D554C4154494F4E2061637454
:101000006976652020002021212020204C414E447B
:10101000494E47202020202121202000202121206E
:101020004C69506F20766F6C7461676520212120B8
:10103000200020202020204D696B726F4B6F707450
:101040006572202020202000202020202020202029
:1010500020202020202020202020202020002020B0
:101060002532692E2531695620200020202532693D
:101070002E25316956202000414C543A2534696DA3
:1010800020256300414C543A2534696D20200041ED
:101090004C543A2D2D2D2D200020202532693A2543
:1010A00030326920200020202532693A253032690B
:1010B0002020004449523A20253364256300430030
:1010C000200020202535692020002020253569209A
:1010D0002000493A2532692E2531694120003A0025
:1010E0003A003A002D2D2D2D2D2D2D2D2D2B2D2D72
:1010F0002D2D2D2D2D2D2D2D2D002D2D2D2D2D2D4D
:101100002D2D2D2D2D2D2D2D2D2D2D2D2D2D2D003C
:101110003A005341543A2532642000444953543A2A
:101120002533646D004420003344002121004D41EB
:10113000473A25337525252000484D3A2533642547
:101140006320256300696E636C3A25326425632849
:101150002532692900202020202532756D2F733A11
:101160002020484D3A2533642563202563004552ED
:10117000523A202532642021004552523A20002163
:1011800021204C69506F20766F6C74616765202157
:101190002100207777772E4D696B726F4B6F7074DB
:1011A00065722E6465202000202532693A25303290
:1011B0006920202532692E25316956202534696D34
:1011C000416800202532693A2530326920202532D5
:1011D000692E25316956202534696D4168004449DE
:1011E000523A253364256300414C543A2534696DE5
:1011F00000414C543A2534696D00414C543A2D2D30
:101200002D2D2000256300484D3A253364256320A9
:1012100020444953543A2533646D202563005057C8
:10122000523A2532692E25316941202825695729EE
:1012300020004346002020004750533A2532756D68
:101240002F73205341543A2564200020203344203A
:10125000004E4F464958004447505320002020205C
:101260004E6F204E6176694374726C2020202020DE
:101270002020002532692E2569202532692E256916
:10128000202532692E2569202532692E25694100E5
:1012900025336920253369202533692025336925C5
:1012A0006343002532692E2569202532692E256980
:1012B00041002532692E2569202532692E256920B5
:1012C0002532692E2569202532692E2569410025A0
:1012D00033692025336925634320202020202020E6
:1012E00020002533692025336920253369202533E3
:1012F00069256343004552523A202532642021007B
:101300004552523A20002121204C69506F20766FBF
:101310006C7461676520212100207777772E4D69F5
:101320006B726F4B6F707465722E64652020005372
:10133000657474696E673A257520257320004D69C0
:101340006E3A2532692E25316956202573200041D9
:101350004C543A00504F54493A2533752000284FD9
:101360004E29202000284F46462920004C494D494F
:101370005400564152494F0044495341424C454460
:101380000043463A0044495341424C45440020281A
:101390004F4E29200020284F464629002054454121
:1013A0004348004750533A0044495341424C454456
:1013B000002846524545290028484F4D4529002818
:1013C00041494429200028484F4C442900204653D5
:1013D0003A257573656B2000484F4D4520414C54AC
:1013E0003A0025756D00484F4C4420004E693A255F
:1013F000346920526F3A25346920433A2533690015
:1014000047733A2534692059613A253469200050E0
:10141000313A2534692050323A25346920333A254F
:1014200033690050343A2534692050353A253469FF
:1014300020363A253369004C4F4F50494E47212002
:10144000004848212000434F4D50415353204F4600
:10145000462120004C6F616420576179706F696E7E
:101460007473002852656C617469766520506F73DF
:101470006974696F6E7329004163746976652057DA
:10148000503A2532642F256420004E6F2057507348
:101490002061637469766520202020200025326950
:1014A0002E2531695620002573002020200025328A
:1014B00069202020004C6F6164206C6973743A00CD
:1014C0004C6F6164206C6973743A202D2D20004E9E
:1014D0006F2053442D4361726420202000285365FF
:1014E00074202D3E204C6F61642900202020202094
:1014F000202020202020202000214E6F2047505304
:101500002D4669782120004C6F6164205761797005
:101510006F696E74730028466978656420506F7334
:101520006974696F6E732900416374697665205729
:10153000503A2532642F256420004E6F2057507397
:101540002061637469766520202020002532692E91
:101550002531695620002573004C6F6164206C6949
:1015600073743A0020202000253264202846495810
:101570002900202D2D004E6F2053442D43617264AD
:101580002020200028536574202D3E204C6F61647C
:101590002900202020202020202020202020200082
:1015A00053746F72652073696E676C6520506F733A
:1015B0006974696F6E00202532692E2531695620C5
:1015C00000202532693A253032692000414C543AD6
:1015D0002534696D004449523A202533642563005F
:1015E00043616D3A202533690053746F7265207032
:1015F0006F696E743A002020200025326420002D8F
:101600002D004E6F2053442D436172642020200032
:1016100028536574202D3E2053746F726529002174
:101620004E6F204750532D4669782120004C6F6142
:10163000642073696E676C6520506F736974696F9D
:101640006E00202532692E25316956200020253272
:10165000693A25303269200057503A2532642F25E7
:101660006420446973743A2533646D2000414C54FE
:101670003A2534692F25696D2000414C543A2534B0
:10168000696D20202020004449523A2025336425EA
:10169000630043616D3A20253369006C6F616420FB
:1016A000706F696E743A0020202000253264002D8E
:1016B0002D004E6F2053442D436172642020200082
:1016C00028536574202D3E204C6F616429002573DA
:1016D000004D6F746F7274657374202F205365749E
:1016E000706F696E7473004D25693D25326925322E
:1016F000692E256941204D25693D253269253269CC
:101700002E256941004D25693D2532692532692E16
:10171000256941204D25693D2532692532692E25EF
:101720006941002121214D6F746F727465737420BB
:10173000416B746976212121004D6F746F722025F1
:1017400069004143432063616C6962726174696F2F
:101750006E004143433A2020204E3A2533692052FF
:101760003A2533692000537469636B3A202020289E
:1017700025692F2569292020202020002121004FC4
:1017800066660043616C69627261746500536176DC
:101790006520202020202020202020002853455490
:1017A0002900537769636820475053206F6666218C
:1017B000003E002A002000202020202000200020C1
:1017C000002000206F6B6179200020004D6F746F46
:1017D00072732072756E6E696E6721212100200080
:1017E000004F505152535453565748005859005ABD
:1017F0005545464748410049424A4A00000000001A
:10180000000000000000444C4D00000000004E00AD
:1018100000004B00430A0D7777772E4D696B726F8E
:101820004B6F707465722E646520286329204869A7
:1018300053797374656D7320476D6248000A0D74A7
:10184000686520757365206F6620746869732073FE
:101850006F667477617265206973206F6E6C792092
:101860007065726D6974746564200A0D6F6E206F07
:10187000726967696E616C204D696B726F4B6F7036
:101880007465722D48617264776172650055736585
:101890007200486F5454205634004143542044533E
:1018A0004C004A657469005370656B7472756D0005
:1018B00050504D000A0D52656365697665723A2095
:1018C00000532E427573004D554C5449504C4558A9
:1018D00000756E6B6E6F776E2E205573696E672084
:1018E00050504D2E2E2E006E6F7420737570706FD9
:1018F00072746564206279206861726477617265D0
:1019000021000A0D202D204C4942204E4F542043E7
:101910004F4D50415449424C452021212121000A7C
:101920000D0A0D212120426F6F746C6F6164657226
:10193000206E6F7420636F6D70617469626C6520D6
:10194000746F204861726477617265203E20322E88
:10195000322021210A0D0A0D000A0D466C696768C4
:1019600074436F6E74726F6C0A0D486172647761B4
:1019700072653A25642E25640A0D536F667477618B
:1019800072653A5625642E253032642563200000A6
:1019900011241FBECFEFD0E4DEBFCDBF12E0A0E028
:1019A000B1E0ECE7F4E601E00BBF02C007900D9256
:1019B000A03FB107D9F71DE0A0EFB2E001C01D9232
:1019C000A038B107E1F77AEAE2E0F0E081E2809343
:1019D0005700149120EF37EF41E050E0C6E2D5E028
:1019E0006FE0DA01C9012F5F3F4F4F4F5F4FABBF31
:1019F000FC0187918993615067FFF3CF84EE8ABD24
:101A000080912E058093FA04893138F086E0809326
:101A1000150187E0809314017BEAE6E2F5E06EE0D1
:101A2000819178277095615067FFFACF80913505D5
:101A3000781721F0173911F40000FECF0E942D0F06
:101A40000C943DB20C94000086E891E09F938F9334
:101A50008AEE9BE19F938F93E0913905F0913A05CF
:101A600009950F900F900F900F9008950E94D551F7
:101A70008091050A9091060A2FEF8D3E920714F08F
:101A8000109204018A5B9F4FCCF48091040188235B
:101A9000A9F481E080930401809174058F5F8093A5
:101AA0007405853038F088EE93E090932E03809390
:101AB0002D03089566E970E00E94924208951F93F5
:101AC000CF93DF93182F882311F18CEA91E09F9335
:101AD0008F938AEE9BE19F938F93E0913905F0916C
:101AE0003A05099580912701909128016BE270E0F9
:101AF0000E94B0B1CB018F5F809300010F900F90D7
:101B00000F900F90873018F086E08093000180914D
:101B1000FD07823318F590910001989FE001112490
:101B20001123F1F068EC70E0892F0E9492428091BD
:101B3000000199279F938F9384EB91E09F938F935C
:101B40008AEE9BE19F938F93E0913905F0913A05DE
:101B500009958DB79EB706968DBF02C0C82FDD27A9
:101B6000CF3FD10519F010F0CFEFD0E0C0930201C4
:101B700090915208923330F480910001899FE001E6
:101B8000112402C0C92FDD27CF3FD10519F010F075
:101B9000CFEFD0E0C093F90230915308323330F4E4
:101BA00080910001839FE001112402C0C32FDD2733
:101BB000CF3FD10519F010F0CFEFD0E0C093F8027D
:101BC0008091F90290910201981720F4915090931E
:101BD000F9029F5FC91720F091509093F8029F5F20
:101BE0008091F9022091F802821728F0332319F02E
:101BF00021502093F902112309F462C0892F6AE071
:101C00000E9490B1892F99279F938F938091020111
:101C10000E9490B199279F938F938FEB91E09F93B0
:101C20008F93CAEEDBE1DF93CF93E0913905F0911A
:101C30003A0509958DB79EB708968DBF8091F80239
:101C40008823E9F06AE00E9490B1892F99279F9339
:101C50008F938091F8020E9490B199279F938F9360
:101C600084ED91E09F938F93DF93CF93E0913905BB
:101C7000F0913A0509958DB79EB708968DBF809172
:101C8000F9028823E9F06AE00E9490B1892F992730
:101C90009F938F938091F9020E9490B199279F930F
:101CA0008F9386EE91E09F938F93DF93CF93E09194
:101CB0003905F0913A0509958DB79EB708968DBF05
:101CC000DF91CF911F91089580915708E82FFF274A
:101CD000EE0FFF1FE95FF54F80819181C3970CF4F0
:101CE00058C08091FB02813011F0833081F491E083
:101CF0009093D40482E08093FB028DE08093B00146
:101D000085E08093D2049093D1049093FD0280915A
:101D10005808E82FFF27EE0FFF1FE95FF54F80817E
:101D20009181C3977CF082E0809305018091FE024F
:101D30009091FF020E940420882309F48DC0109224
:101D4000FD025BC0808191818E5C9F4F0CF084C04E
:101D500084EC99E00E94FB1F9093FF028093FE02A7
:101D600080910501823009F071C09091FD0280914F
:101D7000D504981708F06AC0892F8F5F8093FD0201
:101D80008093D40495E09093D2048093D1048DE0A5
:101D90005BC0808191818E5C9F4F0CF05AC0809116
:101DA000FB028150823080F491E09093D30483E071
:101DB0008093FB0285E18093B00185E08093D0049D
:101DC0009093CF049093FC0280915808E82FFF274E
:101DD000EE0FFF1FE95FF54F80819181C3978CF073
:101DE00082E0809305018091FE029091FF020E94A3
:101DF0000420882389F11092FC0281E08093050180
:101E00000895808191818E5C9F4F34F584EC99E038
:101E10000E94FB1F9093FF028093FE0280910501B8
:101E20008230A1F49091FC028091D504981770F44F
:101E3000892F8F5F8093FC028093D30495E0909369
:101E4000D0048093CF0485E18093B0011092050106
:101E5000089581E08093FB020895CFEFD0E4DEBFC8
:101E6000CDBF88249924C1E07C2E14B815B88AE02F
:101E70008AB98FE58BB9B7EECB2EB3E0DB2E2EEC13
:101E80003FEFC20ED31ED7FEFACF6624199B0DC0BA
:101E90004C9B04C085E1809303010EC086E18093D2
:101EA000030181E08093A00307C089E180930301CF
:101EB00081E08093A0035C9881E887B93E9A8FEF18
:101EC00088B98BE184B981E085B9469A84B7877F68
:101ED00084BF8091600088618093600010926000F0
:101EE00084EC99E090932E0380932D031092E903E4
:101EF0001092E8031092EB031092EA031092ED03A4
:101F00001092EC0320910301243128F084EC94E03A
:101F1000A0E0B0E004C08BE095E0A0E0B0E08093EA
:101F2000450190934601A0934701B093480128983A
:101F3000293111F4299A01C029980E9464200E9435
:101F400035200E94F21B0E9455400E944A2481E0E5
:101F50000E94523B0E944B720E94328087E00E9496
:101F6000B6AD80910301893111F4299A01C02998F5
:101F700078940E94313A809103018431E8F488E139
:101F800090E02CE00FB6F894A895809360000FBE07
:101F9000209360008CEF91E09F938F938AEE9BE1FA
:101FA0009F938F93E0913905F0913A0509950F9031
:101FB0000F900F900F90EECF8091870382608093F7
:101FC000870310928A03C0E0D0E00E94194E85E09A
:101FD00090E00E94FB1F6C018091870380FD05C08B
:101FE000C6010E9404208823B9F3219631E0C43F42
:101FF000D30758F38EE292E09F938F93AAEEAA2E16
:10200000ABE1BA2EBF92AF92E0913905F0913A055B
:102010000995C0E0D0E00F900F900F900F9000E175
:1020200019E0F7E7EF2EF8E0FF2EF701808124E0BA
:1020300030E0E20EF31E181684F406C08091870388
:1020400080FF02C00E94194EC6010E94042088230E
:1020500021F4F801838188238CF7F801838187FFBD
:102060002CC0CE0101966AE070E00E949CB19F9363
:102070008F9380E492E09F938F93BF92AF92E09111
:102080003905F0913A0509958091F1028F5F8093AF
:10209000F102F801948584E6989FC00111242585FA
:1020A000280F8DB79EB706968DBF222331F0809101
:1020B0005C05281710F420935C052196015F1F4FE3
:1020C000C031D10508F4B1CFC0E0D0E000E119E0A3
:1020D000E7E7EE2EE8E0FE2EF801838187FD1DC0C4
:1020E000F70180811816CCF42196DF93CF932197C6
:1020F00083E492E09F938F938AEE9BE19F938F936B
:10210000E0913905F0913A05099582E080932B031F
:102110002DB73EB72A5F3F4F2DBFF80183818078EE
:102120008383219624E030E0E20EF31E015F1F4F0F
:10213000C031D10588F280915C058F3F99F164E64A
:102140000E9490B1892F99279F938F9380915C056E
:102150000E9490B199279F938F9381E692E09F937D
:102160008F93CAEEDBE1DF93CF93E0913905F091D5
:102170003A05099580915C058456EDB7FEB738960F
:10218000EDBF833078F487E792E09F938F93DF93DE
:10219000CF93E0913905F0913A0509950F900F9092
:1021A0000F900F900E94240D9091D8078091F1021A
:1021B000981728F480915A05806180935A059930C8
:1021C00020F088E080933F0102C090933F0180E9B6
:1021D00092E09F938F93CAEEDBE1DF93CF93E09180
:1021E0003905F0913A05099588EE93E00E94FB1FAE
:1021F0006C010E9488240F900F900F900F90C601E1
:102200000E9404208823D9F380EB92E09F938F9360
:10221000DF93CF93E0913905F0913A05099580E07D
:102220000E949843289880ED97E090932E03809326
:102230002D038EE090E00E944B389927182F00273D
:102240008FE090E00E944B38080F111D1093F702A9
:102250000093F6028AE090E00E944B389927182FED
:1022600000278BE090E00E944B38080F111D10935F
:10227000F5020093F4020F900F900F900F900F5FF4
:102280001F4F39F08091F6029091F7028F5F9F4FB8
:1022900041F41092F7021092F6021092F502109299
:1022A000F4028091F4029091F5029F938F938091B4
:1022B000F6029091F7029F938F9385EB92E09F93A4
:1022C0008F93DF93CF93E0913905F0913A0509950B
:1022D0000E947E2A88E893E190933E0180933D011D
:1022E000C1E0C09375058C2F0E945F0D809100089E
:1022F0000E94FAAC0E94240D80ED97E00E94FB1F23
:102300006C018AEF90E00E94FB1F93E090933207EC
:102310001092F00280915B08EDB7FEB73896EDBFE2
:1023200084FF02C0C093FA029093400112BC11BC1A
:1023300080910103882311F04798FECF80913103EB
:10234000882309F45CC380911901882309F457C3D9
:10235000F894809131038150809331037894809177
:102360007405882319F00E94360D02C00E94A45201
:102370000E94194E28988091DC03882331F08091C7
:10238000DC0381508093DC0352C080916F00806237
:1023900080936F001092080A1092070A80915A05E4
:1023A000886080935A058091DA07A82FBB27AA0F6F
:1023B000BB1FFD01E15BF54F118210828091DB07AD
:1023C000E82FFF27EE0FFF1FCF01815B954FEC0138
:1023D00019821882A95FB54F11961C921E92E95F6F
:1023E000F54F118210828091DD07E82FFF27EE0F55
:1023F000FF1FE95FF54F118210828091DC07E82F03
:10240000FF27EE0FFF1FE95FF54F11821082109238
:10241000060A1092050A1092030A1092020A1092FC
:10242000010A1092000A10924E0A10924D0A8091F1
:102430003D0190913E01019790933E0180933D01B3
:1024400080913D0190913E01892B21F0809188037C
:102450008823C9F180913D0190913E01892BD9F4E7
:102460000E94833B85E090E090933E0180933D0184
:1024700080916C0790916D07019690936D07809302
:102480006C0780915A05816080935A0580913307CB
:1024900082608093330780910C0190910D018F5FD2
:1024A0009F4F91F48091DB03882371F088EA91E6D5
:1024B00090932E0380932D0380E890E090930D017C
:1024C00080930C0101C028980E94B9AE809131031D
:1024D000882309F092C28091F204882319F00E94A7
:1024E0004F9F8BC28091F504882319F00E9452A05F
:1024F00084C280912C03882311F40E946C72809115
:102500001201882311F00E94BE200E943F1C0E94ED
:10251000AD17C6010E940420882309F46AC224E191
:1025200030E0C20ED31E0E947C2020919101309198
:1025300092018FEF2F3F3807C9F18091C60388239E
:1025400069F5E091F403F091F503E217F30731F137
:102550008091B003882321F480918E048823F1F0C8
:10256000CF01821B930B845E9D4F68E671E00E9451
:10257000B0B1845B9040833091051CF082E090E024
:1025800006C0CFEF8E3F9C0714F48EEF9FEFE81B41
:10259000F90BF093F503E093F40308C08FEF9FEF7E
:1025A000909392018093910110928E048091000883
:1025B000863019F40E94C98604C0843011F40E9448
:1025C0007EA08091A003882331F1809179079091BA
:1025D0007A078C52914074F08091420790914307A2
:1025E00080509240C4F48091790790917A07835586
:1025F00093408CF0639432E3361570F48091DB03E2
:10260000882331F08091590580628093590504C078
:102610008093C70301C0662480918803882329F42E
:1026200080918C0B8E3150F405C080915A058260E8
:1026300080935A058091330782600FC080912D03EB
:1026400090912E03892B59F480913D0190913E0188
:10265000079728F0809133078D7F8093330780910F
:10266000FA02882361F08091DC03873940F01092F0
:10267000FA0288E893E190932E0380932D038091D2
:102680000701882321F081508093070120C08091A9
:10269000DC038823E1F480910C0190910D018F5FA0
:1026A0009F4FA9F42091FA02223089F088E99AE339
:1026B00090932E0380932D0380E09CE090930D0176
:1026C00080930C01222319F082E08093FA0280911A
:1026D000A701893C70F081508093A70180915A0531
:1026E0008B7F80935A0580915D05816080935D05A5
:1026F00053C080910E0B8823F9F080915A058460B5
:1027000080935A0589E08093930480910C01909105
:102710000D018F5F9F4F81F48091DB03882361F06F
:1027200088E99AE390932E0380932D0380E098EA42
:1027300090930D0180930C011092850410928404F3
:102740001092830410928204109281041092010B63
:102750008FEF8093760B1092400B10923F0B1092EC
:10276000420B1092410B8FEF9FEF90933E0B8093A3
:102770003D0B1092CB031092CC031092CD0310921C
:10278000CE031092CF0380915D058E7F80935D050F
:1027900010928F041092A70180910201282F3327F5
:1027A000809127019091280128173907F4F0809132
:1027B000A90380628093A90380910C0190910D017F
:1027C0008F5F9F4F91F480912701909128010B9783
:1027D00064F080E797E190932E0380932D0380E0CF
:1027E00093E090930D0180930C0180910A0388235C
:1027F00069F0815080930A03813041F410925205B0
:1028000080ED97E090932E0380932D0380915708DD
:10281000882311F00E94640E809100038F5F8093E3
:102820000003813309F09CC0109200038091C8041A
:10283000882319F081508093C8048091D2048823A2
:1028400019F081508093D2048091D004882319F02C
:1028500081508093D00480918F0483FF02C08AE06E
:1028600005C080919903882319F0815080939903C2
:102870008091A90381FF0AC08091F2029091F30236
:1028800001969093F3028093F20204C05AEA852ED7
:1028900055E0952E8091AA039091AB03805094400F
:1028A00008F04EC020917B0730917C0740917D0756
:1028B00050917E0780911F0190912001A0912101EC
:1028C000B0912201281739074A075B0764F4809109
:1028D0007B0790917C07A0917D07B0917E070596BC
:1028E000A11DB11D20C020917B0730917C07409134
:1028F0007D0750917E0780911F0190912001A0914A
:102900002101B091220182179307A407B5079CF417
:1029100080917B0790917C07A0917D07B0917E0705
:102920000597A109B10980937B0790937C07A09339
:102930007D07B0937E078091A7038B7F8093A703C9
:102940008091020199270196209127013091280159
:10295000821793072CF48091A9038F7D8093A9039C
:102960000894811C911C32E783163BE0930609F022
:1029700040C0882499242091F6023091F7022F5FFD
:102980003F4F3093F7022093F6028091F40290912A
:10299000F50201969093F5028093F402832F992714
:1029A000682F8EE090E00E9453388091F60290915B
:1029B000F7029070682F8FE090E00E94533880916A
:1029C000F4029091F502892F9927682F8AE090E010
:1029D0000E9453388091F4029091F5029070682F14
:1029E0008BE090E00E94533884E190E00E94FB1F4E
:1029F0006C010E9412780E946C8071107A9477208A
:102A000039F40E94D677882319F08CE0782E8ECC8A
:102A100080912C03882309F089CC0E946C7286CCAB
:102A200040E020E030E0F901E952FD4F85919491BA
:102A3000480F2F5F3F4F82E020303807A0F3842FEC
:102A4000992708951F920F920FB60F9211248F931A
:102A50009F93EF93FF93809109018823E1F4809184
:102A60001C0390911D03019690931D0380931C03FA
:102A7000FC01EA5AF94FE081ED3019F08C3D9105E7
:102A800039F410921D0310921C0381E08093090118
:102A9000E093C60004C010921D0310921C03FF9126
:102AA000EF919F918F910F900FBE0F901F901895EF
:102AB0001F920F920FB60F9211242F933F934F93B3
:102AC0005F936F937F938F939F93AF93BF93CF93B6
:102AD000EF93FF9390E080910103813029F480917E
:102AE000C6008093CE00D1C080910103823029F4CA
:102AF0008091C60080937805C8C08091C6008093FD
:102B00001403509122035C3D10F0909323038091B5
:102B100014038D3009F06AC080912303823009F0DC
:102B200065C090932303852F992788589A4FFC01FD
:102B30003297408120911E0330911F03241B3109DD
:102B4000DC0111978C91281B3109C9019F7090936A
:102B50001F0380931E0346E0969587954A95E1F7FB
:102B6000982F935C909320032F733070235C2093F5
:102B700021038081981729F48C91281711F491E092
:102B800006C090E0809111038F5F809311038091C4
:102B90001303882309F079C0992309F476C081E0F2
:102BA00080931303580F509310035150E52FFF27C4
:102BB000E858FA4F8DE0808380917A05823509F0DC
:102BC00064C0C091DB03CC2309F05FC00E947E2A61
:102BD00088E190E02CE00FB6F894A895809360000F
:102BE0000FBE20936000C0932B034FC0209123039E
:102BF000822F992781309105F9F0823091051CF4DC
:102C0000892B21F040C0029711F13DC0809114033F
:102C1000833239F480911303882319F481E080937F
:102C20002303809114038093780581E0809322032D
:102C300080911403992722C02F5F20932303E52F4F
:102C4000FF27E858FA4F80911403808309C0E52FCD
:102C5000FF27E858FA4F8091140380835C3D20F4ED
:102C60005F5F5093220302C010922303209114034C
:102C700080911E0390911F03820F911D90931F035B
:102C800080931E0302C010922303FF91EF91CF9116
:102C9000BF91AF919F918F917F916F915F914F9174
:102CA0003F912F910F900FBE0F901F901895AC0180
:102CB000A0E0B0E09D01A817B90748F4E6E5F6E00A
:102CC0008191280F311D1196A417B507C8F33F70E5
:102CD000FD01EA5AF94FC90156E0969587955A9534
:102CE000E1F7835C80831196FD01EA5AF94F2F7357
:102CF0003070822F835C8083A95AB94F8DE08C930A
:102D000010920901809156068093C6000895A0E0B4
:102D1000B0E0EDE8F6E10C9409B22C859D850E85B6
:102D2000BB2483E2809356069F59909357062093C5
:102D3000580633E0E32EF12C002309F49EC0CF8423
:102D4000D888BE016D5E7F4FA989BA89015010975E
:102D500009F493C01097B9F0F601EB0DF11DB3948F
:102D60009081119791F4002349F1FB016E5F7F4F31
:102D7000DB01C080D1806E5F7F4F0D90BC91A02D94
:102D8000BB24015002C090E019C01097B9F0F601C1
:102D9000EB0DF11DB3944081119791F4002341F1A3
:102DA000FB016E5F7F4FDB01C080D1806E5F7F4F84
:102DB0000D90BC91A02DBB24015002C040E018C072
:102DC0001097B1F0F601EB0DF11DB394108111973E
:102DD00081F4002371F0FB013296DB01CD90DC9091
:102DE000BF016E5F7F4FA081B181BB24015001C044
:102DF00010E0F701EA5AF94F892F86958695835C92
:102E000080830894E11CF11CF701EA5AF94F892FDD
:102E100099278370907024E0880F991F2A95E1F715
:102E200055279A0194E0369527959A95E1F7822BDC
:102E3000835C80830894E11CF11CF701EA5AF94F86
:102E40004F705070440F551F440F551F812F992705
:102E500026E0969587952A95E1F7842B835C8083FD
:102E60000894E11CF11CF701EA5AF94F1F73135C37
:102E700010830894E11CF11C6ACFC7010E94571609
:102E8000E9E00C9425B2A3E07A2F4091100346505C
:102E9000442309F458C0E72FFF27E858FA4F8081F0
:102EA0008D537F5FE72FFF27E858FA4F20812D537E
:102EB0007F5FE72FFF27E858FA4F30813D537F5F50
:102EC000E72FFF27E858FA4F60816D537F5F9927FE
:102ED000880F991F880F991F522F52955F70582B9A
:102EE000822F99278F709070F4E0880F991FFA95C0
:102EF000E1F7232F26952695282B832F992783707A
:102F00009070E6E0880F991FEA95E1F7682B415031
:102F10004F3FC9F0EA2FFF27E858FA4F5083AF5FC1
:102F200041504F3F81F0EA2FFF27E858FA4F2083A6
:102F3000AF5F41504F3F39F0EA2FFF27E858FA4F73
:102F40006083AF5FA5CF8BE795E090930F038093ED
:102F50000E03A350A0930D030895A2E0B0E0E3EBAD
:102F6000F7E10C940FB280911303882309F42EC467
:102F70000E94431780917905823609F0E4C280915E
:102F80007A0599278037910509F4AFC081379105FB
:102F9000C4F48A36910509F441C28B36910544F494
:102FA0008B34910571F18636910509F46AC1CBC263
:102FB0008D36910509F469C08E36910509F44DC02E
:102FC000C2C28437910541F1853791054CF48137B0
:102FD000910509F491C08337910509F4EAC0B3C2A1
:102FE0008737910509F4DCC1883791052CF48537C2
:102FF000910509F498C1A7C28937910509F47DC1EB
:10300000A2C2E0910E03F0910F0380819181909311
:1030100094018093930197C280911003A0910E03B5
:10302000B0910F03853140F080E1EEE5F5E00D90C1
:1030300001928A95E1F70DC08D919D910D90BC9103
:10304000A02D80935E0590935F05A0936005B093DB
:10305000610580EF80930B034BC0809109018823A9
:10306000E1F38DE490E09F938F938AE698E09F933D
:103070008F9381E08F938F938EE48F930E948716B6
:103080008DB79EB707968DBF5EC2A0910E03B0911B
:103090000F031C91113081F48DE4EAE6F8E00D9005
:1030A00001928A95E1F70E946C39198380915A0543
:1030B0008F7E80935A0501C019828091090188236F
:1030C000E1F381E090E09F938F93CE0101969F936F
:1030D0008F9381E08F938F938DE48F930E94871657
:1030E000ADB7BEB71796ADBF2EC281E08093160371
:1030F0008FEF8093070127C28091DB038823E1F5DE
:10310000E0910E03F0910F03E0818E2F8A508A30F8
:1031100058F48983882311F481E003C0863010F0CD
:1031200085E0898361E00EC08E2F84518A3070F46F
:103130008983882311F481E003C0863010F085E094
:10314000898360E089810E94EE3912C0E983EF3FF4
:1031500019F40E94CF3989838981882311F481E091
:1031600003C0863010F085E0898389810E94693828
:1031700080E00E945F0D03C00E94CF398983809157
:1031800009018823E1F380E990E09F938F9389ED13
:1031900097E09F938F9381E090E09F938F93CE0170
:1031A00001969F938F9382E08F9381E08F9381E5C7
:1031B0002DC120910E0330910F03D9018C918150C4
:1031C000853008F045C0F90181818A3609F040C098
:1031D0008091DB038823E1F52F5F3F4F80E9E9ED24
:1031E000F7E0D9010D9001928A95E1F7F9018291FA
:1031F0000E94DC3880911A089927AA27BB27BC01B6
:10320000CD0124EC39E040E050E00E9471B1DC01D6
:10321000CB018093890190938A01A0938B01B09395
:103220008C0180911B089927AA27BB27BC01CD01DF
:103230000E9471B1DC01CB018093850190938601DE
:10324000A0938701B09388010E94CF39898301C080
:103250001982809109018823E1F381E090E09F9336
:103260008F93CE0101969F938F9381E08F938F93DD
:1032700083E58F930E9487168DB79EB707968DBF03
:103280002BC08091DB03882309F05DC1E0910E0320
:10329000F0910F03E0818E2F8150853018F48E2F2E
:1032A0000E9469380E94CF3989838091090188235F
:1032B000E1F381E090E09F938F93CE0101969F937D
:1032C0008F9381E08F938F9386E48F930E9487166C
:1032D000ADB7BEB71796ADBF1091DB03112341F414
:1032E0006EE670E089810E949242812F0E945F0DFC
:1032F000809100080E94FAAC26C119822981A09110
:103300000E03B0910F03E7E0FAE08D91992787FD56
:10331000909593A382A3822F8F5F8983282F329663
:103320008C3098F310C1E0910E03F0910F0380816F
:103330000E94C53F8A83882319F481E0898301C0F4
:103340001982809109018823E1F388E090E09F933E
:103350008F9388E099E09F938F9321E030E03F9333
:103360002F9380910E0390910F039F938F933F9320
:103370002F93CE0102969F938F933F932F93CE016D
:10338000820F931F9F938F9384E08F9381E08F939D
:1033900085E58F930E948716EDB7FEB773963CC004
:1033A00080910D03893008F4CEC020910E03309136
:1033B0000F032F5F3F4F88E0A8E0B9E0F9010190CB
:1033C0000D928A95E1F7D9018E910E941F3F8A8361
:1033D000882319F481E0898301C019828091090151
:1033E0008823E1F321E030E03F932F93CE01029652
:1033F0009F938F933F932F93CE01820F931F9F93A1
:103400008F9382E08F9381E08F9387E58F930E9463
:103410008716EDB7FEB73B96EDBF95C08091DB03F5
:10342000882309F090C00E94B1AC8983823019F0E2
:10343000843009F088C020E430E0F8948091C10025
:103440008F738093C1008091C9008F738093C900EE
:103450008091C100877E8093C1008091C900877EE2
:103460008093C9008091C80087FF03C08091CE007F
:10347000F9CF8091C00087FF03C08091C600F9CFCB
:10348000E0910E03F0910F03E081E13021F482E03E
:10349000809301032EC0E43611F421E830E081E08E
:1034A00080930103832F99278093CD002093CC0034
:1034B0008091CD008093C5008091CC008093C400A2
:1034C0008091CA008F7D8093CA008091CA008F7E50
:1034D0008093CA008091C9008B7F8093C90080913E
:1034E000CA0084608093CA008091CA008260809381
:1034F000CA008091CA00877F8093CA008091C20071
:10350000877F8093C2008091C9008E7F8093C9001D
:103510008091C10088618093C1008091C900886159
:103520008093C9008091C10080688093C100809120
:10353000C90080688093C90010926E0010926F00DD
:1035400010927000789480917A05992784369105BD
:1035500009F4C3C085369105ACF48136910509F4B0
:103560006FC0823691052CF48B34910509F45DC04F
:1035700025C18236910509F473C08336910509F49B
:1035800087C01CC18C36910509F4F5C08D369105B4
:103590004CF48736910509F40EC18836910509F47B
:1035A000BAC00CC18437910529F08637910509F41A
:1035B000F0C004C180911003A0910E03B0910F03DD
:1035C000803140F080E1EEE5F5E00D9001928A95C2
:1035D000E1F70DC08D919D910D90BC91A02D809330
:1035E0005E0590935F05A0936005B093610580919F
:1035F00009018823E1F31F92809106018F9384E5EE
:103600008F930E9487168AEF80930B038FEF80932E
:10361000070180EA9FE00E94FB1F909303038093C1
:1036200002030F900F900F90C9C0E0910E03F0912C
:103630000F03808191819093940180939301BEC088
:10364000E0910E03F0910F03808180930801803296
:1036500018F08FE1809308018FEF80930701AEC0CF
:1036600080911003843108F0A9C0A0910E03B0919D
:103670000F0387E0EDE4F5E00D9001928A95E1F704
:10368000809151058093740784E680930A0396C065
:103690008091060390910703892B89F4E0910E0332
:1036A000F0910F03E081EE2351F08AE0E89FC00122
:1036B00011240E94FB1F90934A0580934905E091D5
:1036C0000E03F0910F0390818AE0989FC0011124AE
:1036D000909307038093060315C08FEF8093070133
:1036E000E0910E03F0910F0390818AE0989FC00152
:1036F00011249093090380930803892B19F081E02A
:103700008093180380EA9FE00E94FB1F90930303BD
:103710008093020353C08FEF80930701E0910E0363
:10372000F0910F03908197FD08C082E0809315030C
:1037300010920503109204031AC0909580917D03A6
:10374000892B80937D0391818AE0989FC001112489
:10375000909305038093040384E08093150380EA2B
:103760009FE00E94FB1F909303038093020381E07C
:103770008093190323C08FEF80930701E0910E031C
:10378000F0910F03808180937E0381E080931A0380
:1037900015C080910D03882351F0E0910E03F09144
:1037A0000F03E081E23019F4E093170307C081E0D2
:1037B0008093170303C081E080931B0310921303CF
:1037C00010920F0310920E0310920D03E3E0CE5FF0
:1037D0000C942BB2982F8091C00085FFFCCF909362
:1037E000C60008950F931F9388E18093C1008091D4
:1037F000C00082608093C0008091C1008068809387
:10380000C1008091C10080648093C10000E010E09D
:103810000093C5008AE290E08093C4008091080381
:10382000909109030E94FB1F90934C0580934B05D8
:103830008CED90E00E94FB1F9093770580937605B6
:1038400082E0809354058CE08093550510925805D2
:103850008BE0809356058FEF80935C058091030188
:1038600080935B050E9410158093570510930F03FA
:1038700000930E0310920D031F910F910895AAE17A
:10388000B0E0E5E4FCE10C940EB2809109018823DC
:1038900009F4C5C280910203909103030E940420A1
:1038A000882361F01092050310920403109209031B
:1038B00010920803109207031092060380910403EC
:1038C00090910503892B41F0809154069091550603
:1038D0000E940420882329F480911903882309F485
:1038E00060C080910901882309F45BC080911503B1
:1038F00008E817E08430A8F00E94942A80E590E060
:103900009F938F931F930F9381E08F938F9388E4FE
:103910008F930E9487162DB73EB7295F3F4F2DBF6B
:1039200034C010927F0387ED94E09F938F9387E8D4
:103930009AE29F938F93E0913905F0913A050995AA
:1039400084E190E09F938F931F930F9381E090E029
:103950009F938F9385E193E09F938F9382E08F9362
:1039600081E08F9388E48F930E94871680911503DE
:10397000982F8F5F809315032DB73EB7215F3F4F80
:103980002DBF943010F01092150380910403909194
:1039900005030E94FB1F90935506809354061092D6
:1039A000190380911A03882351F18091090188231A
:1039B00031F10E94942A80E590E09F938F9388E8EC
:1039C00097E09F938F9321E030E03F932F9389E21C
:1039D00091E09F938F933F932F938EE793E09F9374
:1039E0008F9383E08F9381E08F938CE48F930E9479
:1039F000871610921A038DB79EB70F968DBF9091C0
:103A00001703992309F449C080910901882309F417
:103A100044C0923069F580910B0B898380910C0B27
:103A20008A8380910D0B8D8380910F0B88878FEF98
:103A30008E838F83809156058B8380915C05898767
:103A400080915D058A878AE090E09F938F93CE01F5
:103A500001969F938F9381E08F938F9386E58F9349
:103A60000E9487162DB73EB7295F3F4F2DBF13C069
:103A70008AE090E09F938F9384E595E09F938F93E6
:103A800081E08F938F9386E58F930E9487168DB781
:103A90009EB707968DBF1092170380911B03882352
:103AA000E1F0809109018823C1F087E090E09F93C5
:103AB0008F938DE495E09F938F9381E08F93809116
:103AC00006018F9387E48F930E94871610921B0341
:103AD0002DB73EB7295F3F4F2DBF809108039091CE
:103AE0000903892B41F080914B0590914C050E9470
:103AF0000420882321F480911803882339F18091D0
:103B00000901882319F10E94A44182E490E09F9367
:103B10008F9382E397E09F938F9381E08F938F93AE
:103B200084E48F930E948716109218038DB79EB776
:103B300007968DBF8091080390910903009731F09B
:103B40000E94FB1F90934C0580934B0580910603C8
:103B500090910703892B09F4A0C0809149059091A9
:103B60004A050E940420882309F497C08091090126
:103B7000882309F492C08091140B9091150B9093B7
:103B80003C0580933B058091160B9091170B909309
:103B90003E0580933D052091F60A3091F70A409149
:103BA000F80A5091F90ADA01C90163E0880F991FF8
:103BB000AA1FBB1F6A95D1F7820F931FA41FB51FC1
:103BC000820F931FA41FB51F20914501309146011C
:103BD0004091470150914801BC01CD010E94E5B1DF
:103BE0003093400520933F058091FE039091FF03A1
:103BF000A0910004B091010449E0B595A79597956F
:103C000087954A95D1F7809341058091FA03909169
:103C1000FB03A091FC03B091FD0339E0B595A79596
:103C2000979587953A95D1F7809342058091060440
:103C300090910704A0910804B091090429E0B5957A
:103C4000A795979587952A95D1F7809343058091FD
:103C5000790790917A0790934505809344058EE00B
:103C600090E09F938F938BE395E09F938F9381E0F8
:103C70008F938F9383E48F930E948716809106031E
:103C8000909107030E94FB1F90934A05809349057A
:103C90002DB73EB7295F3F4F2DBF809108018F3F61
:103CA00071F1992704E0880F991F0A95E1F789526D
:103CB0009D4F8E01055F1F4F40E150E0BC01C801E0
:103CC0000E94BBAF80E190E09F938F931F930F936F
:103CD00081E090E09F938F9388E091E09F938F9392
:103CE00082E08F9381E08F9381E48F930E94871607
:103CF0008FEF809308018DB79EB70B968DBF809193
:103D000074078823D1F0809109018823B1F081E004
:103D100090E09F938F9384E797E09F938F9381E048
:103D20008F938F9382E48F930E948716109274076B
:103D30002DB73EB7295F3F4F2DBF809116038823D3
:103D4000C9F0809109018823A9F086E490E09F934F
:103D50008F9387E09AE09F938F9381E08F938F9367
:103D600080E58F930E948716109216038DB79EB739
:103D700007968DBF80917605909177050E9404206B
:103D8000882309F44CC080910901882309F447C0B5
:103D90008091A701882369F58091140B9091150BF0
:103DA00090936F0580936E058091160B9091170B81
:103DB00090937105809370058091B803809372058C
:103DC0008091B7038093730588E090E09F938F9371
:103DD0008EE695E09F938F9381E08F9383E08F939E
:103DE0008BE68F930E9487162DB73EB7295F3F4F12
:103DF0002DBF80917405853018F086E0809374059E
:103E000080912A03882319F083E690E002C087EEB0
:103E100093E00E94FB1F9093770580937605E4E082
:103E2000C65E0C942AB21F920F920FB60F92112405
:103E30002F933F935F936F937F938F939F93AF9352
:103E4000BF93EF93FF9380912C03882329F08091F7
:103E50002C03815080932C038091AE04882319F0A9
:103E600081508093AE048091340381508093340359
:103E70008F3F09F051C089E0809334038091320371
:103E80009091330301969093330380933203809192
:103E900013018F5F817080931301882349F480910F
:103EA0003103843028F4809131038F5F8093310394
:103EB000349903C081E080932A0380912D0390916F
:103EC0002E03892B11F180912D0390912E030B97D6
:103ED00050F080912D0390912E030A9790932E031A
:103EE00080932D0304C010922E0310922D03809115
:103EF0002D0390912E0320910C0130910D0182230E
:103F00009323892B41F0479A07C08FEF9FEF90933F
:103F10000D0180930C01479880912A03882309F4AE
:103F20005AC02091A701222309F055C08091E40ACC
:103F300083FF51C086B19927FC01E071F07084FFC6
:103F400013C080912F03909130030196909330031A
:103F500080932F0380912F0390913003895E9340CB
:103F6000D0F120932A0337C080912F039091300322
:103F7000892B69F180912F03909130038A569140EB
:103F800030F580912F039091300369E270E00E9438
:103F90009CB180912F0390913003860F971F9093CF
:103FA000300380932F0380912F03909130030B9760
:103FB00050F080912F03909130030A9790939401D1
:103FC0008093930104C0F0939401E09393011092C5
:103FD000300310922F03FF91EF91BF91AF919F910A
:103FE0008F917F916F915F913F912F910F900FBEB5
:103FF0000F901F9018952091320330913303280FB2
:10400000391FC9010196089520913203309133037D
:10401000821B930B892F9927869580749070089541
:10402000CF93DF930E94FB1FEC01CE010E9404207E
:104030008823D9F3DF91CF910895CF93DF930E9426
:10404000FB1FEC0109C080911901882329F090938E
:1040500019018FEC80937A00CE010E940420982FE2
:10406000882389F3DF91CF9108959FB7F8945F98E3
:104070003E9A469A8091B0008F708093B0008091F4
:10408000B00083608093B0008091B1008B73809307
:10409000B1008091B1008B608093B1001092B200AA
:1040A0008FEF8093B3008091B00080688093B00060
:1040B000809170008A7F8093700080917000826090
:1040C000809370009FBF08958AE090E00E94FB1FDC
:1040D000909376078093750782E085BD83EB84BD5E
:1040E0008FEF88BD84EB87BD86E086BD80916E0032
:1040F000816080936E00089580915A08209170012C
:1041000082FF30C0909109088CE3989FB001112480
:104110009091080880E5989FA0011124922F905853
:1041200097FD9D5F9595959586E09802C0011124B5
:1041300020910A0130910B01281B390B30930B01A0
:1041400020930A01421753072CF050930B01409320
:104150000A0108952617370784F070930B016093C6
:104160000A010895822F992736E0880F991F3A9502
:10417000E1F790930B0180930A010895EF92FF926B
:104180000F931F93CF93DF9380911008E82FFF27A1
:10419000E75BFE4F9681C0818091120120915C08FF
:1041A000813009F01FC127FF05C0C0E0D0E0E0E08A
:1041B000F0E046C0892F992787FD9095A92FB92F48
:1041C00020911A0430911B0440911C0450911D044D
:1041D000BC01CD010E9471B197FF04C061587F4FAF
:1041E0008F4F9F4F7B018C0187E015950795F794C2
:1041F000E7948A95D1F78C2F992787FD9095A92F61
:10420000B92F209116043091170440911804509151
:104210001904BC01CD010E9471B197FF04C061581F
:104220007F4F8F4F9F4FC7E09595879577956795FF
:10423000CA95D1F7F801E701C61BD70BE80BF90BBC
:1042400020918C0430918D04C901B3E0880F991F2F
:10425000BA95E1F7821B930BAA2797FDA095BA2F79
:10426000C81BD90BEA0BFB0B80916E019927AA277B
:10427000BB27BC01CD019E01AF010E9471B197FF28
:1042800004C061507E4F8F4F9F4FFC01EB01A9E0AE
:10429000F595E795D795C795AA95D1F710915A0846
:1042A00060910A0170910B0112FF05C0709311011A
:1042B0006093100118C0409110015091110180913C
:1042C0000F08282F3327CB01841B950BB9010E94BF
:1042D000B0B18091100190911101860F971F9093BA
:1042E00011018093100110FF14C080911001909172
:1042F000110197FD0F9674E0959587957A95E1F7F2
:10430000AA2797FDA095BA2FC80FD91FEA1FFB1F38
:1043100015C0809110019091110197FD0F9664E0F6
:10432000959587956A95E1F7AA2797FDA095BA2FED
:104330008C1B9D0BAE0BBF0BFD01EC0120914408C3
:10434000222321F133278091260390912703829F16
:10435000A001839F500D929F500D1124CA01AA27DE
:1043600097FDA095BA2F8C0F9D1FAE1FBF1F2F5F0B
:104370003F4F442737FD4095542FBC01CD010E948B
:10438000E5B1309327032093260304C0D09327037D
:10439000C093260380910808282F3327220F331F4C
:1043A000220F331F809126039091270382179307D2
:1043B0007CF080910908282F3327220F331F220F0A
:1043C000331F80912603909127032817390724F47F
:1043D0003093270320932603809112018F5F8093EF
:1043E000120102C127FF05C0C0E0D0E0E0E0F0E02C
:1043F00046C0892F992787FD9095A92FB92F209125
:104400001604309117044091180450911904BC010E
:10441000CD010E9471B197FF04C061587F4F8F4F4B
:104420009F4F7B018C0197E015950795F794E794D2
:104430009A95D1F78C2F992787FD9095A92FB92FA1
:1044400020911A0430911B0440911C0450911D04CA
:10445000BC01CD010E9471B197FF04C061587F4F2C
:104460008F4F9F4FFC01EB0187E0F595E795D795BE
:10447000C7958A95D1F7CE0DDF1DE01FF11F809102
:104480006D019927AA27BB27BC01CD019E01AF0171
:104490000E9471B197FF04C061507E4F8F4F9F4FB4
:1044A000FC01EB01B9E0F595E795D795C795BA956D
:1044B000D1F780916F019927A6E0880F991FAA95DF
:1044C000E1F740910E0150910F0120910F08332721
:1044D000841B950BB9010E94B0B180910E0190919F
:1044E0000F01860F971F90930F0180930E0180910B
:1044F0005A0881FF14C080910E0190910F0197FD21
:104500000F9674E0959587957A95E1F7AA2797FD20
:10451000A095BA2FC80FD91FEA1FFB1F15C08091A5
:104520000E0190910F0197FD0F9664E09595879588
:104530006A95E1F7AA2797FDA095BA2F8C1B9D0BD2
:10454000AE0BBF0BFD01EC0120914508222321F1A8
:1045500033278091240390912503829FA001839F9C
:10456000500D929F500D1124CA01AA2797FDA095C6
:10457000BA2F8C0F9D1FAE1FBF1F2F5F3F4F4427C9
:1045800037FD4095542FBC01CD010E94E5B1309319
:1045900025032093240304C0D0932503C093240350
:1045A00080910C08282F3327220F331F220F331F2F
:1045B0008091240390912503821793077CF08091CA
:1045C0000D08282F3327220F331F220F331F80910E
:1045D0002403909125032817390724F430932503E9
:1045E0002093240310921201E6E0CDB7DEB70C94BD
:1045F00028B21F920F920FB60F9211242F933F9360
:104600004F935F938F939F93EF93FF938091350325
:10461000882309F0FEC08091B00086FFC4C080915D
:10462000B0008F7B8093B0003091380320910E084A
:104630003323D9F433278DED96E0289FA001299FDD
:10464000500D389F500D1124CA012091360330912E
:104650003703821B930B90932903809328031092B6
:10466000370310923603469AD1C0231738F48AE0F4
:1046700090E09093290380932803C8C089EA93E0CF
:10468000909329038093280380919903882389F0CC
:10469000363078F4E32FFF27E75BF74F80818823DC
:1046A00041F09927880F991F880F991F87559E4FB2
:1046B0004DC0832F99278330910529F184309105CE
:1046C00034F48130910549F0029781F02FC0843095
:1046D0009105E1F00597E9F029C0809128039091B8
:1046E0002903209126033091270308C080912803D5
:1046F000909129032091240330912503820F931F69
:104700008050924023C08091B80A05C08091990AD8
:1047100002C08091C10A282F3327220F331F220F96
:10472000331F8091280390912903E8CFE32FFF27BF
:10473000EE0FFF1FE95FF54F20813181220F331FFC
:104740008091280390912903820F931F909329034E
:1047500080932803809128039091290355E08D3D93
:10476000950718F08CED95E005C08757914030F41F
:1047700087E791E0909329038093280320912803F1
:10478000309129032C5B3040309329032093280378
:104790008091360390913703820F931F90933703D4
:1047A0008093360333C08091B00080648093B00062
:1047B0008CEB90E09093290380932803809136033B
:1047C0009091370384549F4F90933703809336031F
:1047D00080912B03882321F480912B03823011F4E4
:1047E000469801C0469A809138038F5F80933803C2
:1047F000282F332780910E08992701968217930757
:104800002CF481E0809312011092380381E08093B0
:104810003503209128033091290341E02F373407D5
:1048200030F08FEF8093B3002F5F30400FC02F3FE9
:104830003105C9F0C0F0A9014F5F50404F37510515
:1048400050F480E88093B30020583040309329031F
:104850002093280312C08FEF8093B3005093290355
:10486000409328030AC0809128038093B3001092DC
:1048700029031092280310923503FF91EF919F9125
:104880008F915F914F913F912F910F900FBE0F909D
:104890001F90189510927C008FEC80937A000895F9
:1048A0008091A003609117017091180120914D0330
:1048B000882379F0CB01AA27BB27332727FD309522
:1048C000432F532FBC01CD010E9471B1DC01CB01FC
:1048D00016C084E0660F771F8A95E1F7CB01AA27FF
:1048E000BB27332727FD3095432F532FBC01CD0124
:1048F0000E9471B1DC01CB010497A109B109809339
:10490000450390934603A0934703B093480308954B
:10491000CF93DF9310924D030E94502483E090E0E8
:104920000E944B38C82FDD27C03FD10508F42A96D6
:10493000C7BD8C2F809588BD86E990E00E941D2020
:1049400080911D0190911E018152934010F0C0EFA3
:10495000D0E0C630D10510F1C7BD8C2F809588BD41
:1049600084E690E00E941D208CEE94E09F938F934C
:104970008AEE9BE19F938F93E0913905F0913A0580
:10498000099580911D0190911E010F900F900F903D
:104990000F908152934010F42197DBCFC09385078D
:1049A0006C2F83E090E00E9453388091E60780FFEF
:1049B0000AC0809185078A508C3D28F08091590566
:1049C0008064809359058FE0809316018091A00345
:1049D0008823E9F080910301873150F4CC38D10568
:1049E000B0F480EA90E08C1B9D0B6AE170E009C096
:1049F000CA3AD10560F48CEB90E08C1B9D0B6FE004
:104A000070E00E949CB1CB01815F80931601809180
:104A10001601282F332780911D0190911E01829F3E
:104A2000A001839F500D929F500D1124CA01AA2707
:104A3000BB2780931F0190932001A0932101B09385
:104A400022018CE291E00E941D20DF91CF91089518
:104A50001F920F920FB60F921124EF92FF920F93B5
:104A60001F932F933F934F935F936F937F938F93F6
:104A70009F93AF93BF93CF93DF93EF93FF93809177
:104A80006503282F3327442755278F5F80936503BD
:104A9000F9012231310508F00AC5EA5BFF4F0C9499
:104AA00037B2809178009091790046C0809178006B
:104AB00090917900EBC1809178009091790090936A
:104AC000690380936803FBC18091240490912504BD
:104AD0002091780030917900821B930B9093780796
:104AE000809377078091770790917807909373036D
:104AF0008093720303C28091780090917900209195
:104B0000260430912704821B930B90938407809393
:104B10008307809183079091840790937503809316
:104B20007403C7C480916C0390916D032091780049
:104B300030917900820F931F90936D0380936C03E3
:104B400081E0B8C480916A0390916B032091780052
:104B500030917900820F931F90936B0380936A03C7
:104B600084E0A8C480915B0883FF26C08091270160
:104B7000909128019C01220F331F280F391F40916B
:104B80007800509179008BE090E0489FB001499FF8
:104B9000700D589F700D1124CB016EE170E00E94E2
:104BA0009CB1260F371F369527953695279530935C
:104BB00028012093270142C080917B0390917C03C0
:104BC000892B91F42091780030917900C90153E04C
:104BD000880F991F5A95E1F7820F931F820F931F39
:104BE00090937C0380937B0320917800309179002F
:104BF000C90143E0880F991F4A95E1F7820F931F7F
:104C0000820F931F20917B0330917C0382179307BF
:104C100018F02E5F3F4F02C02250304030937C038B
:104C200020937B0380917B0390917C036FE170E084
:104C30000E949CB1709328016093270185E03AC4DB
:104C4000809178009091790090937A07809379070A
:104C50008091790790917A07409120045091210426
:104C6000841B950B60911F04262F332727FD309559
:104C7000821B930B90935303809352038091A00364
:104C8000882309F071C080915203909153030297D9
:104C90007CF172E04E3E57070CF0A7C020916603EE
:104CA000309167032B5F3F4F309367032093660378
:104CB000255030408091AA039091AB03845F9140CE
:104CC00030F4215F3F4F3093670320936603809158
:104CD000660390916703853691050CF486C04F5F9B
:104CE0005F4F50932104409320048456904037C076
:104CF00080915203909153038F5F9F4F0CF075C0CA
:104D000082E0473258070CF470C02091660330915E
:104D100067032550304030936703209366032B5F71
:104D20003F4F8091AA039091AB03845F914030F490
:104D30002F503040309367032093660380916603C1
:104D4000909167037FEF8C3997070CF04EC041506C
:104D5000504050932104409320048C599F4F9093CE
:104D600067038093660341C08091AD0A9091AE0ABB
:104D70008F5C9F41D4F1809152039091530302972D
:104D8000ACF02091660330916703C90101969093BE
:104D9000670380936603895893413CF166301CF4A5
:104DA0006F5F60931F04275833411BC080915203EB
:104DB000909153038F5F9F4FC4F42091660330910D
:104DC0006703C9010197909367038093660388572F
:104DD0009C4E5CF46B3F1CF0615060931F0429579C
:104DE0003C4E309367032093660380915203909169
:104DF00053039C01442737FD4095542F8091F603BF
:104E00009091F703A091F803B091F903820F931FDB
:104E1000A41FB51F8093F6039093F703A093F803A4
:104E2000B093F9032091F6033091F7034091F80312
:104E30005091F90357FF04C021503C4F4F4F5F4F33
:104E40009AE055954795379527959A95D1F7809192
:104E5000F6039091F703A091F803B091F903821B38
:104E6000930BA40BB50B8093F6039093F703A093D9
:104E7000F803B093F903F7C080916A0390916B0334
:104E80002091780030917900820F931F90936B03EB
:104E900080936A03109264030FC3209178003091CD
:104EA00079008091680390916903280F391F8FEF73
:104EB00097E0821B930B9093590380935803809142
:104EC0001501F8C280912404909125042091780066
:104ED00030917900821B930B90937807809377072A
:104EE0008091770790917807209172033091730336
:104EF000820F931F90935703809356038091140160
:104F0000D9C2809178009091790020912604309147
:104F10002704821B930B90938407809383078091CF
:104F20008307909184072091740330917503820F59
:104F3000931F9093550380935403BBC220916C033D
:104F400030916D038091780090917900280F391F7E
:104F5000220F331F220F331F30936D0320936C03F6
:104F6000C90137FD079603E0959587950A95E1F706
:104F700090935D0380935C0380916E0390916F0327
:104F8000820F931F97FD01969595879590936F03D8
:104F900080936E032091360430913704821B930B6B
:104FA0009093260180932501209162033091630341
:104FB0008091250190912601280F391F37FF02C0EB
:104FC0002F5F3F4F359527953093630320936203FE
:104FD000B7CD20916A0330916B0380917800909156
:104FE0007900280F391F220F331F220F331F3093F0
:104FF0006B0320936A03C90137FD0796A3E09595DB
:105000008795AA95E1F790935B0380935A0380916B
:10501000700390917103820F931F97FD01969595F0
:10502000879590937103809370032091340430919D
:105030003504821B930B90932401809323012091CC
:105040006003309161038091230190912401280F26
:10505000391F37FF02C02F5F3F4F3595279530939B
:1050600061032093600383E025C28091A00388231D
:1050700009F180E00E9432AB9B01AC0120503F4F10
:105080004F4F5F4F57FF06C09B01AC0121503D4F72
:105090004F4F5F4F79E055954795379527957A950E
:1050A000D1F72093390330933A0340933B03509355
:1050B0003C0310C08091D6039091D703A091D803F0
:1050C000B091D9038093390390933A03A0933B03A3
:1050D000B0933C031092650381E0809319018091A5
:1050E000490390914A03019690934A0380934903A0
:1050F000809178009091790090931E0180931D011A
:105100008091A003882309F490C080911D019091A3
:105110001E017C01002711278091450390914603D1
:10512000A0914703B0914803E81AF90A0A0B1B0B38
:10513000E0927603F092770300937803109379035B
:1051400080913804909139040097C1F00A9708F0D3
:10515000B0C180911601282F332744275527C80155
:10516000B7010E9471B1DC01CB0180931F019093C4
:105170002001A0932101B09322019BC180911601CF
:10518000282F33274427552780911F019091200114
:10519000A0912101B0912201BC01CD010E94E5B195
:1051A00080911F0190912001A0912101B0912201D5
:1051B000821B930BA40BB50B80931F0190932001CE
:1051C000A0932101B093220180911F0190912001B1
:1051D000A0912101B09122018E0D9F1DA01FB11F32
:1051E00080931F0190932001A0932101B09322018D
:1051F00080917B0790917C07A0917D07B0917E07FD
:1052000020911F01309120014091210150912201F4
:10521000821B930BA40BB50B80933D0390933E032D
:10522000A0933F03B093400344C180911D0190912E
:105230001E01AA27BB27C0917603D0917703E09186
:105240007803F0917903C80FD91FEA1FFB1FC093A1
:105250007603D0937703E0937803F09379038091FA
:105260007A038F5F80937A03803108F422C18091A2
:105270001F0190912001A0912101B09122019C0178
:10528000AD0163E0220F331F441F551F6A95D1F70C
:10529000281B390B4A0B5B0B2C0F3D1F4E1F5F1F4A
:1052A0008091450390914603A0914703B091480334
:1052B000281B390B4A0B5B0B57FF04C0295F3F4F7C
:1052C0004F4F5F4F03E055954795379527950A95C2
:1052D000D1F720931F013093200140932101509377
:1052E0002201C0917B07D0917C07E0917D07F0916E
:1052F0007E0780911F0190912001A0912101B09122
:105300002201C81BD90BEA0BFB0BC0933D03D093C2
:105310003E03E0933F03F093400320914E0330910E
:105320004F03409150035091510357FF04C0215F38
:105330003F4F4F4F5F4F14E0559547953795279551
:105340001A95D1F780914E0390914F03A09150038D
:10535000B0915103821B930BA40BB50B80934E03AA
:1053600090934F03A0935003B093510380914E0349
:1053700090914F03A0915003B09151038C0F9D1F4A
:10538000AE1FBF1F80934E0390934F03A093500313
:10539000B093510380914E0390914F03A09150031D
:1053A000B0915103B7FF03C00F96A11DB11DC4E01A
:1053B000B595A79597958795CA95D1F720913D0307
:1053C00030913E03281B390B64E0213036071CF076
:1053D00020E034E006C07CEF2030370714F420E0F2
:1053E0003CEF80914B0390914C0380914B03909143
:1053F0004C0397FF03C0909581959F4FA901F3E05F
:10540000440F551FFA95E1F78D5B9240C4F08091EF
:105410004B0390914C039C01E4E0220F331FEA956B
:10542000E1F7281B390B240F351F37FF02C0215F1E
:105430003F4F74E0359527957A95E1F717C0809135
:105440004B0390914C039C0165E0220F331F6A953A
:10545000E1F7281B390B240F351F37FF02C0215EEF
:105460003F4F45E0359527954A95E1F730934C033A
:1054700020934B038091760390917703A09178035A
:10548000B0917903B7FF03C00196A11DB11DB59579
:10549000A795979587958093760390937703A0932C
:1054A0007803B093790388E080937A0302C0109266
:1054B000650382E0809364038091640380937C00A1
:1054C00080916503882319F08FEC80937A00FF9117
:1054D000EF91DF91CF91BF91AF919F918F917F918C
:1054E0006F915F914F913F912F911F910F91FF907D
:1054F000EF900F900FBE0F901F90189590E2E8E884
:10550000F7E08FE49193815087FFFCCF089590914D
:105510007F03903540F4E92FFF27E857F84F808349
:105520009F5F90937F030895AF92BF92CF92DF92D7
:10553000FF920F931F93CF93DF9380918003882373
:1055400021F520917D0320FF0AC080917E038823EE
:1055500011F0815002C08091290180937E0321FFC8
:105560000CC090917E0380912901981719F4109234
:105570007E0303C09F5F90937E03822F992780FF55
:1055800004C081FF02C010927E030E947E2A809197
:105590007E03282F332747E85AE2E0913905F0913E
:1055A0003A058A3090F481E180937F033F932F93F3
:1055B0008EEE94E09F938F935F934F9309952DB751
:1055C0003EB72A5F3F4F2DBF11C080E180937F031C
:1055D0003F932F9383EF94E09F938F935F934F9329
:1055E00009954DB75EB74A5F5F4F4DBF20917E036F
:1055F000822F9927AA27BB27FC01449710F00C940F
:105600001036E85AFF4F0C9437B210927F0388EFA0
:1056100094E09F938F93C7E8DAE2DF93CF93E09112
:105620003905F0913A05099584E180937F030F9045
:105630000F900F900F9081E690E09F938F938CE0F6
:1056400090E09F938F9382E090E09F938F9380915F
:1056500003016AE00E9490B1892F99279F938F934D
:10566000809103010E9490B199279F938F9388E0C6
:1056700095E09F938F93DF93CF93E0913905F0915D
:105680003A05099588E280937F038DB79EB70E9601
:105690008DBF8BE698E09F938F93809101019927AE
:1056A0009F938F9380E295E09F938F93DF93CF93A7
:1056B000E0913905F0913A0509958091A703EDB77E
:1056C000FEB73896EDBF81FF12C088E380937F0359
:1056D0008AE295E09F938F93DF93CF93E091390512
:1056E000F0913A0509950F900F900F900F908091CF
:1056F0005A0599278C010071107084FF06C08CE355
:1057000080937F038FE295E09EC490919304992348
:1057100051F18CE380937F03892F99279F938F9377
:105720008CE395E09F938F93DF93CF93E0913905BE
:10573000F0913A0509951F930F939091930481E19D
:10574000989FC0011124805F924F9F938F93DF93A6
:10575000CF93E0913905F0913A0509952DB73EB701
:10576000245F3F4F36C790915905992371F08CE320
:1057700080937F03892F99279F938F9384E495E0EB
:105780009F938F93DF93CF93B5C69091880399230E
:10579000B1F08CE380937F03892F99279F938F9398
:1057A0008BE595E09F938F93DF93CF93E09139053D
:1057B000F0913A0509958DB79EB7069686C58091FA
:1057C0003D0190913E01069730F48CE380937F0376
:1057D00081E795E038C490918C0B9E3110F00C94C9
:1057E00019368CE380937F03892F99279F938F939A
:1057F0008EE795E01EC110927F038091D6039091B1
:10580000D703A091D803B091D903BC01CD0125E005
:1058100030E040E050E00E94E5B13F932F9382E9F1
:1058200095E09F938F93C7E8DAE2DF93CF93E091FF
:105830003905F0913A05099584E180937F032DB7EE
:105840003EB72A5F3F4F2DBF8091D2039091D30383
:10585000A091D403B091D503BC01CD0125E030E087
:1058600040E050E00E94E5B13F932F938FE995E02F
:105870009F938F93DF93CF93E0913905F0913A0591
:10588000099588E280937F034DB75EB74A5F5F4F0B
:105890004DBF80911D0190911E019F938F938CEAC3
:1058A00095E09F938F93DF93CF93E0913905F0912B
:1058B0003A0509958CE380937F038DB79EB70696D2
:1058C0008DBF87B599279F938F9389EB95E09F9321
:1058D0008F93DF93CF93E0913905F0913A050995C5
:1058E000EDB7FEB73696EDBF8091A003882311F483
:1058F0000C94193689E380937F0386EC95E09F939F
:105900008F93DF93CF93E0913905F0913A05099594
:105910008DE480937F030F900F900F900F908091F4
:10592000160199279F938F938AEC95E09F938F930D
:10593000DF93CF93E0913905F0913A0509952DB7A2
:105940003EB72A5F3F4F45C610927F038DEC95E02E
:105950009F938F93C7E8DAE2DF93CF93E091390505
:10596000F0913A05099584E180937F030F900F90A1
:105970000F900F9080911A0490911B04A0911C0429
:10598000B0911D04B7FF04C081509C4FAF4FBF4F73
:105990001AE0B595A795979587951A95D1F7BF9376
:1059A000AF939F938F938AED95E09F938F93DF93AF
:1059B000CF93E0913905F0913A05099588E28093FB
:1059C0007F034DB75EB7485F5F4F4DBF80911604B0
:1059D00090911704A0911804B0911904B7FF04C066
:1059E00081509C4FAF4FBF4FFAE0B595A795979563
:1059F0008795FA95D1F7BF93AF939F938F9389EED5
:105A000095E09F938F93DF93CF93E0913905F091C9
:105A10003A0509958CE380937F038DB79EB708966E
:105A20008DBF8091ED0A9091EE0A9F938F9388EF3E
:105A300095E09F938F93DF93CF93C3C3E1E0FE2E56
:105A4000C1E0D0E009E01AE09F2D969584E1989F8F
:105A5000C001112480937F03F801828193819F9379
:105A60008F932196DF93CF932197808191819F938C
:105A70008F93DF93CF9387E096E09F938F9387E890
:105A80009AE29F938F93E0913905F0913A05099539
:105A90002DB73EB7245F3F4F2DBF32E0F30E229665
:105AA0000C5F1F4F48E04F1578F60C941936109292
:105AB0007F038091020A9091030A9F938F938091B4
:105AC000050A9091060A9F938F9389E196E09F9330
:105AD0008F9307E81AE21F930F93E0913905F09135
:105AE0003A05099584E180937F038DB79EB70896A8
:105AF0008DBF8091000A9091010A9F938F938091AE
:105B00004D0A90914E0A81589F4F9F938F9389E23F
:105B100096E09F938F931F930F93E0913905F09137
:105B20003A05099588E280937F03EDB7FEB7389672
:105B3000EDBF8091DF07E82FFF27EE0FFF1FE95F22
:105B4000F54F8081918181589F4F9F938F938091D2
:105B5000DE07E82FFF27EE0FFF1FE95FF54F80817B
:105B6000918181589F4F9F938F9389E396E09F93F4
:105B70008F931F930F93E0913905F0913A050995A2
:105B80008CE380937F032DB73EB7285F3F4F2DBF37
:105B90008091E107E82FFF27EE0FFF1FE95FF54F28
:105BA0008081918181589F4F9F938F938091E007CF
:105BB000E82FFF27EE0FFF1FE95FF54F80819181EE
:105BC00081589F4F9F938F9389E496E09F938F9383
:105BD0001F930F93E0913905F0913A0509954DB760
:105BE0005EB7485F5F4F8FC410927F0389E596E0F0
:105BF0009F938F93C7E8DAE2DF93CF93E091390563
:105C0000F0913A05099584E180937F030F900F90FE
:105C10000F900F9080913604909137049F938F934B
:105C2000209136043091370437FF02C0295F3F4F7F
:105C300073E0359527957A95E1F780915C03909113
:105C40005D03821B930B9F938F9387E696E09F9350
:105C50008F93DF93CF93E0913905F0913A05099541
:105C600088E280937F038DB79EB708968DBF8091A1
:105C70003404909135049F938F9320913404309194
:105C8000350437FF02C0295F3F4F63E03595279504
:105C90006A95E1F780915A0390915B03821B930B05
:105CA0009F938F9386E796E09F938F93DF93CF9395
:105CB000E0913905F0913A0509958CE380937F03D3
:105CC000EDB7FEB73896EDBF809132049091330462
:105CD0009F938F93809132049091330420915803C5
:105CE00030915903821B930B9F938F9385E896E025
:105CF0009F938F93DF93CF93E0913905F0913A050D
:105D000009951092810361C48091810399270097BE
:105D100021F0019709F479C09BC110927F0384E9B7
:105D200096E09F938F9307E81AE21F930F93E091F9
:105D30003905F0913A05099584E180937F030F902E
:105D40000F900F900F9080912604909127049F93BD
:105D50008F9380915403909155039F938F9381EA81
:105D600096E09F938F931F930F93E0913905F091E5
:105D70003A05099588E280937F034DB75EB7485F87
:105D80005F4F4DBF80912404909125049F938F9382
:105D900080915603909157039F938F9380EB96E0E9
:105DA0009F938F931F930F93E0913905F0913A05DC
:105DB00009958CE380937F038DB79EB708968DBFBE
:105DC00080912004909121049F938F93809152039E
:105DD000909153039F938F938FEB96E09F938F93B4
:105DE0001F930F93E0913905F0913A050995809141
:105DF0007D03EDB7FEB73896EDBF83FF1CC18091E0
:105E000081038F5F8093810316C110927F0383ED1E
:105E100096E09F938F93C7E8DAE2DF93CF93E09108
:105E20003905F0913A05099584E180937F030F903D
:105E30000F900F900F9080912604909127049F93CC
:105E40008F9380912404909125049F938F9380EEEB
:105E500096E09F938F93DF93CF93E0913905F09174
:105E60003A0509952DB73EB7285F3F4F2DBF80916A
:105E7000050A9091060A892B31F48091020A9091CB
:105E8000030A892BF9F088E280937F038091020A4C
:105E90009091030A9F938F938091050A9091060A2F
:105EA0009F938F9384EF96E09F938F93DF93CF938D
:105EB000E0913905F0913A0509954DB75EB7485F15
:105EC0005F4F4DBF8091A90380FF7BC080919901F6
:105ED000803229F08F3219F08D3209F072C041E022
:105EE0004093800380911D08882319F486E08093F5
:105EF0001D0880917D03282F332720FF0BC0809140
:105F00002404909125040197909325048093240400
:105F10004093820321FF0BC08091240490912504BB
:105F2000019690932504809324044093820322FFDA
:105F30000BC0809126049091270401979093270429
:105F4000809326044093820323FF0BC08091260494
:105F50009091270401969093270480932604409300
:105F600082038DE080937F0387E097E09F938F9378
:105F7000DF93CF93E0913905F0913A0509950F90A1
:105F80000F900F900F9080918203E0913905F0916E
:105F90003A05882351F08CE380937F038BE097E0F0
:105FA0009F938F93DF93CF932AC58CE380937F03D6
:105FB0008CE197E09F938F9387E89AE29F938F936A
:105FC0001EC58DE080937F0381E397E09F938F93BD
:105FD000DF93CF93E0913905F0913A05099510923E
:105FE00080038091A9030F900F900F900F9080FD78
:105FF00025C080918203882309F18CE380937F037D
:1060000085E397E09F938F93DF93CF93E0913905DA
:10601000F0913A05099580917D030F900F900F90B4
:106020000F9082FF04C00E94574310928103809119
:106030007D0383FFFEC510928203FBC58CE3809332
:106040007F0389E497E09F938F93DF93CF93D3C42B
:1060500010928103EEC510927F03809127019091E9
:1060600028016AE070E00E94B0B19F938F93809105
:106070002701909128016AE070E00E94B0B17F93FF
:106080006F938AE597E09F938F9307E81AE21F9337
:106090000F93E0913905F0913A05099584E18093D9
:1060A0007F038DB79EB708968DBF8091860B909128
:1060B000870B6AE070E00E949CB19F938F93809160
:1060C000860B9091870B6AE070E00E949CB17F93F1
:1060D0006F938EE697E09F938F931F930F93E091BA
:1060E0003905F0913A05099588E280937F03EDB771
:1060F000FEB73896EDBF8091880B9091890B9F93E6
:106100008F9382E897E09F938F931F930F93E09173
:106110003905F0913A0509958CE380937F032DB7FB
:106120003EB72A5F3F4F2DBF80918A0B90918B0B1A
:106130009F938F9382E997E09F938F931F930F9381
:10614000E0913905F0913A05099510928103D7C184
:1061500010927F0384EA97E09F938F9307E81AE2F7
:106160001F930F93E0913905F0913A05099588E264
:1061700080937F030F900F900F900F908091DC031E
:1061800099279F938F938DEA97E09F938F931F9307
:106190000F93E0913905F0913A0509958CE38093CE
:1061A0007F038DB79EB706968DBF8091040A99270D
:1061B00001979F938F938DEB97E09F938F931F93FE
:1061C0000F93E0913905F0913A050995EDB7FEB7C7
:1061D0003696EDBF2EC510927F038DEC97E09F930E
:1061E0008F9307E81AE21F930F93E0913905F0911E
:1061F0003A05099584E180937F030F900F900F90EB
:106200000F90809102016AE00E9490B1892F992736
:106210009F938F93809102010E9490B199279F9341
:106220008F938DED97E09F938F931F930F93E09142
:106230003905F0913A05099588E280937F032DB7DF
:106240003EB7285F3F4F2DBF8091F8026AE00E9461
:1062500090B1892F99279F938F938091F8020E9484
:1062600090B199279F938F938BEE97E09F938F9395
:106270001F930F93E0913905F0913A0509958CE34E
:1062800080937F034DB75EB7485F5F4F4DBF8091EE
:10629000F9026AE00E9490B1892F99279F938F930A
:1062A0008091F9020E9490B199279F938F9389EF73
:1062B00097E09F938F931F930F93E0913905F0918F
:1062C0003A0509958DB79EB708968DBFB2C45DEDAE
:1062D000C52E53E0D52E20E030E0E90143E0F42E56
:1062E000C0937F03F60181916F0199279F938F934C
:1062F00089010F5F1F4F1F930F9387E098E09F93D3
:106300008F9387E89AE29F938F93E0913905F091FC
:106310003A0509952DB73EB7285F3F4F2DBFFA9438
:1063200064969801F7FEDCCF84C491EEC92E93E009
:10633000D92EC0E0D0E08E0183E0F82E00937F03D9
:10634000F60181916F0199279F938F932596DF9393
:10635000CF9384E198E09F938F9387E89AE29F938D
:106360008F93E0913905F0913A0509952DB73EB725
:10637000285F3F4F2DBFFA940C5E1F4F2497F7FE06
:10638000DDCF57C410927F0381E298E09F938F93F3
:1063900007E81AE21F930F93E0913905F0913A054F
:1063A000099584E180937F030F900F900F900F90D9
:1063B0008091F4029091F5029F938F938FE298E081
:1063C0009F938F931F930F93E0913905F0913A05B6
:1063D000099588E280937F034DB75EB74A5F5F4FB0
:1063E0004DBF8091F6029091F7029F938F938CE3BB
:1063F00098E09F938F931F930F93E0913905F0914D
:106400003A05099589E480937F038DB79EB7069678
:106410008DBF89E498E09F938F931F930F93E09132
:106420003905F0913A05099580917D030F900F9001
:106430000F900F9083FFFDC31092F7021092F602A7
:1064400060E070E08EE090E00E946438F2C3109249
:106450007F0381E598E09F938F9307E81AE21F93EB
:106460000F93E0913905F0913A05099584E1809305
:106470007F030F900F900F900F9080919301909158
:1064800094019F938F9389E598E09F938F931F9337
:106490000F93E0913905F0913A05099588E28093D0
:1064A0007F03EDB7FEB73696EDBF8091A10A9091BC
:1064B000A20A9F938F9387E698E09F938F931F93F1
:1064C0000F93E0913905F0913A0509958CE380939B
:1064D0007F032DB73EB72A5F3F4F2DBF8091ED0A56
:1064E0009091EE0A9F938F9385E798E09F938F9307
:1064F0001F930F93E0913905F0913A0509954DB737
:106500005EB74A5F5F4F4DBF94C310927F0383E82D
:1065100098E09F938F93C7E8DAE2DF93CF93E091FF
:106520003905F0913A05099584E180937F030F9036
:106530000F900F900F908091700199279F938F93E8
:106540008BE898E09F938F93DF93CF93E091390589
:10655000F0913A05099588E280937F038DB79EB745
:1065600006968DBF809126039091270397FD039691
:1065700095958795959587959F938F9389E998E051
:106580009F938F93DF93CF93E0913905F0913A0574
:1065900009958CE380937F03EDB7FEB73696EDBF88
:1065A0008091090899279F938F93809108089927D4
:1065B0009F938F9387EA98E09F938F93DF93CF9376
:1065C000E0913905F0913A0509952DB73EB7285F5E
:1065D0003F4F2DBF2EC38091D8078D3008F04EC09D
:1065E00010927F0385EB98E09F938F93A7E8CA2EC4
:1065F000AAE2DA2EDF92CF92E0913905F0913A05C6
:1066000009950F900F900F900F90C0E1D9E000E036
:1066100010E0F2E0FF2E802F8C5E80937F0388A92C
:1066200099278F7790709F938F9389A199278F7760
:1066300090709F938F938A8999278F7790709F93FB
:106640008F938B8199278F7790709F938F9385EC91
:1066500098E09F938F93DF92CF92E0913905F0916C
:106660003A0509954DB75EB7445F5F4F4DBFFA9449
:106670000C5E1F4FEC96F7FECECFDBC2C0E1D9E037
:10668000CC24DD24E3E0FE2EC0927F0388A9992765
:106690008F7790709F938F9389A199278F779070B0
:1066A0009F938F938A8999278F7790709F938F9369
:1066B0008B8199278F7790709F938F9386ED98E0C9
:1066C0009F938F9307E81AE21F930F93E091390588
:1066D000F0913A0509958DB79EB70C968DBFFA9447
:1066E000E4E1F0E0CE0EDF1EEC96F7FECDCF84E2C3
:1066F00080937F0387EE98E09F938F931F930F9370
:10670000E0913905F0913A05099588E380937F037C
:106710000F900F900F900F908BEE98E068C18091D2
:10672000D8078D3008F046C010927F0380EF98E0C4
:106730009F938F9377E8C72E7AE2D72EDF92CF927E
:10674000E0913905F0913A0509950F900F900F905F
:106750000F90C0E1D9E000E010E062E0F62E802F5B
:106760008C5E80937F038CA999279F938F938DA133
:1067700099279F938F938E8999279F938F938F81CA
:1067800099279F938F9380E099E09F938F93DF9257
:10679000CF92E0913905F0913A0509952DB73EB7B2
:1067A000245F3F4F2DBFFA940C5E1F4FEC96F7FE0F
:1067B000D6CF56C0C0E1D9E0CC24DD2453E0F52E7D
:1067C000C0927F038CA999279F938F938DA19927BE
:1067D0009F938F938E8999279F938F938F8199276A
:1067E0009F938F9381E199E09F938F9307E81AE23B
:1067F0001F930F93E0913905F0913A0509954DB734
:106800005EB7445F5F4F4DBFFA9484E190E0C80EDD
:10681000D91EEC96F7FED4CF84E280937F0382E208
:1068200099E09F938F931F930F93E0913905F09117
:106830003A05099588E380937F030F900F900F909E
:106840000F9086E299E09F938F931F930F93E091AF
:106850003905F0913A0509950F900F900F900F9020
:106860008EE480937F038BE299E09F938F9387E878
:106870009AE29F938F93BFC08091D8078D3008F024
:1068800067C010927F038DE299E09F938F9347E852
:10689000C42E4AE2D42EDF92CF92E0913905F091D6
:1068A0003A05099587E480937F030F900F900F902E
:1068B0000F9088E399E09F938F93DF92CF92E091BE
:1068C0003905F0913A050995FF240F900F900F902C
:1068D0000F90C0E0D0E08E01802F8C5E80937F030C
:1068E0008C2F8D5F0E9449809F938F938C2F8E5F9A
:1068F0000E9449809F938F938C2F8F5F0E944980C5
:106900009F938F938C2F0E9449809F938F9382E453
:1069100099E09F938F93DF92CF92E0913905F091A8
:106920003A0509959E012C5F3F4F8091D807992722
:10693000EDB7FEB73C96EDBF281739070CF079C1CB
:10694000F3940C5E1F4FE901F2E0FF1528F671C1C8
:10695000C0E0D0E06E0133E0F32EC0927F038C2FB5
:106960008D5F0E9449809F938F938C2F8E5F0E9432
:1069700049809F938F938C2F8F5F0E9449809F93B4
:106980008F938C2F0E9449809F938F9383E599E08A
:106990009F938F9307E81AE21F930F93E0913905B5
:1069A000F0913A0509952DB73EB7245F3F4F2DBFB3
:1069B000FA9444E150E0C40ED51E2496F7FECDCFE4
:1069C00088E380937F0384E699E09F938F931F93DE
:1069D0000F93E0913905F0913A0509958CE4809385
:1069E0007F030F900F900F900F9088E699E09F9390
:1069F0008F931F930F93E0913905F0913A05099514
:106A00000F900F900F900F9014C110927F038AE6A1
:106A100099E09F938F9387E89AE29F938F93E091F9
:106A20003905F0913A05099584E180937F03FF24AD
:106A30000F900F900F900F9003E119E0C0E0D0E0AD
:106A400056E0F51619F08CE0F81689F489E799E01C
:106A50009F938F9387E89AE29F938F93E0913905F4
:106A6000F0913A0509950F900F900F900F90F80153
:106A7000808147E85AE2E0913905F0913A0587FFB5
:106A800011C02196DF93CF9321978CE799E09F93D4
:106A90008F935F934F9309952DB73EB72A5F3F4F72
:106AA0002DBF0BC081E899E09F938F935F934F9325
:106AB00009950F900F900F900F90F3942196015F1E
:106AC0001F4F3FE03F1508F0BBCFB3C08091D80700
:106AD0008D3008F065C010927F0385E899E09F93A0
:106AE0008F9327E8A22E2AE2B22EBF92AF92E091B6
:106AF0003905F0913A050995FF240F900F900F90FA
:106B00000F9094E0C92ED12CC0E1D9E000E010E054
:106B1000802F8C5E80937F038AAD99279F938F93FC
:106B200089AD99279F938F938BA599279F938F93D7
:106B30008AA599279F938F938C8D99279F938F93E5
:106B40008B8D99279F938F938D8599279F938F93F3
:106B50008C8599279F938F9381E999E09F938F93D9
:106B6000BF92AF92E0913905F0913A050995809175
:106B7000D80799274DB75EB74C5E5F4F4DBFC8161B
:106B8000D9060CF056C0F3940C5E1F4FEC9684E0CF
:106B900090E0C80ED91E92E09F1508F0B9CF49C009
:106BA000C0E1D9E000E010E083E0F82E00937F031D
:106BB0008AAD99279F938F9389AD99279F938F9340
:106BC0008BA599279F938F938AA599279F938F933E
:106BD0008C8D99279F938F938B8D99279F938F935C
:106BE0008D8599279F938F938C8599279F938F935A
:106BF00085EB99E09F938F9387E89AE29F938F9319
:106C0000E0913905F0913A050995EDB7FEB7749614
:106C1000EDBFFA940C5E1F4FEC96F7FEC7CF09C08C
:106C200080912901281719F42150209329011092ED
:106C30007E0310927D03DF91CF911F910F91FF9002
:106C4000DF90CF90BF90AF900895F999FECF92BD9D
:106C500081BDF89A80B599270895F999FECF1FBA9A
:106C600092BD81BD60BD0FB6F894FA9AF99A0FBE35
:106C700008954AEA20E030E02617370740F4FC0187
:106C80008191480F2F5F3F4F26173707C8F3842F96
:106C900099270895EAEA40E050E04617570778F44C
:106CA0009C01F999FECF32BD21BDF89A80B5E80F5D
:106CB0004F5F5F4F2F5F3F4F4617570790F38E2F61
:106CC0009927089581E08093DC0782E08093DB07B9
:106CD00083E08093DA0784E08093DD0785E080938A
:106CE000DE0786E08093DF0787E08093E00788E097
:106CF0008093E10789E08093E2078AE08093E307CD
:106D00008BE08093E4078CE08093E50708959AE692
:106D10009093D9078CE0EDE5F8E011928A95E9F7B8
:106D20008AE08093F90710921D088BE18093F507A4
:106D30008EE480931A0880931B0880E280931C08DD
:106D4000109259089093E60782E780935B0880E5EC
:106D500080935C0886E08093000810923E081092B1
:106D60003B0838E03093F30786EE8093F40780E425
:106D70008093F60785E08093E9072EE12093E707EB
:106D80008EE68093EE079091A003992391F084E121
:106D90008093EA0788E28093E8072093EC0781E07C
:106DA0008093ED078FE78093EF078CE38093410892
:106DB0000DC08FE08093EA072093E8079093EC07DB
:106DC0003093ED079093EF07909341088FE0809305
:106DD000EB0710924F088CE0809350081092020845
:106DE00010920308109204081092050810921F08D0
:106DF00010922008109221081092220890E8909397
:106E0000060842E340930708E2E0E0935A0888E16D
:106E10008093080886EE8093090883E080930E082B
:106E20005DE7509311085093120850931308909304
:106E30000A0875E570930B0866E460930C088CED06
:106E400080930D088CE380930F08109210089AEA43
:106E5000909323088CEC8093250810922708909338
:106E6000280898E290932408909326081092290805
:106E70001092540840935508409314082AE5209333
:106E800015084093160836E030932A0884E680936C
:106E90002B0880932C0820932D0888E780932E08D8
:106EA000909332088BE480932F087093300880937E
:106EB00031083093330888E08093340840933508D4
:106EC0008AE2809336081092370810923A089CE8BC
:106ED00090933808E093390810923C0810923D08CE
:106EE00081E48093FE072093FF0710923F081092E1
:106EF000400886E9809342085093170884E3809302
:106F00001808109243081092440810924508909374
:106F10004608609347089093480860934908109288
:106F20004A0810924B0810924C0810924D0810928B
:106F30004E081092510880E28093FD078FE1809304
:106F400053088EE18093520880EF80935608109288
:106F500057081092580808950E9487368AE0809357
:106F6000F00780E18093F10726E02093F2079AE58D
:106F70009093F70788E78093F8079093FA07809338
:106F8000FB072093FC0780E2809301088CE3809349
:106F900019088BE480931E0886E491E6A3E7B4E722
:106FA00080935D0890935E08A0935F08B09360089B
:106FB00060E970E089ED97E00E94393680936908B6
:106FC0000895CF93DF930E94873688E08093F0077F
:106FD00030E13093F10726E02093F20794E6909396
:106FE000F70788E78093F8079093FA078093FB07E9
:106FF0002093FC073093010886E48093190880935E
:107000001E08ADE5B8E085E0EAE2F1E0ED010190AF
:1070100009928A95E1F760E970E0CD0184589040CB
:107020000E94393680936908DF91CF9108950E94BC
:10703000873626E02093F0078AE08093F10784E00A
:107040008093F20794E69093F70788E78093F80718
:107050009093FA078093FB072093FC0780E18093CD
:10706000010886E48093190880931E0885E491E660
:10707000A3E7B9E780935D0890935E08A0935F084B
:10708000B093600860E970E089ED97E00E943936BE
:10709000809369080895F999FECF92BD81BDF89A51
:1070A00080B599270895F999FECF1FBA92BD81BD89
:1070B00060BD0FB6F894FA9AF99A0FBE089565E28A
:1070C00076E30E94FFAF08954DE256E30E9439B087
:1070D0000895EF92FF920F931F93CF93C82F815083
:1070E000853008F0C3E081E9C89F8001112483ED59
:1070F000E82E8FEFF82EE00EF11E60E970E0C70178
:107100000E944A36682F98012D593F4F8FB3992717
:10711000AC014270507081FDF9CF32BD21BDF89AAB
:1071200080B5861711F0CA0129C08FB399279C0139
:107130002270307081FDF9CFF2BCE1BCF89A80B5C5
:107140008A3611F0C9011AC081E9C89FC001112413
:107150008D9725E236E341E950E0BC0189ED97E0E7
:107160000E94DAAF0E9403780E94CCA98091560851
:107170008E3B10F41092560881E090E0CF911F9161
:107180000F91FF90EF900895282F863010F025E0A2
:1071900003C0882309F421E020930101F999FECF6F
:1071A0001FBA82E090E092BD81BD20BD0FB6F89479
:1071B000FA9AF99A0FBE0895CF93C82F8091D907F4
:1071C0008A3609F051C0C63010F0C5E003C0CC23A8
:1071D00009F44AC00E949EAE80915C0882FF07C0FD
:1071E0008091FE07843618F080E58093FE0760E901
:1071F00070E089ED97E00E9439368093690881E953
:10720000C89FC00111242DE236E341E950E069ED49
:1072100077E08D970E9417B02DE236E34CE050E006
:107220006AED77E080E590E00E9417B06CE070E0D6
:107230008AED97E00E943936282FF999FECF1FBAC0
:107240008CE590E092BD81BD20BD0FB6F894FA9A0E
:10725000F99A0FBE8C2F0E94C4380E9403780E94B6
:10726000CCA981E090E002C080E090E0CF91089549
:107270006DE470E088EE93E00E944A36482F8FB3A9
:1072800099279C012270307081FDF9CF85E394E04D
:1072900092BD81BDF89A80B5841779F48FB3992790
:1072A0009C012270307081FDF9CF88EE93E092BD91
:1072B00081BDF89A80B5813011F0C901089525E2A9
:1072C00036E34EE450E068EE73E08AE698E00E9410
:1072D000DAAF81E090E0089580916A088130A9F4E6
:1072E0006DE470E08AE698E00E9439368093B70832
:1072F0002DE236E34EE450E06AE678E088EE93E073
:107300000E9417B081E090E0089580E090E0089539
:10731000CF93DF9381E080936A08EAE6F8E08FE09C
:10732000158616861786108A8150349687FFF8CF07
:1073300080E480937708809378081092790880938E
:107340007A0880937B0890EC90937C0810927D08DB
:1073500080937E0880937F08109280089093810824
:107360009093820880938308109284088093850804
:1073700090938608ABE6B8E08CE0E0E3F1E0ED0145
:10738000019009928A95E1F76DE470E0CD010197D3
:107390000E9439368093B708DF91CF910895F9990B
:1073A000FECF82E090E092BD81BDF89A80B5282F93
:1073B000863078F023E0322FF999FECF1FBA82E0B1
:1073C00090E092BD81BD30BD0FB6F894FA9AF99A5B
:1073D0000FBE20930101822F992708951F93CF9309
:1073E000C82F162F863010F0C5E003C0882309F49B
:1073F000C1E08C2F99278230910541F083309105AF
:1074000044F4019731F40E94AC3705C00E94E13783
:1074100002C00E9417381123E1F06CE070E080E5B3
:1074200090E00E944A36282FF999FECF8CE590E033
:1074300092BD81BDF89A80B5821759F425E236E3F2
:107440004CE050E060E570E08AED97E00E94DAAF32
:1074500002C00E9462368C2F0E94DC38CF911F91AF
:107460000895DF92EF92FF920F931F93CF93FF2423
:10747000DF2CEF2C81E190E00E944B3890910301CA
:107480009817A9F15C9A8AED99E09F938F938AEE01
:107490009BE19F938F93E0913905F0913A0509950F
:1074A000809103010F900F900F900F90863169F437
:1074B00081E190E00E944B38853139F44C9905C048
:1074C0006F2D81E090E00E9453386091030181E1CB
:1074D00090E00E94533888E190E028E00FB6F894DD
:1074E000A895809360000FBE20936000FFCF81E0DD
:1074F00090E00E944B388A3611F031E0E32E6CE0C8
:1075000070E080E590E00E944A36C82FF999FECFDE
:107510008CE590E092BD81BDF89A80B58C1711F48E
:1075200021E0D22EC1E001E010E0EE2029F48C2F02
:107530000E9469388823B9F591E0F92E1F930F93C3
:1075400082E09AE09F938F938AEE9BE19F938F93C3
:10755000E0913905F0913A0509952DB73EB72A5FBC
:107560003F4F2DBF0130110521F00230110521F0F0
:1075700006C00E94AC3705C00E94E13702C00E94DD
:107580001738DD2059F025E236E34CE050E060E5A5
:1075900070E08AED97E00E94DAAF02C00E94623686
:1075A0008C2F0E94DC38CF5F0F5F1F4FC63008F46E
:1075B000BCCFFF2019F083E00E94C4380E94CF396D
:1075C000C82F0E9469388C2F99279F938F9388E248
:1075D0009AE09F938F930AEE1BE11F930F93E09124
:1075E0003905F0913A05099581E090E00E944B3809
:1075F0002DB73EB72A5F3F4F2DBF8F3F21F00E942E
:107600003839882399F481E49AE09F938F931F93EC
:107610000F93E0913905F0913A0509950E94883958
:107620000E946C390F900F900F900F90EE2029F070
:107630006AE681E090E00E9453381092D80790E00B
:10764000EAE6F8E0CFE08585181614F49F5F04C0E1
:10765000158616861786108AC1503496C7FFF3CF59
:107660009093D807892F99279F938F938BE698E063
:107670009F938F9382E69AE09F938F931F930F932C
:10768000E0913905F0913A0509950E94240D8DB7D6
:107690009EB708968DBFCF911F910F91FF90EF90ED
:1076A000DF900895982F2FB7F8943998389A88B1B9
:1076B000836088B98091B9008C7F8093B9008AE299
:1076C0008093B80010928D0310928B0310928A035E
:1076D0009923B1F0E0E1F9E08FE01082118212828B
:1076E00013821482158216821782168610861186DE
:1076F000128613861486158681503F9687FFEDCF3C
:1077000078942FBF089510928D0384E98093BC0074
:1077100080E88093BC001092BD001092BA001092D5
:10772000BB001092B9001092B8001092890380E05B
:107730000E94523B1092BB0085E88093BC00809170
:10774000870382608093870308951F920F920FB67C
:107750000F9211242F933F938F939F93EF93FF9357
:1077600080918D03282F33278F5F80938D032330E3
:10777000310509F41CC1243031055CF42130310598
:1077800009F452C0223031050CF097C0232B71F060
:1077900035C32530310509F470C1253031050CF4AD
:1077A0001EC12630310509F436C228C381E080931A
:1077B000890309C080918B03803190F480918B0301
:1077C0008F5F80938B0380918B03E82FFF27EE0F51
:1077D000FF1FEE0FFF1FE659F74F8585181654F768
:1077E00080918B038F7080938B03809193038F5FC5
:1077F0008093930390913F01981770F41092930334
:10780000109286031092850385E080938D0380910A
:107810008A03880F8D5A04C080918B03880F8E5A7B
:107820008093BB0085E826C180918B039927FC01DA
:1078300024E0EE0FFF1F2A95E1F7E81BF90BE05F4C
:10784000F64F81818093BB0085E88093BC008091D6
:107850008B039927FC01E295F295F07FFE27E07FEC
:10786000FE27E81BF90BE05FF64F808180FF9DC08B
:1078700080918B039927FC01E295F295F07FFE271A
:10788000E07FFE27E81BF90BE05FF64F828188233B
:1078900029F08091D807873008F4C6C2809185030B
:1078A00090918603892B09F0BFC280918303909148
:1078B0008403892B09F0B8C278C080918B0321E042
:1078C00030E002C0220F331F8A95E2F780918303D4
:1078D0009091840328233923232B89F080918B03F3
:1078E0009927FC01E295F295F07FFE27E07FFE27C5
:1078F000E81BF90BE05FF64F80E184830FC08091B5
:107900008B039927FC01E295F295F07FFE27E07F3B
:10791000FE27E81BF90BE05FF64F148280918B0382
:107920009927FC01E295F295F07FFE27E07FFE2784
:10793000E81BF90BE05FF64F8481282F3327220FD5
:10794000331F220F331F220F331F80918B03992780
:10795000FC0134E0EE0FFF1F3A95E1F7E81BF90B4D
:10796000E05FF64F82818770822B8093BB0085E8B1
:107970008093BC0020918B0381E090E002C0880FCF
:10798000991F2A95E2F7209185033091860382237F
:107990009323892B51F088E099E090939103809391
:1079A000900388E0809392033FC284E024C2E09178
:1079B0009003F091910381918093BB0085E88093BF
:1079C000BC00F0939103E093900380919203815067
:1079D00080939203882309F427C283E00CC280912C
:1079E000B900803379F580918E03882329F4809142
:1079F0008B038F5F80938E0380918B039927FC010B
:107A0000E295F295F07FFE27E07FFE27E81BF90B59
:107A1000E05FF64F838199278F7790708F379105BC
:107A20008CF480918B039927FC01E295F295F07F0D
:107A3000FE27E07FFE27E81BF90BE05FF64F83810E
:107A40008F5F838310928D0384E98093BC008AE06A
:107A500090E090933E0180933D0180918B038F5F76
:107A600080938B0310928D03809187038E7F809388
:107A7000870385EA8093BC00D7C18091B900803428
:107A8000D9F180918A039927FC01E295F295F07F64
:107A9000FE27E07FFE27E81BF90BE05FF64F8381AE
:107AA0008F77838380918A038F5F80938A0380918D
:107AB0008A038031A0F010928A03109284031092FE
:107AC000830380918F038F5F80938F03803138F021
:107AD00010928F03809187038D7F8093870380911D
:107AE000870381608093870310928D0384E98093DC
:107AF000BC001092890388C080918A039927FC01F9
:107B0000E295F295F07FFE27E07FFE27E81BF90B58
:107B1000E05FF64F83818068838380918A03992791
:107B2000FC01E295F295F07FFE27E07FFE27E81B3F
:107B3000F90BE05FF64F808180FF42C080918A039D
:107B40009927FC01E295F295F07FFE27E07FFE2762
:107B5000E81BF90BE05FF64F848199270097D9F075
:107B6000409709F048C088E099E090939103809392
:107B7000900388E08093920380918A039927FC0107
:107B800034E0EE0FFF1F3A95E1F7E81BF90BE05FD9
:107B9000F64F148230C090918A038FE0989FC00105
:107BA00011248B5E964F9093910380939003909154
:107BB0008A0380918F039817D9F48091400119C0EE
:107BC00090918A038FE0989FC00111248B5E964F9D
:107BD00090939103809390038091870381FD06C069
:107BE00090918A0380918F03981711F482E001C06D
:107BF00081E08093920380919203813011F485E8B3
:107C000001C085EC8093BC0080918E038093880333
:107C100010928E0309C1E0919003F091910380913D
:107C2000BB00808380919003909191030196909383
:107C300091038093900380919203815080939203EB
:107C4000823010F085ECD4C0813011F485E8D0C0CA
:107C50008091870381FF7DC08091A90380FD79C059
:107C600080918A039927FC0124E0EE0FFF1F2A95DB
:107C7000E1F7E81BF90BE05FF64F868199278C7FCF
:107C80009070883F910591F480918A039927FC01B7
:107C9000E295F295F07FFE27E07FFE27E81BF90BC7
:107CA000E05FF64F8081816080830FC080918A03FE
:107CB0009927FC01E295F295F07FFE27E07FFE27F1
:107CC000E81BF90BE05FF64F108280918A03992739
:107CD000FC01E295F295F07FFE27E07FFE27E81B8E
:107CE000F90BE05FF64F8681883F89F480918A0323
:107CF0009927FC01E295F295F07FFE27E07FFE27B1
:107D0000E81BF90BE05FF64F8081866021C080910F
:107D10008A039927FC01E295F295F07FFE27E07F28
:107D2000FE27E81BF90BE05FF64F8681893F89F457
:107D300080918A039927FC01E295F295F07FFE2756
:107D4000E07FFE27E81BF90BE05FF64F808184603F
:107D500080838091A90381FF23C080918A039927A2
:107D6000FC0134E0EE0FFF1F3A95E1F7E81BF90B39
:107D7000E05FF64F86818E3F98F480918A039927C1
:107D8000FC0124E0EE0FFF1F2A95E1F7E81BF90B39
:107D9000E05FF64F86858F5F868789E08093B0012C
:107DA00080918A038F5F80938A0380918A03803158
:107DB000A0F010928A0310928403109283038091A2
:107DC0008F038F5F80938F03803138F010928F0381
:107DD000809187038D7F8093870310928D0384E9C0
:107DE0008093BC00809187038160809387031AC0D1
:107DF0008093BC0086E080938D0316C010928D03A3
:107E000084E98093BC00809187038160809387031D
:107E10008AE090E090933E0180933D0110928B03A5
:107E200010928A0310928903FF91EF919F918F9195
:107E30003F912F910F900FBE0F901F9018950F93A9
:107E40001F93CF93DF93182F8091DB03882321F4B6
:107E500080910B03882319F081E090E091C01131EB
:107E600008F08CC01123C9F0812F9927FC0144E050
:107E7000EE0FFF1F4A95E1F7E81BF90BE05FF64FA5
:107E80003C9780813C9688230CF078C03F97808196
:107E900080FD03C083E090E073C0809108099927BA
:107EA0008B709070029719F084E090E069C067E0F1
:107EB00070E088E099E00E94393690910F098917A7
:107EC00019F085E090E05CC000913F0180E1809373
:107ED0003F0184E690E090933E0180933D010E9433
:107EE000FB1FEC018091870380FD05C0CE010E943D
:107EF00004208823B9F3112319F48FEF9FE00BC0FE
:107F0000212F33272150304081E090E002C0880FBC
:107F1000991F2A95E2F79093860380938503109228
:107F20008B0310928A0388EE93E00E94FB1FEC0102
:107F300010928D03809187038E7F8093870385EA5B
:107F40008093BC008091870380FD05C0CE010E9414
:107F500004208823B9F38091850390918603892BAF
:107F600029F0CE010E940420882311F300933F01E1
:107F70008091850390918603009711F082E090E054
:107F8000DF91CF911F910F9108950F931F93CF937E
:107F9000DF93982F8091DB03882321F480910B03DA
:107FA000882319F081E090E07BC09131B0F49923EF
:107FB00019F486E090E074C0C92FDD27FE0154E07B
:107FC000EE0FFF1F5A95E1F7EC1BFD0BE05FF64F3C
:107FD0003C9780813C9687FD03C082E090E060C0C2
:107FE0003F97808180FD03C083E090E059C088EE18
:107FF00093E00E94FB1F8C018091870380FD05C0E8
:10800000C8010E9404208823B9F3219781E090E001
:1080100002C0880F991FCA95E2F79093840380935A
:10802000830310928B0310928A0310920809109216
:108030000F0910928D03809187038E7F80938703B1
:1080400085EA8093BC008091870380FD05C0C8014C
:108050000E9404208823B9F38091830390918403C4
:10806000892B29F0C8010E940420882311F38091F4
:10807000080999278B709070029719F084E090E0BE
:108080000FC067E070E088E099E00E943936909177
:108090000F09891719F085E090E002C080E090E0B8
:1080A000DF91CF911F910F910895CF93DF9380E0DF
:1080B00021E83FEFCFE4DAE0E7E0FAE0DF018530E6
:1080C00020F411961C921E9202C0318320831982E3
:1080D000188222968F5F12963296833280F38FE752
:1080E00090E09093460A8093450A81E89FEF909331
:1080F000440A8093430A1092480A1092470A109249
:108100003304109232041092350410923404109209
:10811000370410923604DF91CF9108951F920F9289
:108120000FB60F9211240F931F932F933F934F93EA
:108130005F936F937F938F939F93AF93BF93CF93EF
:10814000DF93EF93FF9340918600509187008091D9
:10815000950390919603481B590B8091860090914E
:1081600087009093960380939503CA018D549440A1
:10817000A0919703B0919803835F9A4158F480913E
:1081800097038093040A149714F01092430181E03E
:1081900090E0C1C0A131B1050CF0C1C0CA018B5F34
:1081A0009040845B914008F0B1C080914101909172
:1081B0004201481B590BE0914308EE2351F0FF2781
:1081C000EE0FFF1FE95FF54F8081918184369105A5
:1081D000ECF4FD01EA0FFB1FE95FF54F808191810F
:1081E000FA01E81BF90BCF01F7FF03C090958195C9
:1081F0009F4F06975CF48091DC03883C20F48091CB
:10820000DC03865F01C088EC8093DC03FD01EA0F8C
:10821000FB1FE95FF54F808191819C01220F331F85
:10822000280F391F240F351F37FF02C02D5F3F4F26
:10823000E901D595C795D595C795CA0101968C17C3
:108240009D0714F4219706C041505040C417D5072C
:108250000CF421968091DC03833CD8F08D010A0F49
:108260001B1FF801E95FF54F808191819E01281B5A
:10827000390BC90163E070E00E94B0B1CB01880FF7
:10828000991F860F971F015B154FF801918380831B
:1082900007C0AA0FBB1FA15BB54F11961C921E927F
:1082A000E0919703F0919803EE0FFF1FE95FF54F00
:1082B000D183C0838091DC03823340F58091DA075B
:1082C000E82FFF27EE0FFF1FE95FF54F11821082A5
:1082D0008091DB07E82FFF27EE0FFF1FE95FF54FC7
:1082E000118210828091DD07E82FFF27EE0FFF1F1C
:1082F000E95FF54F118210828091DC07E82FFF279C
:10830000EE0FFF1FE95FF54F1182108280919703F6
:108310009091980301969093980380939703FF910F
:10832000EF91DF91CF91BF91AF919F918F917F910D
:108330006F915F914F913F912F911F910F910F90EE
:108340000FBE0F901F9018958091140B9091150BF4
:1083500090933507809334078091160B9091170BFB
:1083600090933707809336078091E80A9091E90A45
:1083700097FD0396959587959595879590933907E1
:10838000809338078091FA0A9091FB0A97FD039633
:10839000959587959595879590933B0780933A0798
:1083A0008091320490913304209158033091590305
:1083B000821B930B90933D0780933C078091D603DB
:1083C0009091D703A091D803B091D903BC01CD01FE
:1083D0002AE030E040E050E00E94E5B130933F07F2
:1083E00020933E078091790790917A0790934107F7
:1083F0008093400780919301909194019093450759
:10840000809344078091270190912801909347071A
:10841000809346078091DC039927909349078093C6
:1084200048078091A10A9091A20A90934B078093EC
:108430004A0780911109992790934D0780934C0723
:1084400080912009992790934F0780934E07809140
:108450002F099927909351078093500780913E09E7
:108460009927909353078093520780912603909108
:10847000270390935D0780935C078091C0039091E0
:10848000C10390935F0780935E078091860B909164
:10849000870B909361078093600780918A0B90917E
:1084A0008B0B90936307809362078091D203909126
:1084B000D303A091D403B091D503BC01CD012AE030
:1084C00030E040E050E00E94E5B130936507209332
:1084D000640780918C0B992790936F0780936E07A8
:1084E0008091840490918504909371078093700724
:1084F0008091820490918304909373078093720714
:1085000080915905882321F480915A05882321F010
:1085100080913307816003C0809133078E7F809301
:1085200033070895EF92FF920F931F93CF93DF933A
:10853000182F7B010CE08091DB038823E9F5809103
:108540000301893111F4299801C0299A11501F3F64
:1085500061F1F0922E03E0922D03E70180912D034B
:1085600090912E03892B11F4209781F38091310390
:10857000882361F01092310380912D0390912E0396
:10858000892B09F421970E94B9AE0150002331F4E0
:108590000E94D677882311F00CE0E0CF80912C0365
:1085A0008823E1F60E946C72D9CF80910301893152
:1085B00011F4299A01C02998E6E0CDB7DEB70C94F2
:1085C00028B2EF92FF920F931F9310927A0080913E
:1085D0005C0390915D039093A80A8093A70A809111
:1085E0005A0390915B0390939D0A80939C0A80911B
:1085F0005803909159039093F00A8093EF0A2091C9
:10860000540330915503C901880F991F880F991F92
:10861000820F931F820F931F9093E90A8093E80AB9
:108620002091560330915703C901880F991F880F75
:10863000991F820F931F820F931F9093FB0A8093C1
:10864000FA0A8FEC80937A0080911A089927AA275A
:10865000BB2744ECE42E49E0F42E012D112DBC0182
:10866000CD01A80197010E9471B1DC01CB0180937B
:10867000890190938A01A0938B01B0938C01809122
:108680001B089927AA27BB27BC01CD010E9471B105
:10869000DC01CB018093850190938601A093870133
:1086A000B09388011F910F91FF90EF9008958091F2
:1086B00036049091370490932D0480932C0480917C
:1086C00034049091350490932B0480932A04809174
:1086D000320490913304909329048093280460918C
:1086E00026047091270484E090E00E946438609131
:1086F00024047091250486E090E00E946438609123
:108700002C0470912D0482E190E00E946438609105
:108710002A0470912B0484E190E00E9464386091F7
:1087200028047091290486E190E00E94643808953D
:10873000A0E0B0E0EEE9F3E40C9404B2782E21E07E
:10874000622EEE24FF24570147018701109259053C
:10875000F0922704E0922604F0922504E09224048B
:10876000F0922104E092200410921F04F09237044A
:10877000E0923604F0923504E0923404F09233042F
:10878000E092320410926B0110926A0110924D0334
:1087900023E0821729F48091A70382608093A703C6
:1087A0000E94E14284E690E00E941D200E94E14286
:1087B0008091E60780FF14C080911D0190911E01F9
:1087C000875B934058F480911D0190911E018E5E4D
:1087D000924020F080914D03882311F00E9488245C
:1087E000C0911D01D0911E0187B58B5F87BD87B5F4
:1087F000809588BD9FE1C92E8AE090E00E941D20EF
:108800008091580390915903E80EF91E80915C0302
:1088100090915D03A80EB91E80915A0390915B035D
:10882000880E991E8091790790917A07080F191F79
:10883000CA94C7FEE1CF80911D0190911E01825F15
:10884000934080F480911D0190911E01459750F056
:1088500080911D0190911E01C81BD90BD093180166
:10886000C093170187B5855087BD87B5809588BDB2
:108870009501205F3F4F3695279536952795309384
:10888000370420933604C4014096969587959695B3
:108890008795909335048093340440E150E0E40ED2
:1088A000F51EB5E0F694E794BA95E1F7F09233043B
:1088B000E0923204040F151FA5E016950795AA95BE
:1088C000E1F71093210400932004909331048093E6
:1088D000300430932F0420932E0452E0751629F5AE
:1088E0008091E80A9091E90A97FF03C090958195DD
:1088F0009F4F6CE070E00E94B0B1709327046093CA
:1089000026048091FA0A9091FB0A97FF03C0909584
:1089100081959F4F6CE070E00E94B0B17093250488
:10892000609324040E945743AEC084E090E00E940C
:108930005F38909327048093260486E090E00E949D
:108940005F389C0190932504809324048091260431
:10895000909127048150984018F421503840A0F19C
:1089600083E89AE09F938F938AEE9BE19F938F9386
:10897000E0913905F0913A0509958091E80A9091C6
:10898000E90A97FF03C0909581959F4F6CE070E0D6
:108990000E94B0B170932704609326048091FA0A74
:1089A0009091FB0A97FF03C0909581959F4F6CE0D3
:1089B00070E00E94B0B17093250460932404662493
:1089C0000F900F900F900F9082E190E00E945F381F
:1089D00090932D0480932C0484E190E00E945F38F2
:1089E00090932B0480932A0486E190E00E945F38E4
:1089F0009C0190932904809328048091A70381FF10
:108A000042C040912C0450912D04CA0180509941DC
:108A100081589C40A0F480912A0490912B0465E237
:108A20008138960760F469E18030960740F064E091
:108A3000213B360720F463E020323607C0F48BE98F
:108A40009AE09F938F938AEE9BE19F938F93E0919F
:108A50003905F0913A05099566248091A7038D7F29
:108A60008093A7030F900F900F900F900CC050931E
:108A70003704409336049093350480933404309344
:108A800033042093320412BC11BC1092A80A109235
:108A9000A70A10929D0A10929C0A1092F00A109256
:108AA000EF0A88EC90E00E941D2080915403909181
:108AB00055039C01220F331F220F331F280F391F2C
:108AC000280F391F3093E90A2093E80A8091560352
:108AD000909157038C01000F111F000F111F080FF9
:108AE000191F080F191F1093FB0A0093FA0A8091AF
:108AF000F507C82EDD24EE24FF24442737FD4095DA
:108B0000542FC701B6010E9471B14B015C01609303
:108B10001A0470931B0480931C0490931D04980105
:108B2000442737FD4095542FC701B6010E9471B10B
:108B3000DC01CB018093160490931704A0931804D2
:108B4000B093190480920E0490920F04A092100426
:108B5000B092110480930A0490930B04A0930C0428
:108B6000B0930D04109206041092070410920804AA
:108B70001092090400919301109194011093F50350
:108B80000093F4038FEF9FEF9093920180939101F4
:108B900084E690E090938E0180938D0180911A0875
:108BA0009927AA27BB27BC01CD0124EC39E040E07E
:108BB00050E00E9471B1DC01CB018856954CAF4F5B
:108BC000BF4F8093890190938A01A0938B01B0934A
:108BD0008C0180911B089927AA27BB27BC01CD01D6
:108BE0000E9471B1DC01CB018856954CAF4FBF4F4D
:108BF0008093850190938601A0938701B0938801AB
:108C0000C801AA2797FDA095BA2F20914501309160
:108C100046014091470150914801BC01CD010E949D
:108C200071B1DC01CB018093F60A9093F70AA0930F
:108C3000F80AB093F90A1092F1031092F0030E941F
:108C40000378772029F08091A90384608093A90399
:108C50008FEF8093760B1092770B80E28093780BE6
:108C600084E68093DC0380912B03882311F0579ACC
:108C700017C080915A08992780FF05C082FF03C062
:108C800080EE9EE202C080E091E190930B01809320
:108C90000A0181E0809312010E94BE200E94BE2042
:108CA00080911A0490911B04A0911C04B0911D04A2
:108CB000E0904501F0904601009147011091480174
:108CC000BC01CD01A80197010E94E5B159016A01DB
:108CD0008091160490911704A0911804B091190482
:108CE000BC01CD01A80197010E94E5B1B901C50100
:108CF0000E941FA28C010E94457C9C019093AE0AA9
:108D00008093AD0A8091200490912104AA2797FDB9
:108D1000A095BA2F7DE0880F991FAA1FBB1F7A95D7
:108D2000D1F78050904FAF43B040442737FD409576
:108D3000542FBC01CD010E94E5B1C90180509E4F66
:108D40009093210480932004053111050CF06624D2
:108D5000772081F08091A003882361F0C9018C58AD
:108D600090408234910530F0809159058062809363
:108D700059056624809136049091370480569940B5
:108D8000815C9B4228F08091590581608093590550
:108D9000809134049091350480569940815C9B42C7
:108DA00028F08091590582608093590580913204A2
:108DB000909133048C5291408957954028F08091CE
:108DC0005905846080935905809126049091270469
:108DD0008C529140835C914028F0809159058860C5
:108DE0008093590580912404909125048C529140E0
:108DF000835C914028F080915905806180935905EA
:108E0000809120049091210480509240835591409C
:108E100028F0809159058062809359058091590509
:108E20008111662486E4809380010E94CCA982E0AF
:108E30000E9432AB80911F0190912001A0912101ED
:108E4000B091220180937B0790937C07A0937D07CC
:108E5000B0937E0710924C0310924B0310924E0376
:108E600010924F0310925003109251031092F60388
:108E70001092F7031092F8031092F90310926D0705
:108E800010926C070E9450248091A70381FF07C0B5
:108E900080911D08882319F484E080931D081092A6
:108EA0009D0410929C04862D9927EEE0CDB7DEB785
:108EB0000C9420B2A3E1B0E0E0E6F7E40C9400B239
:108EC00080913204909133042091580330915903DA
:108ED000821B930B9093F00A8093EF0A80916203B8
:108EE0009091630397FD07969C0183E03595279544
:108EF0008A95E1F73093A80A2093A70A809160032E
:108F00009091610397FD079603E0959587950A95E3
:108F1000E1F790939D0A80939C0A3093B00A2093C6
:108F2000AF0A9093AB0A8093AA0A8091E80A9091C5
:108F3000E90AAC01440F551F480F591F20915403F3
:108F400030915503C901880F991F880F991F820F0F
:108F5000931F820F931F480F591F57FF02C04D5F89
:108F60005F4F55954795559547955093E90A40931E
:108F7000E80A8091FA0A9091FB0AAC01440F551F50
:108F8000480F591F2091560330915703C901880F8C
:108F9000991F880F991F820F931F820F931F480FED
:108FA000591F57FF02C04D5F5F4F55954795559527
:108FB00047955093FB0A4093FA0A8091B90A909121
:108FC000BA0A2091540330915503820F931F909356
:108FD000BA0A8093B90A8091F20A9091F30A20911B
:108FE000560330915703820F931F9093F30A809397
:108FF000F20A809122049091230401969093230415
:109000008093220480913D0390913E03A0913F0301
:10901000B09140038093D6039093D703A093D803D5
:10902000B093D9038091390390913A03A0913B0307
:10903000B0913C038093410390934203A093430378
:10904000B09344038FEC80937A0010921901209121
:109050000A0430910B0440910C0450910D042987AF
:109060003A874B875C8729543B46414050402CF05F
:1090700028E43BE641E050E00DC089859A85AB8548
:10908000BC85885B9449AE4FBF4F4CF428EB34E964
:109090004EEF5FEF2D833E834F83588708C089854D
:1090A0009A85AB85BC858D839E83AF83B8872091DD
:1090B0000E0430910F0440911004509111042D873B
:1090C0003E874F87588B29543B46414050402CF0F7
:1090D00028E43BE641E050E00DC08D859E85AF85DC
:1090E000B889885B9449AE4FBF4F4CF428EB34E904
:1090F0004EEF5FEF29833A834B835C8308C08D85F5
:109100009E85AF85B88989839A83AB83BC83A09100
:10911000EF0AB091F00ABB8BAA8BFD01CF01AA2701
:1091200097FDA095BA2FA0900604B0900704C090B8
:109130000804D0900904A80EB91ECA1EDB1EA09216
:109140000604B0920704C0920804D0920904E0908B
:10915000F60AF090F70A0091F80A1091F90AE80E61
:10916000F91E0A1F1B1FE092F60AF092F70A0093FD
:10917000F80A1093F90AF091BF03F98BFF2309F065
:1091800094C18091BE03882309F08FC180919C0A0D
:1091900090919D0AAA2797FDA095BA2FBC01CD01F9
:1091A00029813A814B815C810E9471B19B01AC01A4
:1091B00097FF04C02150384F4F4F5F4F6BE05595DC
:1091C0004795379527956A95D1F780916A01682E62
:1091D000772488249924CA01B901A40193010E942B
:1091E00071B1DC01CB018093420490934304A093BE
:1091F0004404B0934504B7FF04C08150904FAF4F73
:10920000BF4F1C012D013CE055944794379427949F
:109210003A95D1F72092420430924304409244049C
:10922000509245048091A70A9091A80AAA2797FD19
:10923000A095BA2FBC01CD012D813E814F8158856B
:109240000E9471B197FF04C06150784F8F4F9F4FBC
:109250002BE095958795779567952A95D1F7A40189
:1092600093010E9471B1DC01CB018093460490937D
:109270004704A0934804B0934904B7FF04C0815049
:10928000904FAF4FBF4F9C01AD018CE05595479576
:10929000379527958A95D1F7209346043093470454
:1092A00040934804509349048091420490914304B0
:1092B0009093960A8093950A809146049091470472
:1092C0009093980A8093970A221933094409550903
:1092D0002093460430934704409348045093490434
:1092E000E20EF31E041F151FE092F60AF092F70A31
:1092F0000093F80A1093F90A809169018823B1F468
:1093000057FF04C02F5F3F4F4F4F5F4F5595479515
:1093100037952795A21AB30AC40AD50AA092060463
:10932000B0920704C0920804D09209042A893B89AC
:1093300079010027F7FC0095102F80914604909149
:109340004704A0914804B0914904E80EF91E0A1F91
:109350001B1FC801B70129813A814B815C810E94A2
:1093600071B19B01AC0197FF04C02150384F4F4FA2
:109370005F4FBBE05595479537952795BA95D1F73F
:1093800080916B01A82EBB24CC24DD24CA01B90135
:10939000A60195010E9471B1DC01CB0180933A04D2
:1093A00090933B04A0933C04B0933D04B7FF04C0EA
:1093B0008150904FAF4FBF4F3C014D01ACE09594B1
:1093C000879477946794AA95D1F760923A04709243
:1093D0003B0480923C0490923D04C801B7012D816A
:1093E0003E814F8158850E9471B197FF04C0615042
:1093F000784F8F4F9F4FFBE09595879577956795B1
:10940000FA95D1F7A60195010E9471B1DC01CB015B
:1094100080933E0490933F04A0934004B093410492
:10942000B7FF04C08150904FAF4FBF4FAC01BD019B
:10943000ECE07595679557954795EA95D1F7409378
:109440003E0450933F0460934004709341042A8982
:109450003B8937FF03C0309521953F4F21343105BB
:10946000E4F1D401C30197FE07C0B095A095909593
:1094700081959F4FAF4FBF4F81389105A105B10531
:1094800084F4DB01CA0177FF07C0B095A0959095E1
:1094900081959F4FAF4FBF4F81389105A105B10511
:1094A000E4F081E08093F20318C01092980A1092C1
:1094B000970A1092960A1092950A10923E04109202
:1094C0003F04109240041092410410923A0410920A
:1094D0003B0410923C0410923D0480913E04909114
:1094E0003F04A0914004B0914104BC01CD0124E6A9
:1094F00030E040E050E00E94E5B1E0903A04F090A6
:109500003B04E21AF30AF092A60AE092A50A8091BF
:109510003A0490913B04A0913C04B0913D04BC01FD
:10952000CD0124E630E040E050E00E94E5B1DA01F0
:10953000C90120913E0430913F048C01021B130BA2
:1095400010939F0A00939E0A8091450190914601D5
:10955000A0914701B0914801BC01CD0128E631E05E
:1095600040E050E00E9471B12091F60A3091F70A74
:109570004091F80A5091F90A26173707480759070A
:1095800064F0261B370B480B590B2093F60A3093D7
:10959000F70A4093F80A5093F90A2091F60A30919D
:1095A000F70A4091F80A5091F90A57FF0CC0260FAC
:1095B000371F481F591F2093F60A3093F70A40932C
:1095C000F80A5093F90A80919C0A90919D0A8E0D99
:1095D0009F1D2091C4033091C503821B930BAA27C2
:1095E00097FDA095BA2F29853A854B855C85820F1A
:1095F000931FA41FB51F80930A0490930B04A0939C
:109600000C04B0930D04C0908501D0908601E090C9
:109610008701F0908801C816D906EA06FB0684F493
:1096200088EA91E6A0E0B0E08C199D09AE09BF0977
:1096300080930A0490930B04A0930C04B0930D0440
:1096400022273327A9012C193D094E095F09809172
:109650000A0490910B04A0910C04B0910D048217A0
:109660009307A407B50784F488E59EE9AFEFBFEF41
:10967000C80ED91EEA1EFB1EC0920A04D0920B042B
:10968000E0920C04F0920D048091A70A9091A80A30
:10969000800F911F2091C2033091C303821B930B53
:1096A000AA2797FDA095BA2F2D853E854F8558890D
:1096B000820F931FA41FB51F80930E0490930F0475
:1096C000A0931004B0931104E0908901F0908A01F6
:1096D00000918B0110918C01E816F9060A071B070F
:1096E00084F488EA91E6A0E0B0E08E199F09A00B0F
:1096F000B10B80930E0490930F04A0931004B093C9
:10970000110422273327A9012E193F09400B510BC1
:1097100080910E0490910F04A0911004B091110457
:1097200082179307A407B50784F488E59EE9AFEF95
:10973000BFEFE80EF91E0A1F1B1FE0920E04F09205
:109740000F0400931004109311048091060490916B
:109750000704A0910804B091090480931204909327
:109760001304A0931404B093150480910E049091F7
:109770000F04A0911004B091110480931A049093E7
:109780001B04A0931C04B0931D0480910A049091C3
:109790000B04A0910C04B0910D04809316049093D7
:1097A0001704A0931804B093190480912501909197
:1097B000260197FD079633E0959587953A95E1F751
:1097C0009093A80A8093A70A809123019091240185
:1097D00097FD079623E0959587952A95E1F7909355
:1097E0009D0A80939C0A80915C0390915D030F9782
:1097F00034F488E19CEF9093A80A8093A70A8091A3
:109800005C0390915D03079734F480E398EF9093A5
:10981000A80A8093A70A80915C0390915D03815D03
:10982000974034F088EE93E09093A80A8093A70ABB
:1098300080915C0390915D03805E974034F080EDF1
:1098400097E09093A80A8093A70A80915A03909179
:109850005B030F9734F488E19CEF90939D0A80930B
:109860009C0A80915A0390915B03079734F480E33C
:1098700098EF90939D0A80939C0A80915A0390914F
:109880005B03815D974034F088EE93E090939D0AEE
:1098900080939C0A80915A0390915B03805E97406D
:1098A00034F080ED97E090939D0A80939C0A60913C
:1098B0007801662309F4AFC040912501509126013B
:1098C00080914A0490914B04481B590B50935104CA
:1098D000409350042091250130912601280F391F13
:1098E00037FF02C02F5F3F4F3595279530934B04CC
:1098F00020934A04413851051CF080E890E005C0EF
:1099000040585F4F34F480E89FEF90935104809368
:109910005004409123015091240180914C04909176
:109920004D04481B590B50934F0440934E04209113
:10993000230130912401280F391F37FF02C02F5F08
:109940003F4F3595279530934D0420934C04413873
:1099500051051CF080E890E005C040585F4F34F49A
:1099600080E89FEF90934F0480934E04462F552735
:109970008091500490915104849FB001859F700D97
:10998000949F700D11249B0177FF02C0215F3F4F10
:10999000B4E035952795BA95E1F78091A70A9091A3
:1099A000A80A820F931F9093A80A8093A70A809118
:1099B0004E0490914F04849FD001859FB00D949FD9
:1099C000B00D1124AD019D01B7FF02C0215F3F4FD3
:1099D000A4E035952795AA95E1F780919C0A90918E
:1099E0009D0A820F931F90939D0A80939C0A8091F9
:1099F000250190912601860F971F90932601809351
:109A000025018091230190912401840F951F90934B
:109A10002401809323010091AA0A1091AB0A80913E
:109A2000950A9091960A101611065CF59C0197FF15
:109A300004C022273327281B390BC901AA2797FD09
:109A4000A095BA2F20916901332744275527BC01DF
:109A5000CD010E9471B19B01AC0197FF04C0215C54
:109A60003F4F4F4F5F4FF6E05595479537952795F8
:109A7000FA95D1F78091A50A9091A60A820F931FBB
:109A800027C097FF03C0909581959F4FAA2797FD08
:109A9000A095BA2F20916901332744275527BC018F
:109AA000CD010E9471B19B01AC0197FF04C0215C04
:109AB0003F4F4F4F5F4FE6E05595479537952795B8
:109AC000EA95D1F78091A50A9091A60A821B930B83
:109AD0009093A60A8093A50AE090AF0AF090B00A8E
:109AE0008091970A9091980A1E141F045CF59C01BE
:109AF00097FF04C022273327281B390BC901AA2747
:109B000097FDA095BA2F2091690133274427552747
:109B1000BC01CD010E9471B19B01AC0197FF04C053
:109B2000215C3F4F4F4F5F4F76E0559547953795F6
:109B300027957A95D1F780919E0A90919F0A820F7E
:109B4000931F27C097FF03C0909581959F4FAA2729
:109B500097FDA095BA2F20916901332744275527F7
:109B6000BC01CD010E9471B19B01AC0197FF04C003
:109B7000215C3F4F4F4F5F4F66E0559547953795B6
:109B800027956A95D1F780919E0A90919F0A821B32
:109B9000930B90939F0A80939E0A8091E40A87FF1B
:109BA00044C0B989BB2309F040C08091BE0388231B
:109BB000E1F5E1E0EE16E1E0FE064CF08091A70A47
:109BC0009091A80A8E0D9F1D805091400DC0F0E02D
:109BD000EF16FFEFFF0664F48091A70A9091A80AA0
:109BE0008E0D9F1D80509F4F9093A80A8093A70AC7
:109BF00021E0013012074CF080919C0A90919D0A5F
:109C0000800F911F805091400CC03FEF0030130730
:109C100064F480919C0A90919D0A800F911F80505E
:109C20009F4F90939D0A80939C0AE2E1CD5E0C9435
:109C30001CB28091DB03882329F58091A9038C7FD6
:109C40008093A9038091A8038F7D8093A803AEE53C
:109C5000B5E0E0E1F9E09FE080910B03882309F48F
:109C60008C938D918183128291503F9697FFF4CF10
:109C700080910B03882359F080910B0381508093CE
:109C80000B0305C08091A90381608093A903809193
:109C90008903882319F010928903089580938D0316
:109CA000809187038E7F8093870385EA8093BC0031
:109CB0000895882319F480E090E00895E82FFF27A5
:109CC000EE0FFF1FE95FF54F8081918181589F4F13
:109CD0008F3F910521F01CF08FEF90E004C097FFBB
:109CE00002C080E090E099270895CF93DF93ADED17
:109CF000B3E0CEEDD7E057E08991E82FFF27EE0FD4
:109D0000FF1FE95FF54F0190F081E02DE158FF4F13
:109D1000EF3FF10521F01CF0EFEFF0E004C0F7FF9A
:109D200002C0E0E0F0E0893111F4EC931BC04C91EB
:109D3000242F3327E217F307A9F0CF01821B930BDF
:109D400097FD03969595879595958795242F280FD0
:109D50002C93822F9927E817F90714F4215001C09A
:109D60002F5F2C935150119657FFC6CF8091E80773
:109D7000883F38F0EFEFF0E0E81BF109E352FC4FC9
:109D8000808180937D0180917D01882329F0843634
:109D900018F084E680937D018091EA07883F38F0CF
:109DA000EFEFF0E0E81BF109E352FC4F8081809374
:109DB0007C0180917C01882329F0843618F084E6A8
:109DC00080937C018091F707883F38F0EFEFF0E057
:109DD000E81BF109E352FC4F808180937701809169
:109DE00077018B3010F48AE002C08F3F11F480932A
:109DF000770180912408883F38F0EFEFF0E0E81B0E
:109E0000F109E352FC4F80818093BB0A8091BB0A29
:109E1000863010F485E002C08F3F11F48093BB0AB6
:109E200080912608883F38F0EFEFF0E0E81BF10959
:109E3000E352FC4F80818093EB0A8091EB0A8630DD
:109E400010F485E002C08F3F11F48093EB0A8091FB
:109E50001108873F19F4429905C007C0863F41F4B5
:109E6000439B03C08091460816C08091470813C0E9
:109E7000883F38F0EFEFF0E0E81BF109E352FC4FC8
:109E800080818093B80A8091B80A893110F488E102
:109E900002C08F3F11F48093B80A80911208873F67
:109EA00019F4429905C007C0863F41F4439B03C0A3
:109EB0008091480816C08091490813C0883F38F047
:109EC000EFEFF0E0E81BF109E352FC4F8081809353
:109ED000990A8091990A893110F488E102C08F3F74
:109EE00011F48093990A80911308883F38F0EFEFBE
:109EF000F0E0E81BF109E352FC4F80818093C10A36
:109F00008091C10A893110F488E102C08F3F11F4B9
:109F10008093C10A8091E9070E94594E8093B9034A
:109F20008091EC07883F38F0EFEFF0E0E81BF10993
:109F3000E352FC4F808180937B018091EE07883F44
:109F400038F0EFEFF0E0E81BF109E352FC4F8081BD
:109F5000809379018091F607883F38F0EFEFF0E0C9
:109F6000E81BF109E352FC4F808180937A018091D4
:109F7000F807883F38F0EFEFF0E0E81BF109E35213
:109F8000FC4F8081809376018091F907883F38F0FB
:109F9000EFEFF0E0E81BF109E352FC4F8081809382
:109FA00078018091FA07883F38F0EFEFF0E0E81B86
:109FB000F109E352FC4F8081809375018091FB078A
:109FC000883F38F0EFEFF0E0E81BF109E352FC4F77
:109FD00080818093740180910108883F38F0EFEF11
:109FE000F0E0E81BF109E352FC4F8081809372019D
:109FF00080910208883F38F0EFEFF0E0E81BF109AC
:10A00000E352FC4F80818093B80380910308883F1E
:10A0100038F0EFEFF0E0E81BF109E352FC4F8081EC
:10A020008093B70380910408883F38F0EFEFF0E0A9
:10A03000E81BF109E352FC4F80818093B6038091C5
:10A040000508883F38F0EFEFF0E0E81BF109E35234
:10A05000FC4F80818093B50380911F08883F38F0C2
:10A06000EFEFF0E0E81BF109E352FC4F80818093B1
:10A07000B40380912008883F38F0EFEFF0E0E81B50
:10A08000F109E352FC4F80818093B3038091210852
:10A09000883F38F0EFEFF0E0E81BF109E352FC4FA6
:10A0A00080818093B20380912208883F38F0EFEFDF
:10A0B000F0E0E81BF109E352FC4F80818093B1038B
:10A0C00080910608883F38F0EFEFF0E0E81BF109D7
:10A0D000E352FC4F80818093700180910A08883F91
:10A0E00038F0EFEFF0E0E81BF109E352FC4F80811C
:10A0F00080936F0180910708883F38F0EFEFF0E020
:10A10000E81BF109E352FC4F808180936E0180913E
:10A110000B08883F38F0EFEFF0E0E81BF109E3525D
:10A12000FC4F808180936D0180911408883F38F046
:10A13000EFEFF0E0E81BF109E352FC4F80818093E0
:10A140006C0180911708883F38F0EFEFF0E0E81BD2
:10A15000F109E352FC4F808180936B0180911808D4
:10A16000883F38F0EFEFF0E0E81BF109E352FC4FD5
:10A17000808180936A0180911908883F38F0EFEF61
:10A18000F0E0E81BF109E352FC4F80818093690104
:10A1900080914208883F38F0EFEFF0E0E81BF109CA
:10A1A000E352FC4F80818093A40A8091E60780935C
:10A1B000E40A80915B088093C00A80911E08883F62
:10A1C00038F0EFEFF0E0E81BF109E352FC4F80813B
:10A1D0008093680180913B08883F38F0EFEFF0E012
:10A1E000E81BF109E352FC4F80818093FD0A8091C6
:10A1F0007201282F33272F5F3F4F8CE398E2B9017C
:10A200000E94B0B170937F0160937E018091F4074A
:10A210008093EC0A8091F3078093AC0AE0913D08AB
:10A22000EE2309F449C081E08093B003FF27EE0FCD
:10A23000FF1FE95FF54F80819181805C9F4F14F48F
:10A240001092B003809180012091B003821721F118
:10A250008330F8F43091B001222351F08CED95E079
:10A2600090932E0380932D03332369F48EE209C06B
:10A2700088EC90E090932E0380932D03332319F400
:10A2800087E18093B00185E08093C603209380012D
:10A2900003C081508093800180913D0B90913E0BD3
:10A2A00097FF0FC08091B003882359F08091590522
:10A2B00080688093590505C0E093B0038AE08093DD
:10A2C000800180913D0B90913E0B97FF1DC08091C6
:10A2D000DB038823C9F08091B0038823A9F0809123
:10A2E0000C0190910D018F5F9F4F61F488E99AE313
:10A2F00090932E0380932D0380E094EA90930D01B8
:10A3000080930C011092B0038091B003882321F058
:10A310008091A803816003C08091A8038E7F809301
:10A32000A803DF91CF9108958091EF07882301F56D
:10A330006091C0037091C10377FF02C06D5F7F4FD2
:10A3400075956795759567954091270150912801FE
:10A3500080910201282F3327649FC001659F900DD3
:10A36000749F900D1124B9010E949CB1CB0101C0D2
:10A370009927909384018093830180918301909128
:10A3800084018734910538F486E490E09093840149
:10A390008093830108958F3A910530F08FEA90E021
:10A3A00090938401809383010895F8948091DA0753
:10A3B000E82FFF27EE0FFF1FE95FF54F60817181E6
:10A3C0007093060A6093050A8091DB07E82FFF2748
:10A3D000EE0FFF1FE95FF54F408151815093030A53
:10A3E0004093020A8091DD07E82FFF27EE0FFF1F41
:10A3F000E95FF54F208131813093010A2093000AF3
:10A400008091DC07E82FFF27EE0FFF1FE95FF54F74
:10A410000190F081E02DF0934E0AE0934D0A809177
:10A420005205A82FBB27A0FF3DC08091FD0A8138AF
:10A43000C8F180914D05992787FD9095680F791F88
:10A440007093060A6093050A80914E05992787FD4F
:10A450009095480F591F5093030A4093020A809128
:10A460004F05992787FD9095280F391F3093010AD2
:10A470002093000A80915005A1FF0AC0992787FD0B
:10A480009095E80FF91FF0934E0AE0934D0A0AC029
:10A49000992787FD90958E179F0724F490934E0A75
:10A4A00080934D0A78948091050A9091060A80382D
:10A4B00091051CF08FE790E005C081589F4F34F460
:10A4C00081E89FEF9093060A8093050A8091020A23
:10A4D0009091030A803891051CF08FE790E005C049
:10A4E00081589F4F34F481E89FEF9093030A809343
:10A4F000020A8091000A9091010A803891051CF0AF
:10A500008FE790E005C081589F4F34F481E89FEFBA
:10A510009093010A8093000A80914D0A90914E0A0F
:10A52000803891053CF08FE790E090934E0A80933D
:10A530004D0A089581589F4F34F481E89FEF90931E
:10A540004E0A80934D0A0895ABE0B0E0EAEAF2E5E6
:10A550000C9400B20E945A478091A90399278471F4
:10A560009070892B91F580915C0882FF27C08091C3
:10A57000C0039091C1030097F1F022E08835920763
:10A58000D4F49C0197FF02C02D5F3F4F359527956E
:10A59000359527958091FE079927289FA001299F2F
:10A5A000500D389F500D1124CA0164E670E00E94DE
:10A5B000B0B1CB0106C08DE290E003C08091FE07F0
:10A5C00099279093A6038093A5032091A30330912C
:10A5D000A40355E72033350759F41092E70310928E
:10A5E000E6038091AC0A99279093A6038093A50374
:10A5F0006091E6037091E7037A8369838091AC0AE6
:10A6000099270A966817790714F49A8389838091A9
:10A61000DC038436C8F58091A80382FD35C08AE04A
:10A620008093990380915E0490915F04009731F0CC
:10A63000019790935F0480935E040BC01092DB033C
:10A640009093AB038093AA038091A9038D7E80939E
:10A65000A903289A8091AA039091AB03895E934045
:10A6600080F080918C0B853660F08091A5039091ED
:10A67000A6039A8389838091A90380618093A903AB
:10A6800074C51092DB0371C58091DC038D3808F42A
:10A6900042C590914F08992309F445C08091500814
:10A6A000882309F440C0E92FFF27EE0FFF1FE95F61
:10A6B000F54F80819181C397BCF0809197018233DF
:10A6C00061F48091A80385FF08C08091A80380648D
:10A6D0008093A80380E38093B0018091A8038F77D3
:10A6E0008093A80386E917C0808191818E5C9F4F7B
:10A6F000ACF480919701863941F48091A803806879
:10A700008093A8038FE28093B0018091A8038F7B90
:10A710008093A80382E38093970105C08091A803EA
:10A720008F738093A8038091A9038F7E8093A903E0
:10A730009091FF0782E3989FC001112490935F04DA
:10A7400080935E04E981FA81B9978CF08091DB03F4
:10A75000882369F08091AA039091AB03FFEF8F3FAC
:10A760009F0729F001969093AB038093AA03409131
:10A77000AA035091AB034F3F510509F048F51092E1
:10A78000FE031092FF031092000410920104109235
:10A79000FA031092FB031092FC031092FD03109237
:10A7A00052041092530410925404109255041092C3
:10A7B0000604109207041092080410920904809174
:10A7C000A80380628093A80384E68093970151C117
:10A7D0008091A90382608093A9038091A80385FFDB
:10A7E00098C080918F0499279C012470307082FD5D
:10A7F00004C08091A80386FF2AC0809144018D3354
:10A8000031F58091A003882311F180E58093CB037B
:10A8100084EF91E0A0E0B0E08093CC039093CD036F
:10A82000A093CE03B093CF038093D2039093D3032E
:10A83000A093D403B093D50388EE93E09093960150
:10A8400080939501232B19F08DE08093B0018091C6
:10A85000410390914203A0914303B091440387398F
:10A860009105A105B1058CF48091D6039091D70391
:10A87000A091D803B091D903825A9E4FAF4FBF4FDA
:10A8800024F08091E40A80FD21C088EE93E090934B
:10A890009601809395018091A80386FF0FC01092C6
:10A8A000CB038CE291E0A0E0B0E08093D2039093E0
:10A8B000D303A093D403B093D50303C080E3809364
:10A8C000B0018091A8038F718093A8031092FE03BA
:10A8D0001092FF0310920004109201041092FA03E8
:10A8E0001092FB031092FC031092FD0310920604D9
:10A8F000109207041092080410920904495E534014
:10A9000008F4B7C088EE93E09093AB038093AA035A
:10A91000B0C08091A80387FF1AC080914401863798
:10A9200011F08D33A1F48091A003882381F08091F0
:10A9300050088093CB0380EE91EBAFEFBFEF809395
:10A94000CC039093CD03A093CE03B093CF0320917B
:10A9500095013091960143E0283E340708F04AC043
:10A960002F5F3F4F30939601209395011092FE0385
:10A970001092FF0310920004109201041092FA0347
:10A980001092FB031092FC031092FD031092060438
:10A990001092070410920804109209048091410358
:10A9A00090914203A0914303B09144038C52914093
:10A9B000A040B0408093D2039093D303A093D403DC
:10A9C000B093D503285E334009F053C08091A803AB
:10A9D00087FF4FC0809144018B3209F44AC08091B7
:10A9E000A8038F778093A8038091A8038062809347
:10A9F000A8033FC08091A0038823D9F1809144012E
:10AA0000863711F08D32A9F58091D6039091D70346
:10AA1000A091D803B091D903885E9340A040B04084
:10AA200044F52091790730917A0737FF02C02D5FF6
:10AA30003F4F35952795359527958091560899274D
:10AA400082179307B4F4209120043091210437FF3A
:10AA500002C02D5F3F4F3595279535952795821775
:10AA600093073CF410929601109295018EE080932A
:10AA7000B00180914D0A90914E0A813591050CF4F8
:10AA80001DC14091DB03442309F018C180918F045C
:10AA900099279C012071307084FD10C18091000ABB
:10AAA0009091010A8C3491050CF4C6C08091620427
:10AAB0008F5F80936204893C08F400C1142F409397
:10AAC00062043093AB032093AA032091050A3091CE
:10AAD000060A273431056CF48091020A9091030A2A
:10AAE00097FF03C0909581959F4F873491050CF493
:10AAF00044C04091020A5091030A473451053CF08A
:10AB00002634310524F42B5B3F4F0CF011E0473421
:10AB1000510544F08091050A9091060A8734910509
:10AB20000CF012E04634510544F48091050A9091EE
:10AB3000060A873491050CF013E08FEF4A3B580763
:10AB400044F48091050A9091060A873491050CF02F
:10AB500014E04A5B5F4F64F48091050A9091060A05
:10AB6000863491052CF48B5B9F4F14F015E002C0E6
:10AB7000112319F0812F0E94C4388091020A90910C
:10AB8000030A4D96CB9798F48091050A9091060A96
:10AB90008A5B9F4F64F481E0809374051092C70331
:10ABA00088EE93E090932E0380932D0387C08091CD
:10ABB00001010E94693880E00E945F0D80910008C9
:10ABC0000E94FAAC8091E40A80FF10C080911D01C0
:10ABD00090911E01875B934038F480911D01909104
:10ABE0001E018E5E924010F40E948824112381F48D
:10ABF0008091020A9091030A8A5B9F4F4CF48091E6
:10AC0000050A9091060A8634910514F483E001C088
:10AC100081E00E9498438093C70391E090932B03B7
:10AC2000579A80915905882379F58091C703882325
:10AC300091F59093B00132C0855B9F4FCCF5809128
:10AC4000020A9091030A0F964F9790F58091600445
:10AC50009091610401969093610480936004855CF7
:10AC6000994060F1309361042093600482E00E9477
:10AC70009843982F8093C70321E020932B03579A82
:10AC800080915905882311F087E006C0992319F4B3
:10AC90002093B00103C088E18093B0018AE08093E3
:10ACA000C80468E770E0809101010E94924206C0EA
:10ACB00010926204109261041092600480914D0A17
:10ACC00090914E0A8C599F4F0CF01EC2E0913E08A5
:10ACD000AE2FBB27AF77B070AA0FBB1FA15BB54FDC
:10ACE0008D919C911197069714F084E606C08D9182
:10ACF0009C918B5F9F4F1CF48CE98093650480913D
:10AD0000DB032091000A3091010A882309F061C118
:10AD10002C593F4F94F480915C0883FD0AC0FF27B3
:10AD2000EE0FFF1FE95FF54F80819181855B9F4F9B
:10AD3000DCF080913E088823B9F080915C0883FFA5
:10AD400045C180913E08E82FFF27EE0FFF1FE95F06
:10AD5000F54F80819181875F9F4F0CF437C18091BF
:10AD60006504843609F032C180918F0484FD2EC1C0
:10AD70008091C703882329F08091A903886080937C
:10AD8000A90380911F0190912001A0912101B09110
:10AD9000220180937B0790937C07A0937D07B0935B
:10ADA0007E071092D6031092D7031092D803109208
:10ADB000D90310923D0310923E0310923F0310926C
:10ADC000400388E592E09093A4038093A30310923C
:10ADD000390310923A0310923B0310923C031092F5
:10ADE0004E0310924F031092500310925103809122
:10ADF000050A9091060A8D599F4F4CF48091020AE2
:10AE00009091030A8D599F4F873C910530F48091B2
:10AE10003E08882311F480936304809163048F5F5C
:10AE2000809363048E3F08F452C18091A703209160
:10AE3000EF0A3091F00A81FF21C0C90137FF04C039
:10AE400088279927821B930B81349105ACF580915B
:10AE5000A70A9091A80A97FF03C0909581959F4FEC
:10AE6000CD9754F580919C0A90919D0A97FF03C05D
:10AE7000909581959F4FCD970CF11EC0C90137FF6A
:10AE800003C0909581959F4F8197B4F48091A70A54
:10AE90009091A80A97FF03C0909581959F4F459781
:10AEA0005CF480919C0A90919D0A97FF03C0909555
:10AEB00081959F4F459714F01092C7031092630439
:10AEC00080915905882309F074C08091C7038823B5
:10AED00009F46FC080919304882309F06AC081E06F
:10AEE00090E09093AB038093AA0381E08093DB030F
:10AEF000109252041092530410925404109255046C
:10AF0000109206041092070410920804109209048B
:10AF1000109202041092030410920404109205048B
:10AF20008091F507E82EFF24002711278091E80A79
:10AF30009091E90A9C01442737FD4095542FC801A0
:10AF4000B7010E9471B1DC01CB0180930E04909394
:10AF50000F04A0931004B09311048091FA0A909109
:10AF6000FB0A9C01442737FD4095542FC801B701C7
:10AF70000E9471B1DC01CB0180930A0490930B0411
:10AF8000A0930C04B0930D041092FE031092FF03E3
:10AF900010920004109201041092FA031092FB0325
:10AFA0001092FC031092FD0384E68093C60384E3B1
:10AFB00080C08CED95E090932E0380932D038091BB
:10AFC000C703882309F083C081E073C01092630433
:10AFD0007EC02536310594F080915C0883FD0AC05F
:10AFE000FF27EE0FFF1FE95FF54F80819181855BA1
:10AFF0009F4FDCF080913E088823B9F080915C0877
:10B0000083FF63C080913E08E82FFF27EE0FFF1FEC
:10B01000E95FF54F808191818E5C9F4F0CF055C0A8
:10B02000809165048C3909F050C08091050A909197
:10B03000060A8D599F4F4CF48091020A9091030AA1
:10B040008D599F4F873C910538F480913E088823A5
:10B0500019F48093640418C01092FE031092FF0349
:10B0600010920004109201041092FA031092FB0354
:10B070001092FC031092FD031092ED031092EC036A
:10B080001092EB031092EA03809164048F5F809327
:10B0900064048B3F88F01092DB03109264041092DA
:10B0A000AB031092AA038091A8038F718093A80329
:10B0B00086E28093B0010BC0843649F48CEA9DE0AF
:10B0C00090932E0380932D0302C01092640420916C
:10B0D000A3033091A40343E0283E340708F045C0A1
:10B0E00080914B0390914C038B569F4F1CF02F5F28
:10B0F0003F4F05C021153105C1F12150304030933B
:10B10000A4032093A30331C0109265041092A403FA
:10B110001092A3032AC02E5E324038F18091050BB5
:10B120009091060B8059914000F58091D603909143
:10B13000D703A091D803B091D9038C5D9540A0406E
:10B14000B0409CF480E395E79093A4038093A3031D
:10B150008091AA039091AB038A5E934030F089EE10
:10B1600093E09093AB038093AA03809143018150B5
:10B1700080934301809143018F3F21F08091A90387
:10B1800084FF80C30E94754E0E94D5512091F00724
:10B190008091660490916704AC01440F551F480FDD
:10B1A000591F33278091050A9091060A829FB001AA
:10B1B000839F700D929F700D1124460F571F57FFEC
:10B1C00002C04D5F5F4F55954795559547955093F4
:10B1D0006704409366048091680490916904AC010F
:10B1E000440F551F480F591F8091020A9091030A7E
:10B1F000829FD001839FB00D929FB00D11244A0F02
:10B200005B1F57FF02C04D5F5F4F559547955595A2
:10B2100047955093690440936804F8940091DA07C5
:10B22000E02FFF27EE0FFF1FE15BF54F8091F10745
:10B23000482F552780819181849F9001859F300DF3
:10B24000949F300D11248091660490916704820FC1
:10B25000931F90936704809366041091DB07E12F9E
:10B26000FF27EE0FFF1FE15BF54F80819181849FE7
:10B270009001859F300D949F300D112480916804BA
:10B2800090916904820F931F9093690480936804DE
:10B29000789480914D0A90914E0A81589F4F9093D7
:10B2A000E7038093E6038091B003409166045091D8
:10B2B0006704882309F44BC0CA0157FD0396DC01DB
:10B2C000B595A795B595A795809168049091690467
:10B2D00097FD0396FC01F595E795F595E795809127
:10B2E000A801682F772767FD70956A9F90016B9F73
:10B2F000300D7A9F300D112480919604482F5527E8
:10B3000047FD50954E9FC0014F9F900D5E9F900D41
:10B310001124280F391F37FF02C0295F3F4F93E0E8
:10B32000359527959A95E1F73093ED032093EC033B
:10B330006E9F90016F9F300D7E9F300D11244A9FAC
:10B34000C0014B9F900D5A9F900D112443C08091D6
:10B350003C08E82FFF27E75BFE4F86818093A8011A
:10B36000908190939604A82FBB27A7FDB095A49F2A
:10B370009001A59F300DB49F300D1124E92FFF27B8
:10B38000E7FDF0956091680470916904E69FC00143
:10B39000E79F900DF69F900D1124280F391F37FF5E
:10B3A00002C0295F3F4F83E0359527958A95E1F7E5
:10B3B0003093ED032093EC03A69F9001A79F300DDF
:10B3C000B69F300D1124E49FC001E59F900DF49FBE
:10B3D000900D1124281B390B37FF02C0295F3F4F06
:10B3E000F3E035952795FA95E1F73093EB03209339
:10B3F000EA038091000A9091010A909581959F4FF0
:10B400009093E9038093E8038530910514F0049745
:10B4100005C0BFEF8C3F9B0734F404969093E9037B
:10B420008093E80304C01092E9031092E80380912E
:10B43000A3039091A4038150924078F18091EC0392
:10B440009091ED0397FD0796E3E095958795EA9532
:10B45000E1F79093ED038093EC038091EA039091E0
:10B46000EB0397FD079673E0959587957A95E1F73D
:10B470009093EB038093EA031092FE031092FF0374
:10B4800010920004109201041092FA031092FB0330
:10B490001092FC031092FD0343C080918104882325
:10B4A00009F43EC0282F33278091EC039091ED03DF
:10B4B00097FD079663E0959587956A95E1F7289F34
:10B4C000A001299F500D389F500D1124CA0157FD2E
:10B4D0000F9654E0959587955A95E1F79093ED0373
:10B4E0008093EC038091EA039091EB0397FD07961C
:10B4F00043E0959587954A95E1F7289FB001299FEC
:10B50000700D389F700D1124CB0177FD0F96B4E0BC
:10B5100095958795BA95E1F79093EB038093EA03AD
:10B52000C090EC03D090ED03809184049091850449
:10B53000C81AD90AD092ED03C092EC038091EA03B5
:10B540009091EB032091820430918304821B930B32
:10B550009093EB038093EA03809177019927AA27C0
:10B5600097FDA095BA2FBC01CD010E94E5B0DC018A
:10B57000CB0120E030E040E251E4BC01CD010E946B
:10B5800053B0DC01CB01BC01CD010E94B7B0DC019E
:10B59000CB018093F40A809176018093C20A809156
:10B5A00075019927AA2797FDA095BA2FBC01CD0157
:10B5B0000E94E5B0DC01CB0120E030E040E251E444
:10B5C000BC01CD010E9453B0DC01CB01BC01CD0117
:10B5D0000E94B7B0DC01CB018093A30A8091740173
:10B5E0008093B10A8091E40A82FF02C01092C20ADD
:10B5F000C601D7FC03969C0135952795359527956F
:10B6000037FF03C0309521953F4F8091AE03909155
:10B61000AF0382179307B4F4C601D7FE03C0909519
:10B6200081959F4F97FD039695958795959587955D
:10B630009093AF038093AE038536910544F084E682
:10B6400090E001C001979093AF038093AE034091C7
:10B65000EA035091EB03CA0157FD03969C0135950F
:10B6600027953595279537FF03C0309521953F4F96
:10B670008091AC039091AD0382179307B4F4CA0193
:10B6800057FF03C0909581959F4F97FD0396959521
:10B690008795959587959093AD038093AC038536F8
:10B6A000910544F084E690E001C001979093AD03CA
:10B6B0008093AC038091A90384FF08C01092AF036C
:10B6C0001092AE031092AD031092AC03E12FFF274E
:10B6D000EE0FFF1FE95FF54F40911508242F332728
:10B6E000808191812817390744F48091590882FF9D
:10B6F00004C081E08093BD0313C0E12FFF27EE0F4C
:10B70000FF1FE95FF54F842F992720911608821BB0
:10B710009109208131812817390714F41092BD0353
:10B720004091DB07E42FFF27EE0FFF1FE95FF54F86
:10B7300050911508852F992722273327281B390B6D
:10B74000808191818217930744F48091590883FF87
:10B7500004C081E08093BC0316C08091BC038823A1
:10B7600091F0E42FFF27EE0FFF1FE95FF54F809167
:10B7700016089927851B910920813181821793072B
:10B7800014F41092BC03E02FFF27EE0FFF1FE95FB8
:10B79000F54F40911508242F332780819181281778
:10B7A000390744F48091590880FF04C081E08093F8
:10B7B000BA0317C08091BA03882399F0E02FFF27BE
:10B7C000EE0FFF1FE95FF54F842F99272091160890
:10B7D000821B9109208131812817390714F41092B6
:10B7E000BA034091DA07E42FFF27EE0FFF1FE95F4E
:10B7F000F54F50911508852F992722273327281BAD
:10B80000390B808191818217930744F48091590804
:10B8100081FF04C081E08093BB0316C08091BB030D
:10B82000882391F0E42FFF27EE0FFF1FE95FF54F0C
:10B83000809116089927851B9109208131818217F3
:10B84000930714F41092BB038091BD03882319F46D
:10B850008091BC03811181E08093BE038091BA0383
:10B86000882321F48091BB03882351F081E08093E9
:10B87000BF031092BE031092BD031092BC0302C01E
:10B880008093BF038091BE03882321F48091BF037E
:10B89000882369F0809114089927A981BA818A17B1
:10B8A0009B0714F49A83898381E08093F20380914B
:10B8B000A80399279C012470307082FF31C08091C9
:10B8C000840490918504909581959F4F9093ED030A
:10B8D0008093EC03809182049091830490958195EC
:10B8E0009F4F9093EB038093EA03809183019091A3
:10B8F00084019093E7038093E6031092E90310928A
:10B90000E8038091E40A8B778B668093E40A809148
:10B91000C00A8C7B8093C00A88EC8093B9031EC058
:10B920008091A90384FF1AC03093E9032093E803B0
:10B930003093ED032093EC033093EB032093EA0361
:10B940009AE59093F40A88E78093C20A9093A30A39
:10B950008093B10A1092BE031092BF038091B40A83
:10B960009091B50AA091B60AB091B70A20911A0435
:10B9700030911B0440911C0450911D04820F931FB1
:10B98000A41FB51F8093B40A9093B50AA093B60A7A
:10B99000B093B70A8091BC0A9091BD0AA091BE0AEB
:10B9A000B091BF0A209016043090170440901804FC
:10B9B00050901904820D931DA41DB51D8093BC0ADF
:10B9C0009093BD0AA093BE0AB093BF0AB091BF0383
:10B9D000BB83BB2321F48091BE03882301F1109225
:10B9E000B40A1092B50A1092B60A1092B70A1092D1
:10B9F000BC0A1092BD0A1092BE0A1092BF0A1092A1
:10BA00004A03109249031092C3031092C20310928A
:10BA1000C5031092C403EB81EE2309F0E4C18091C9
:10BA2000BE03882309F0DFC18091790790917A07DE
:10BA3000815092402CF48091DB03882309F4D3C118
:10BA40009090760BA090F5076091E80A7091E90A52
:10BA50007B876A878091FA0A9091FB0A9987888789
:10BA600019140CF0BEC0BB24CC24DD24CA01B901DA
:10BA7000A60195010E94E5B179018A0180913F0BF1
:10BA80009091400BAA85BB85A81BB90BFD01CF0186
:10BA9000AA2797FDA095BA2FE81AF90A0A0B1B0BE3
:10BAA000C201B101A60195010E94E5B159016A01E7
:10BAB0008091410B9091420B28853985281B390BC9
:10BAC000C901AA2797FDA095BA2FA81AB90ACA0AD0
:10BAD000DB0A292C332427FC3094432C532CC80137
:10BAE000B701A20191010E9471B197FF04C061509A
:10BAF0007E4F8F4F9F4F3B014C0169E09594879497
:10BB0000779467946A95D1F7C601B501A2019101B6
:10BB10000E9471B197FF04C061507E4F8F4F9F4FBD
:10BB20005B016C0159E0D594C794B794A7945A95DA
:10BB3000D1F78091AE039091AF03813491053CF42D
:10BB40008091AC039091AD0381349105D4F0D40180
:10BB5000C30197FE03C00196A11DB11D3C014D011B
:10BB60009594879477946794D601C501D7FE03C056
:10BB70000196A11DB11D5C016D01D594C794B794C8
:10BB8000A7948091780B282F332727FD3095432FDA
:10BB9000532F261537054805590514F439014A0174
:10BBA000992787FD9095909581959F4FAA2797FD9E
:10BBB000A095BA2F681679068A069B0614F43C01F4
:10BBC0004D012A153B054C055D0514F459016A0128
:10BBD000A816B906CA06DB060CF0C9C05C016D01E7
:10BBE000C6C0EA2CFF2400271127CA01B901A80109
:10BBF00097010E94E5B139014A014A855B85CA0176
:10BC0000AA2797FDA095BA2F681A790A8A0A9B0A73
:10BC1000C201B101A80197010E94E5B159016A0171
:10BC200068857985CB01AA2797FDA095BA2FA81A18
:10BC3000B90ACA0ADB0AD401C30197FE03C00F96F2
:10BC4000A11DB11D3C014D0124E09594879477948A
:10BC500067942A95D1F7D601C501D7FE03C00F9688
:10BC6000A11DB11D5C016D0194E0D594C794B794FA
:10BC7000A7949A95D1F78091AE039091AF03813448
:10BC800091053CF48091AC039091AD038134910512
:10BC9000A4F0C401B30123E030E040E050E00E9492
:10BCA000E5B139014A01C601B50123E030E040E0C9
:10BCB00050E00E94E5B159016A018091000A90911B
:10BCC000010A97FF03C0909581959F4F4A97A4F072
:10BCD000C401B30123E030E040E050E00E94E5B150
:10BCE00039014A01C601B50123E030E040E050E0EF
:10BCF0000E94E5B159016A0189E180938F0171E2E7
:10BD000067167104810491042CF080E2682E712C76
:10BD1000812C912C80EE68168FEF78068FEF8806C5
:10BD20008FEF980644F400EE602E0FEF702E0FEFA9
:10BD3000802E0FEF902E91E2A916B104C104D10418
:10BD40002CF010E2A12EB12CC12CD12CA0EEAA1601
:10BD5000AFEFBA06AFEFCA06AFEFDA0644F4B0EEC3
:10BD6000AB2EBFEFBB2EBFEFCB2EBFEFDB2E8091F4
:10BD70000E0490910F04A0911004B0911104861943
:10BD80009709A809B90980930E0490930F04A09312
:10BD90001004B093110480910A0490910B04A091B7
:10BDA0000C04B0910D048A199B09AC09BD0980935C
:10BDB0000A0490930B04A0930C04B0930D0480919B
:10BDC0009C0390919D03860D971D90939D038093F6
:10BDD0009C0380919A0390919B038A0D9B1D9093E5
:10BDE0009B0380939A038091490390914A038F3F6C
:10BDF000910509F008F452C1E0911D08EE2309F401
:10BE0000FFC08091E80A9091E90A815E9C4F8F53B0
:10BE1000964008F0F5C08091FA0A9091FB0A815E85
:10BE20009C4F8F53964008F0EBC08091F20388231B
:10BE300009F0E6C08091EF0A9091F00A4F96CF97F3
:10BE400008F0DEC0FF27A6E0EE0FFF1FAA95E1F77E
:10BE500020919C0330919D03C901BF010E949CB1B8
:10BE6000261B370B30939D0320939C0320919A034C
:10BE700030919B03C901BF010E949CB1261B370B67
:10BE800030939B0320939A032091F0033091F103A8
:10BE9000C901BF010E949CB1261B370B3093F103EF
:10BEA0002093F0038091AE039091AF03813491050C
:10BEB00094F48091AC039091AD03813491055CF4CE
:10BEC0008091000A9091010A97FF03C09095819597
:10BED0009F4F4A97E4F080919C0390919D0397FDBA
:10BEE00001969595879590939D0380939C038091EF
:10BEF0009A0390919B0397FD019695958795909352
:10BF00009B0380939A031092F1031092F0038091A7
:10BF10009C0390919D03895B9B406CF010929D0364
:10BF200010929C038091360490913704019690936F
:10BF300037048093360480919C0390919D0388542C
:10BF4000944F6CF410929D0310929C0380913604E0
:10BF50009091370401979093370480933604809131
:10BF60009A0390919B03895B9B406CF010929B031A
:10BF700010929A0380913404909135040196909325
:10BF800035048093340480919A0390919B038854E4
:10BF9000944F6CF410929B0310929A038091340496
:10BFA00090913504019790933504809334048091E7
:10BFB000F0039091F1038D5A9D406CF01092F103C3
:10BFC0001092F00380913204909133040196909383
:10BFD0003304809332048091F0039091F1038455EF
:10BFE000924FD4F41092F1031092F0038091320436
:10BFF00090913304019790933304809332040CC0E2
:10C0000010929D0310929C0310929B0310929A032E
:10C010001092F1031092F0031092F2038091C20A81
:10C02000882341F41092C5031092C4031092C303F5
:10C030001092C2038091B40A9091B50AA091B60AF9
:10C04000B091B70A80936A0490936B04A0936C0438
:10C05000B0936D048091BC0A9091BD0AA091BE0A74
:10C06000B091BF0A80936E0490936F04A093700404
:10C07000B09371041092B40A1092B50A1092B60AE5
:10C080001092B70A1092BC0A1092BD0A1092BE0A12
:10C090001092BF0A10924A03109249038090E8035D
:10C0A0009090E903C40197FE04C088279927881956
:10C0B000990904973CF08091E40A84FD03C082E36F
:10C0C0008093C6031091F207A12EBB24CC24DD245B
:10C0D000B401882777FD8095982F940197FE04C0BE
:10C0E0002227332728193909442737FD4095542F33
:10C0F0000E9471B19B01AC01C601B5010E9471B1F2
:10C1000097FF04C061507E4F8F4F9F4F59E0959528
:10C110008795779567955A95D1F79B01812F992738
:10C12000889DD001899DB00D989DB00D1124CD0141
:10C13000B7FD03969595879595958795280F391F97
:10C140008091A3039091A4038150924010F020E0CD
:10C1500030E08091C8039091C903820F931F9C0126
:10C16000442737FD4095542F2093520430935304B5
:10C170004093540450935504809106049091070411
:10C18000A0910804B0910904821B930BA40BB50B7A
:10C190008093060490930704A0930804B0930904C5
:10C1A0008155934CA040B04064F080E593ECA0E052
:10C1B000B0E08093060490930704A0930804B09322
:10C1C00009048091060490910704A0910804B0919D
:10C1D0000904805B9C43AF4FBF4F64F480EB9CE34A
:10C1E000AFEFBFEF8093060490930704A093080479
:10C1F000B0930904809093019090940197FCFAC049
:10C200008091E40A83FFF6C0809190018150809371
:10C210009001882309F0F2C08DE080939001809115
:10C220001A0490911B04A0911C04B0911D04B7FF47
:10C2300004C081509E4FAF4FBF4F39E0B595A795D1
:10C24000979587953A95D1F78C0197FF03C0109584
:10C2500001951F4F8091160490911704A091180426
:10C26000B0911904B7FF04C081509E4FAF4FBF4F2C
:10C2700029E0B595A795979587952A95D1F79C01C3
:10C2800097FF03C0309521953F4F021713070CF419
:10C290008901B80117FF02C0695F7F4F3B01A3E02E
:10C2A00075946794AA95E1F722E030E0620E731E60
:10C2B000A090F60AB090F70AC090F80AD090F90A58
:10C2C000209145013091460140914701509148012C
:10C2D000C601B5010E94E5B119012A013093A20AF5
:10C2E0002093A10A821A930AC401845E9D4F68E6D6
:10C2F00071E00E94B0B1AC01445B50402091C60394
:10C30000222321F03092F5032092F40380918D01D5
:10C3100090918E01009731F0019790938E01809358
:10C320008D0112C0093111057CF48091F0039091C8
:10C33000F103840F951F9093F1038093F003222360
:10C3400019F021502093C60380918D0190918E01A8
:10C35000892BF9F480918F019927489FB001499F5B
:10C36000700D589F700D1124CB01B3010E94B0B124
:10C37000CB01AA2797FDA095BA2FA80EB91ECA1EF9
:10C38000DB1EA092F60AB092F70AC092F80AD09289
:10C39000F90A8091C603882369F58091F40390918E
:10C3A000F5032091A10A3091A20A821B930B845EAF
:10C3B0009D4F68E671E00E94B0B19C01245B304063
:10C3C00080917A0186959927289FD001299FB00DE9
:10C3D000389FB00D11249D01B7FF02C0215F3F4F70
:10C3E000F4E035952795FA95E1F73093C90320934A
:10C3F000C80304C01092C9031092C8038091F203CD
:10C40000882381F01092FA031092FB031092FC0330
:10C410001092FD031092FE031092FF03109200048D
:10C4200010920104BB81BB23F1F48091C20A282F32
:10C4300033274427552780911A0490911B04A0911B
:10C440001C04B0911D04BC01CD010E9471B1DC013E
:10C45000CB01BC01CD0128EF3AE240E050E00E9460
:10C46000E5B1290102C0442455248091BE038823EC
:10C47000F1F48091C20A282F332744275527809151
:10C48000160490911704A0911804B0911904BC01EE
:10C49000CD010E9471B1DC01CB01BC01CD0128EFBF
:10C4A0003AE240E050E00E94E5B1190102C02224C6
:10C4B000332480919E0A90919F0A893C91051CF03B
:10C4C00088EC90E005C088539F4F34F488E39FEFD9
:10C4D00090939F0A80939E0A8091A50A9091A60A44
:10C4E000893C91051CF088EC90E005C088539F4F73
:10C4F00034F488E39FEF9093A60A8093A50A809175
:10C50000A70A9091A80AAA2797FDA095BA2F209173
:10C51000F40AA22EBB24CC24DD24BC01CD01A6014B
:10C5200095010E9471B19B01AC0180919E0A90918E
:10C530009F0AAA2797FDA095BA2FE7E0880F991FB9
:10C54000AA1FBB1FEA95D1F7280F391F4A1F5B1F8F
:10C5500057FF04C0215C3F4F4F4F5F4F76E055952A
:10C560004795379527957A95D1F78201020F131FCA
:10C570001093A80A0093A70A80919C0A90919D0AA3
:10C58000AA2797FDA095BA2FBC01CD01A601950160
:10C590000E9471B19B01AC018091A50A9091A60AFD
:10C5A000AA2797FDA095BA2F67E0880F991FAA1FA9
:10C5B000BB1F6A95D1F7280F391F4A1F5B1F57FF12
:10C5C00004C0215C3F4F4F4F5F4FA6E05595479504
:10C5D00037952795AA95D1F74101820E931E909227
:10C5E0009D0A80929C0A8091EF0A9091F00A880F30
:10C5F000991FAA2797FDA095BA2F2091A30A332748
:10C6000044275527BC01CD010E9471B15B016C012B
:10C6100097FF08C02FE330E040E050E0A20EB31EC9
:10C62000C41ED51EF6E0D594C794B794A794FA9586
:10C63000D1F78091B10A282F3327442755278091BD
:10C64000120490911304A0911404B0911504BC013C
:10C65000CD010E9471B1DC01CB01BC01CD0120EF05
:10C6600035E540E050E00E94E5B1B501620F731F6F
:10C670007093F00A6093EF0A0150104134F080E0AB
:10C6800090E19093A80A8093A70A8091A70A9091BD
:10C69000A80A8050904F34F480E090EF9093A80A5D
:10C6A0008093A70A51E0851650E1950634F080E0AA
:10C6B00090E190939D0A80939C0A80919C0A9091AE
:10C6C0009D0A8050904F34F480E090EF90939D0A43
:10C6D00080939C0A6150704134F080E090E1909327
:10C6E000F00A8093EF0A8091EF0A9091F00A80504F
:10C6F000904F34F480E090EF9093F00A8093EF0A2B
:10C700008091A90385FD16C080910201992720918F
:10C7100027013091280169817A81689FA001699F72
:10C72000500D789F500D1124CA01B9010E949CB18F
:10C730007A836983809172048150809372048F3F61
:10C7400009F062C08091730490917404892B41F4C4
:10C750008091270190912801909374048093730431
:10C7600080912701909128012091730430917404E5
:10C770002817390718F42F5F3F4F09C08091270110
:10C78000909128018217930730F421503040309364
:10C7900074042093730484E6809372048091F902F8
:10C7A000282F332740917304509174044217530784
:10C7B00030F48AE080939F03809399030EC08091A8
:10C7C0000001280F311D2417350738F480919F038D
:10C7D000882319F0815080939F038091F802282FBD
:10C7E00033274217530710F489E10CC080910001F0
:10C7F000280F311D2417350738F480919E038823B4
:10C8000019F0815080939E0380919F03882369F1E2
:10C810008091CC039091CD03A091CE03B091CF0332
:10C82000B7FD23C0209150082093CB038091D603FD
:10C830009091D703A091D803B091D9038D5D954015
:10C84000A040B04034F0822F9927880F991F809321
:10C85000CB0380EE91EBAFEFBFEF8093CC039093CF
:10C86000CD03A093CE03B093CF0380912C038823F4
:10C8700011F40E946C7289819A81880F991F880F28
:10C88000991F9A8389838091E40A80FD02C00C94E9
:10C89000416E8091BE03882311F00C94416E20916B
:10C8A000BF03222311F00C94416E80915905992702
:10C8B0008F779070009711F00C94416E3C0180913D
:10C8C000380490913904892B09F04BC080911D01E7
:10C8D00090911E018959934058F087B58A3F20F402
:10C8E00080914D03815011C081E08093800467C026
:10C8F00080911D0190911E018436910568F587B5E0
:10C90000863030F180914D038F5F80934D0395E029
:10C9100089029001112480918507821B87BD87B50C
:10C92000809588BD8CE291E090932E0380932D0337
:10C930008091A003882319F082E390E002C08EE585
:10C9400091E090933904809338040E94502437C0BA
:10C9500081E080937F0433C020937F042093800480
:10C960002EC070924C0360924B03F8948091A00308
:10C97000882321F081E00E9432AB17C08091D6035A
:10C980009091D703A091D803B091D90374E0880F98
:10C99000991FAA1FBB1F7A95D1F780934E039093DE
:10C9A0004F03A0935003B0935103789480913804BF
:10C9B00090913904019790933904809338048091C1
:10C9C000E40A9091B90381FF3CC0923348F580910D
:10C9D00098018150809398018F3F09F046C0809163
:10C9E000B001882339F48091F303882319F088E299
:10C9F0008093B0011092F3038091D6039091D703F6
:10CA0000A091D803B091D9038093D2039093D3031C
:10CA1000A093D403B093D50381E08093980125C0FF
:10CA2000973418F18091B001882339F48091F30391
:10CA3000882319F487E28093B00188EC80939801F1
:10CA400011C08091EB07989FC0011124AA2797FD80
:10CA5000A095BA2F8093D2039093D303A093D403CD
:10CA6000B093D50381E08093F30380911A049091F1
:10CA70001B04A0911C04B0911D04E0904501F090AE
:10CA800046010091470110914801BC01CD01A80168
:10CA900097010E94E5B159016A01809116049091B5
:10CAA0001704A0911804B0911904BC01CD01A8018C
:10CAB00097010E94E5B1B901C5010E941FA2209112
:10CAC00079013327829FF001839FF00D929FF00D33
:10CAD0001124CF0164E670E00E94B0B19B016C3379
:10CAE000710514F02CE330E0C9010E94457C90935D
:10CAF000AE0A8093AD0A80E2809344011092D10384
:10CB00001092D0038091F303882309F461C78091C8
:10CB1000A90399279C012071307084FD59C7809129
:10CB2000A80382608093A8037091C00A872F992779
:10CB300061E0862E912C8822992280FD04C080918C
:10CB4000E40A81FD10C009811A8130937604209394
:10CB500075043093D1032093D0038091A903806C96
:10CB60008093A903F4C28091A90381FFC0C2009100
:10CB7000830110918401C8010F962091E603309142
:10CB8000E7033B872A878217930708F096C08091B6
:10CB90007F04882309F091C08091A90387FF15C005
:10CBA0008091A9038F778093A9038091410390918D
:10CBB0004203A0914303B09144038093D203909326
:10CBC000D303A093D403B093D503E090A40AEE203E
:10CBD000D9F18091D2039091D303A091D403B09165
:10CBE000D503BC01CD0124E630E040E050E00E94D6
:10CBF000E5B1AE2CBB24CC24DD24A216B306C406BA
:10CC0000D50614F59092D1038092D0038091B001A3
:10CC10008823C1F48091D6039091D703A091D803C3
:10CC2000B091D903BC01CD012FE530E040E050E0E8
:10CC30000E94E5B1A216B306C406D5061CF48AE12B
:10CC40008093B0018DE37CC080917704909178044B
:10CC5000459784F08091410390914203A091430352
:10CC6000B09144038093D2039093D303A093D40351
:10CC7000B093D5038091A90380648093A9032A858A
:10CC80003B85201B310B2F50304037FF03C03095C0
:10CC900021953F4F3093D1032093D00380919F0380
:10CCA000882349F0C90163E070E00E94B0B170933D
:10CCB000D1036093D0038BE243C0C8010F974A852C
:10CCC0005B854817590708F040C08091800488238D
:10CCD000E1F58091A90386FD07C0809177049091CA
:10CCE0007804845D9E4FACF48091A9038F7B809380
:10CCF000A9038091410390914203A0914303B09115
:10CD000044038093D2039093D303A093D403B093AE
:10CD1000D5038091A90380688093A9038A859B85A8
:10CD2000801B910B0F9697FF03C0909581959F4FA5
:10CD3000909581959F4F9093D1038093D0038DE27E
:10CD4000809344011092CA03D9C08DE380934401BB
:10CD50006091CB03662371F12091CC033091CD0318
:10CD60004091CE035091CF038091D2039091D30391
:10CD7000A091D403B091D50382179307A407B507F8
:10CD8000CCF48091A90380648093A903862F99270E
:10CD90009093D1038093D0038AE08093CA038EE5F9
:10CDA000809344018091A90387FFA8C08091A903C3
:10CDB0008F7733C0662309F443C02091CC033091B0
:10CDC000CD034091CE035091CF038091D203909137
:10CDD000D303A091D403B091D503281739074A078C
:10CDE0005B0774F58091A90380688093A903862F5F
:10CDF0009927909581959F4F9093D1038093D0036D
:10CE000086EF8093CA0386E7809344018091A9034B
:10CE100086FF74C08091A9038F7B8093A9038091C2
:10CE2000410390914203A0914303B0914403809346
:10CE3000D2039093D303A093D403B093D5035EC0E1
:10CE40008091A903807C09F459C08091CA0388238A
:10CE500079F5A0904103B0904203C0904303D09075
:10CE60004403D601C501885C9040A040B0402091A9
:10CE7000D2033091D3034091D4035091D50382174C
:10CE80009307A407B5075CF4D601C50188539F4FEB
:10CE9000AF4FBF4F281739074A075B075CF08093F5
:10CEA000D2039093D303A093D403B093D50302C0CD
:10CEB0001092CA038091A9038F738093A9031092E3
:10CEC00076041092750471FF06C084EF91E0909390
:10CED0002E0380932D038091DA03882379F48091C7
:10CEE000D6039091D703A091D803B091D903C397EB
:10CEF000A105B1051CF081E08093DA03609175040F
:10CF0000709176048091D0039091D103680F791FBE
:10CF10007093760460937504CB0177FF04C0882773
:10CF20009927861B970B855F91400CF4C9C04091EF
:10CF3000CA03442389F18091CC039091CD032091C1
:10CF4000D2033091D303821B930B0996439748F485
:10CF50008091CC039091CD03A091CE03B091CF03EB
:10CF600012C0242F332727FD3095432F532F809154
:10CF7000D2039091D303A091D403B091D503820F33
:10CF8000931FA41FB51F8093D2039093D303A09344
:10CF9000D403B093D50324C02091D2033091D3039E
:10CFA0004091D4035091D5038091EB0716161706D4
:10CFB00044F463E00E9490B1280F311D411D511DC2
:10CFC00007C063E00E9490B1281B31094109510953
:10CFD0002093D2033093D3034093D4035093D503CB
:10CFE0001092760410927504A090D603B090D703E7
:10CFF000C090D803D090D903D601C5018050944089
:10D00000A040B0402091410330914203409143033E
:10D010005091440382179307A407B5075CF4D60127
:10D02000C50180509C4FAF4FBF4F281739074A07A3
:10D030005B0744F08093410390934203A093430322
:10D04000B0934403A0904103B0904203C0904303C7
:10D05000D0904403D601C50180509440A040B04018
:10D060002091D2033091D3034091D4035091D50342
:10D0700082179307A407B5075CF4D601C501845253
:10D080009A4FAF4FBF4F281739074A075B0744F045
:10D090008093D2039093D303A093D403B093D5038A
:10D0A0008091C00A81FF06C084E690E090932E0331
:10D0B00080932D038091CB03882311F40E94945117
:10D0C0008091380490913904892BE9F180914103D2
:10D0D00090914203A0914303B09144038093D20303
:10D0E0009093D303A093D403B093D5032CC081E0D5
:10D0F0000E9432AB8091410390914203A09143037F
:10D10000B0914403805D9740A040B0408093D2032B
:10D110009093D303A093D403B093D5038091EF07EA
:10D12000882311F0992702C08FE790E09093840143
:10D1300080938301E981FA81F093C103E093C003F6
:10D140008EE2809344010091C0031091C103A0902E
:10D150004103B0904203C0904303D0904403209118
:10D16000D2033091D3034091D4035091D5032A15B3
:10D170003B054C055D0524F08091C00A80FD3AC452
:10D180008091A0036091380470913904882309F0DC
:10D190004FC2672B49F00091C0031091C103109258
:10D1A000780410927704DCC0D601C501821B930B72
:10D1B000A40BB50B8093560490935704A093580486
:10D1C000B09359048230F0E89F07FFEFAF07FFEFFD
:10D1D000BF072CF481E090E8AFEFBFEF09C08F5F8D
:10D1E0009F47A040B04064F08FEF9FE7A0E0B0E021
:10D1F0008093560490935704A0935804B093590415
:10D20000809156049091570490937804809377040A
:10D2100080917C01282F332744275527809156047D
:10D2200090915704A0915804B0915904BC01CD01CC
:10D230000E9471B197FF04C0615E7F4F8F4F9F4F77
:10D2400055E095958795779567955A95D1F76093B1
:10D250005604709357048093580490935904653092
:10D260003EEF73073FEF83073FEF93072CF484E013
:10D270009EEFAFEFBFEF09C0605074408040904018
:10D2800064F080E094E0A0E0B0E0809356049093D6
:10D290005704A0935804B0935904609056047090BA
:10D2A000570460914B0370914C0377FF02C0695F94
:10D2B0007F4F9B0143E0359527954A95E1F75FEF56
:10D2C000223835071CF421E83FEF05C0203831052E
:10D2D00014F020E830E0C901AA2797FDA095BA2FE5
:10D2E00020917D01332744275527BC01CD010E94A1
:10D2F00071B197FF04C06D5F7F4F8F4F9F4F22E04A
:10D3000095958795779567952A95D1F79B016FEF4E
:10D31000213036071CF420E03FEF06C02F3F3105D7
:10D3200019F014F020E031E08091A903807C49F0ED
:10D33000C90137FD03969C013595279535952795AD
:10D340000DC08091C00A80FF09C0C90137FD079652
:10D350009C01A3E035952795AA95E1F7620E731E0F
:10D3600020917B01222309F454C06091F60370914F
:10D37000F7038091F8039091F90397FF04C0615877
:10D380007F4F8F4F9F4FF7E09595879577956795DE
:10D39000FA95D1F73327442755270E9471B197FF9B
:10D3A00004C0615E7F4F8F4F9F4FE5E09595879555
:10D3B00077956795EA95D1F7609356047093570473
:10D3C00080935804909359046138AFEF7A07AFEF18
:10D3D0008A07AFEF9A072CF480E89FEFAFEFBFEF1B
:10D3E0000AC06F3F71058105910569F064F080E026
:10D3F00091E0A0E0B0E08093560490935704A0938E
:10D400005804B09359048091560490915704680EC3
:10D41000791EC301AA2797FDA095BA2FC090C0031B
:10D42000D090C1039601442737FD4095542FBC018D
:10D43000CD010E9471B197FF04C061507E4F8F4FA4
:10D440009F4F59E095958795779567955A95D1F7B0
:10D45000061B170B8091D0039091D103892B09F003
:10D4600064C01C141D040CF060C02091770430913E
:10D470007804C90137FF03C0309521953F4F2D3304
:10D48000310540F48091EE039091EF0380179107EE
:10D4900074F526C02C53304045E0369527954A95C3
:10D4A000E1F72031310510F02FE030E04091EE033C
:10D4B0005091EF0318161906E4F480E190E0821B06
:10D4C000930B489F9001499F300D589F300D1124B8
:10D4D00094E0369527959A95E1F72017310720F5C6
:10D4E000809181019091820108171907F4F08C0155
:10D4F0001CC0205F3F4F8091810190918201829FEB
:10D50000F001839FF00D929FF00D11249F0184E0A4
:10D51000369527958A95E1F74017510714F08A014F
:10D5200004C00217130708F08901C801AA2797FD54
:10D53000A095BA2F1DE0880F991FAA1FBB1F1A952F
:10D54000D1F72091AD0A3091AE0A442737FD4095BE
:10D55000542FBC01CD010E94E5B120935A043093B1
:10D560005B0440935C0450935D0400915A04109155
:10D570005B048091790490917A049C01220F331FFF
:10D58000280F391F200F311F37FF02C02D5F3F4F7B
:10D59000A901559547955595479550937A04409321
:10D5A00079048091E707282F3327220F331F220F9A
:10D5B000331F241735076CF48091EC0A282F33278A
:10D5C000220F331F220F331F2055304042175307BD
:10D5D00024F030937A04209379048091C00A80FF6C
:10D5E00014C08091790490917A0429813A8182173C
:10D5F000930724F030937A042093790440917904BE
:10D6000050917A045A834983F5C129813A812C19B2
:10D610003D0937FF02C02D5F3F4F35952795359562
:10D6200027956091790470917A04620F731FCAC1C3
:10D63000672B49F00091C0031091C1031092780448
:10D640001092770432C1D601C501821B930BA40B43
:10D65000B50B8093560490935704A0935804B0934D
:10D660005904823070E897077FEFA7077FEFB7076D
:10D670002CF481E090E8AFEFBFEF09C08F5F9F47C8
:10D68000A040B04064F08FEF9FE7A0E0B0E080934F
:10D69000560490935704A0935804B0935904809172
:10D6A0005604909157049093780480937704809166
:10D6B0007C01282F332744275527809156049091C9
:10D6C0005704A0915804B0915904BC01CD010E94A7
:10D6D00071B197FF04C0615E7F4F8F4F9F4F25E070
:10D6E00095958795779567952A95D1F76093560418
:10D6F0007093570480935804909359046530F8EF61
:10D700007F07FFEF8F07FFEF9F072CF484E098EF70
:10D71000AFEFBFEF09C0605078408040904064F0A8
:10D7200080E098E0A0E0B0E0809356049093570426
:10D73000A0935804B0935904609056047090570415
:10D7400080917B01282F33278091520390915303BE
:10D75000829FA001839F500D929F500D11249A012A
:10D7600057FF02C021503F4F232F330F330B8091BF
:10D770004B0390914C03820F931FAA2797FDA0950E
:10D78000BA2F8093560490935704A0935804B093F3
:10D7900059048091CA032091D0033091D10388238A
:10D7A00031F0B3E0220F331FBA95E1F71BC080912F
:10D7B000EB079927289FB001299F700D389F700DA6
:10D7C00011249B01A3E0220F331FAA95E1F7260F36
:10D7D000371F37FF02C0215E3F4FF5E03595279593
:10D7E000FA95E1F73093A2032093A1038091A1035E
:10D7F0009091A2039C01442737FD4095542F8091BE
:10D80000560490915704A0915804B0915904821B7A
:10D81000930BA40BB50B8093560490935704A093DD
:10D820005804B093590420917D013327442755278C
:10D83000BC01CD010E9471B197FF04C0615E7F4FB2
:10D840008F4F9F4FE5E09595879577956795EA957A
:10D85000D1F76093560470935704809358049093C3
:10D8600059046530A8EF7A07AFEF8A07AFEF9A0740
:10D870002CF484E098EFAFEFBFEF09C06050784020
:10D880008040904064F080E098E0A0E0B0E08093B9
:10D89000560490935704A0935804B0935904809170
:10D8A000560490915704680E791E06191709809145
:10D8B000EE039091EF03801791073CF48091810172
:10D8C00090918201081719070CF08C01C801AA2752
:10D8D00097FDA095BA2F6DE0880F991FAA1FBB1F57
:10D8E0006A95D1F72091AD0A3091AE0A442737FDF1
:10D8F0004095542FBC01CD010E94E5B120935A04FC
:10D9000030935B0440935C0450935D0400915A048F
:10D9100010915B048091790490917A049C01220F0C
:10D92000331F280F391F200F311F37FF02C02D5F13
:10D930003F4F359527953595279530937A04209359
:10D9400079048091A3039091A4038159914020F41C
:10D950008091A80385FF03C08091F30702C08091E6
:10D96000E7079927880F991F880F991F209179043D
:10D9700030917A048217930764F48091EC0A992716
:10D98000880F991F880F991F8055904028173907D5
:10D9900024F090937A04809379048091C00A2091B6
:10D9A000790430917A0480FF10C049815A8124178C
:10D9B000350724F050937A044093790460917904F8
:10D9C00070917A047A83698315C03A83298312C0DF
:10D9D0000E94945189819A8190937A04809379046A
:10D9E0008091A903806C8093A9038091A8038D7F07
:10D9F0008093A8038091A90399279C01227030701D
:10DA000081FF30C180917B0490917C04A0917D04C2
:10DA1000B0917E040097A105B10521F08091DA0351
:10DA20008130B9F48091C0039091C103AA2797FD7A
:10DA3000A095BA2F1EE0880F991FAA1FBB1F1A9529
:10DA4000D1F780937B0490937C04A0937D04B093E2
:10DA50007E048091DA03813019F482E08093DA0346
:10DA6000A981BA817D010027F7FC0095102F8091D4
:10DA7000AD0A9091AE0A9C01442737FD4095542F82
:10DA8000C801B7010E9471B1DC01CB0180935A0437
:10DA900090935B04A0935C04B0935D04B7FF04C053
:10DAA0008150904EAF4FBF4F5C016D01FDE0D594AA
:10DAB000C794B794A794FA95D1F7A0925A04B0925C
:10DAC0005B04C0925C04D0925D046091AA037091E3
:10DAD000AB03BFE0603A7B0750F580917B049091E7
:10DAE0007C04A0917D04B0917E049C01AD01EAE02C
:10DAF0005695479537952795EA95D1F7821B930B55
:10DB0000A40BB50BA601950104E0220F331F441F9F
:10DB1000551F0A95D1F7820F931FA41FB51F80933D
:10DB20007B0490937C04A0937D04B0937E046054A6
:10DB30007F4118F580917B0490917C04A0917D0435
:10DB4000B0917E049C01AD011CE056954795379538
:10DB500027951A95D1F7821B930BA40BB50BA60141
:10DB60009501F2E0220F331F441F551FFA95D1F79C
:10DB7000820F931FA41FB51F38C080914B03909153
:10DB80004C0380914B0390914C0397FF03C09095F9
:10DB900081959F4F8436910584F580914103909142
:10DBA00042032091D2033091D303821B930B815007
:10DBB0009F4F8F5F914008F580917B0490917C048A
:10DBC000A0917D04B0917E049C01AD01EEE05695DC
:10DBD000479537952795EA95D1F7821B930BA40BB0
:10DBE000B50B8A0D9B1DAC1DBD1D80937B049093CE
:10DBF0007C04A0937D04B0937E0480917B0490917B
:10DC00007C04A0917D04B0917E047EE0B695A7953A
:10DC1000979587957A95D1F79093C1038093C00328
:10DC20004091ED07442399F055279C01BA010E94C9
:10DC3000B0B1C901861B970B9093EF038093EE035D
:10DC4000260F371F30938201209381011FC010924D
:10DC5000EF031092EE038FEF93E090938201809395
:10DC6000810114C01092DA0310927B0410927C049C
:10DC700010927D0410927E043093C1032093C00360
:10DC800005C08091A903806C8093A90380918F04C3
:10DC900081FF37C089819A8197FD03969595879575
:10DCA000959587952091A5033091A60328173907EC
:10DCB00060F48091C0039091C103892B31F0220F51
:10DCC000331F220F331F3A832983809141039091A0
:10DCD0004203A0914303B09144038093D2039093F5
:10DCE000D303A093D403B093D50388E99AE3909328
:10DCF0002E0380932D0380E09EE090930D0180938E
:10DD00000C012091AC0A822F9927880F991F880F48
:10DD1000991F889649815A818417950714F09A8330
:10DD200089838091EC0A9927880F991F880F991F82
:10DD30008055904069817A818617970714F49A83F9
:10DD4000898380918803882341F480918C0B8E3FD6
:10DD500020F080919304882311F18091AA0390917F
:10DD6000AB030297C097D8F489819A8118161906D7
:10DD7000B4F481E090E09093AB038093AA03A22FC8
:10DD8000BB27AA0FBB1FAA0FBB1F9896BA83A983F4
:10DD900080918C0B883218F489E08093B0018091D7
:10DDA0002C03882311F40E946C72E981FA81F093AC
:10DDB0004307E09342078091520490915304A0914D
:10DDC0005404B091550412E0880F991FAA1FBB1F7D
:10DDD0001A95D1F70091EF0A1091F00A081B190B60
:10DDE000E13AF1058CF0CF01F7FD01969595879505
:10DDF000801791070CF48C01909581959F4F08171F
:10DE000019076CF48C010BC00135110514F000E505
:10DE100010E0FFEF003B1F0714F400EB1FEF8091B1
:10DE2000EC0A282F3327220F331F220F331FC9017B
:10DE300049815A81841B950B801791070CF48C0142
:10DE400069817A81621B730B061717070CF48B012B
:10DE50008091A70A9091A80A6091EC037091ED035C
:10DE6000861B970B9093B30A8093B20AD090C20A94
:10DE70002091FE033091FF03409100045091010472
:10DE8000DD2041F0461A570AC201AA2797FDA09546
:10DE9000BA2F04C0AA2797FDA095BA2F280F391FC3
:10DEA0004A1F5B1F2093FE033093FF03409300043F
:10DEB000509301048091FE039091FF03A091000410
:10DEC000B091010481509A4FA040B04064F080E0CE
:10DED0009AEFA0E0B0E08093FE039093FF03A0933D
:10DEE0000004B09301048091FE039091FF03A09180
:10DEF0000004B091010480509640AF4FBF4F64F4CE
:10DF000080E096E0AFEFBFEF8093FE039093FF03B6
:10DF1000A0930004B0930104C090FC072091B20AC2
:10DF20003091B30A78E07C1598F08C2D9927829F68
:10DF3000D001839FB00D929FB00D1124CD01B7FD8C
:10DF400007965C0163E0B594A7946A95E1F712C067
:10DF50008C2D86959927829FF001839FF00D929FCB
:10DF6000F00D1124CF01F7FD03965C01B594A79441
:10DF7000B594A79480907E0190907F0194014427EE
:10DF800037FD4095542F8091FE039091FF03A0919F
:10DF90000004B0910104BC01CD010E94E5B1A20EC4
:10DFA000B31EE09068016E2D772788279927980186
:10DFB00017FF04C022273327201B310B37FF02C075
:10DFC0002F5F3F4F3595279549815A81240F351F83
:10DFD000442737FD4095542F0E9471B197FF04C02C
:10DFE000615C7F4F8F4F9F4F26E095958795779582
:10DFF00067952A95D1F79B016A157B050CF45B01A7
:10E0000066277727621B730BA616B7060CF45B0115
:10E0100080919C0A90919D0A6091EA037091EB03B4
:10E02000861B970B90939B0A80939A0A2091FA0380
:10E030003091FB034091FC035091FD03DD2041F042
:10E04000261A370AC101AA2797FDA095BA2F04C046
:10E05000AA2797FDA095BA2F280F391F4A1F5B1FCB
:10E060002093FA033093FB034093FC035093FD038A
:10E070008091FA039091FB03A091FC03B091FD0302
:10E0800081509A4FA040B04064F080E09AEFA0E049
:10E09000B0E08093FA039093FB03A093FC03B0934A
:10E0A000FD038091FA039091FB03A091FC03B091D2
:10E0B000FD0380509640AF4FBF4F64F480E096E080
:10E0C000AFEFBFEF8093FA039093FB03A093FC03A1
:10E0D000B093FD0320919A0A30919B0A78E07C1559
:10E0E00098F08C2D9927829FD001839FB00D929F2D
:10E0F000B00D1124CD01B7FD07966C01B3E0D594A6
:10E10000C794BA95E1F712C0C6948C2D9927829FC7
:10E11000F001839FF00D929FF00D1124CF01F7FDC8
:10E1200003966C01D594C794D594C7949401442761
:10E1300037FD4095542F8091FA039091FB03A091F5
:10E14000FC03B091FD03BC01CD010E94E5B1C20EFC
:10E15000D31E6E2D772788279927980117FF04C0B3
:10E1600022273327201B310B37FF02C02F5F3F4F81
:10E170003595279549815A81240F351F442737FD4E
:10E180004095542F0E9471B197FF04C0615C7F4F8E
:10E190008F4F9F4FE6E09595879577956795EA9520
:10E1A000D1F79B016C157D050CF46B016627772771
:10E1B000621B730BC616D7060CF46B0180912C03FF
:10E1C000882311F40E946C728091AC0A682F772723
:10E1D0007D836C838091EC0AA82FBB27BF83AE831D
:10E1E000E0903F0860E1862E69E0962E57E7652EA5
:10E1F00058E0752E4FE0342E33EC432E3AE0532E88
:10E20000F301208112160CF030C1203429F4298149
:10E210003A813B872A871FC049815A81CA01AA27B0
:10E2200097FDA095BA2F332727FD3095432F532F05
:10E23000BC01CD010E9471B197FF04C0615C7F4FAA
:10E240008F4F9F4F26E095958795779567952A95EF
:10E25000D1F77B876A87F3012181203439F42A853D
:10E260003B852A0D3B1D3B872A872AC0203C39F479
:10E270004A855B854A195B095B874A8721C0C501CE
:10E28000AA2797FDA095BA2F332727FD3095432F56
:10E29000532FBC01CD010E9471B197FF04C0615C96
:10E2A0007F4F8F4F9F4FB6E09595879577956795F0
:10E2B000BA95D1F7AA85BB85A60FB71FBB87AA87DA
:10E2C000F3012281203439F42A853B852C0D3D1D34
:10E2D0003B872A872AC0203C39F44A855B854C1944
:10E2E0005D095B874A8721C0C601AA2797FDA095D3
:10E2F000BA2F332727FD3095432F532FBC01CD0173
:10E300000E9471B197FF04C0615C7F4F8F4F9F4F98
:10E31000A6E09595879577956795AA95D1F7AA85F3
:10E32000BB85A60FB71FBB87AA87F30123812034C3
:10E3300039F42A853B85200F311F3B872A872AC065
:10E34000203C39F44A855B85401B510B5B874A872B
:10E3500021C0C801AA2797FDA095BA2F332727FD12
:10E360003095432F532FBC01CD010E9471B197FF0F
:10E3700004C0615C7F4F8F4F9F4FF6E09595879566
:10E3800077956795FA95D1F7AA85BB85A60FB71F34
:10E39000BB87AA87F401808181FD08C0D2018D91DD
:10E3A0009C91EA85FB858E179F0774F4D2018D91AD
:10E3B0009C91EA85FB858E0F9F1F97FD0196959591
:10E3C00087959B878A871EC0EE2049F42A853B8566
:10E3D000220F331F281B390B3B872A8713C031E0DC
:10E3E0003E1580F42E2D33274A855B85841B950BC3
:10E3F000B9010E94B0B1CB016A857B85680F791F96
:10E400007B876A878C819D81880F991F880F991F50
:10E41000AA85BB858A179B075CF48E819F81880F34
:10E42000991F880F991FEA85FB85E817F90714F0F3
:10E430009B878A878A859B8597FD03969595879507
:10E4400095958795F4018183880F991F880F991FEF
:10E450002A853B85281B390BC901880F8283EA85F1
:10E46000FB85D201ED93FC9303C0F401118212826B
:10E470003A9422E030E0420E531E44E050E0640E35
:10E48000751E6FE070E0860E971E37FEB9CEE2E192
:10E49000C55F0C941CB284B1806A84B93D9A82E550
:10E4A0008CBD1DBC459A81E08093000B8AEA809365
:10E4B000110B83E88093120B8AE08093130B109268
:10E4C000150B1092140B1092170B1092160B109242
:10E4D000790B1092350B08953091000B332309F01E
:10E4E00070C00DB407FE6DC085E080932C03459A83
:10E4F0002EB58091970499278130910589F082305B
:10E5000091051CF4892B21F03EC00297B9F03BC065
:10E510003093340B209398042138A9F581E008C08A
:10E52000253549F480919804820F8093980482E005
:10E530008093970428C03093970425C08091340BB2
:10E54000E82FFF27EA5AF44F20838F5F8093340B24
:10E55000909198048032A0F0291769F480E2A6E532
:10E56000BBE0E6E3FBE00D9001928A95E1F781E0E4
:10E570008093350B02C03093350B1092970403C083
:10E58000920F909398042091100B2232A0F445989A
:10E590000000000000000000E091090BF0910A0B60
:10E5A000E20FF11D80818EBD8091320B9081890F29
:10E5B0008093320B03C081E08093000B2F5F209388
:10E5C000100B0895EF92FF920F931F93CF93DF9359
:10E5D0008091F5079927880F991F880F991F7C0153
:10E5E0000027F7FC0095102F80911A0490911B04CE
:10E5F000A0911C04B0911D04BC01CD01A80197019C
:10E600000E94E5B13093150B2093140B80911604F2
:10E6100090911704A0911804B0911904BC01CD0188
:10E62000A80197010E94E5B13093170B2093160BB8
:10E630002091F60A3091F70A4091F80A5091F90AB0
:10E64000DA01C90163E0880F991FAA1FBB1F6A95F1
:10E65000D1F7820F931FA41FB51F820F931FA41F12
:10E66000B51F2091450130914601409147015091DD
:10E670004801BC01CD010E94E5B130931D0B2093F0
:10E680001C0BC0913204D0913304809158039091B7
:10E6900059039E01281B390B3093230B2093220B27
:10E6A000E0912204F09123048091B90A9091BA0A72
:10E6B000BF010E94B0B19B01220F331F220F331FF5
:10E6C000260F371F260F371F37FF02C02D5F3F4F22
:10E6D00035952795359527953093190B2093180B71
:10E6E0008091F20A9091F30ABF010E94B0B19B01A0
:10E6F000220F331F220F331F260F371F260F371FFE
:10E7000037FF02C02D5F3F4F3595279535952795EB
:10E7100030931B0B20931A0B1092230410922204A7
:10E720001092BA0A1092B90A1092F30A1092F20AE1
:10E730008091130B99278C30910509F44EC28D30CE
:10E7400091053CF48A30910599F00B9709F416C2B3
:10E75000A7C28131910509F4BFC18231910524F42A
:10E76000409709F442C09CC2439709F4A6C098C2DE
:10E770008091B8038093260B8091B7038093270B79
:10E780008091B6038093280B8091B5038093290B69
:10E790008091B40380932A0B8091B30380932B0B59
:10E7A0008091B20380932C0B8091B10380932D0B49
:10E7B0008091A90380932E0B8091A80380932F0B47
:10E7C0008091A903837F8093A90380912701909171
:10E7D00028019093310B8093300B429961C2809154
:10E7E000A803877F8093A8035BC28091860B9091DA
:10E7F000870B9093270B8093260B8091990490911F
:10E800009B04892B8093280B80918C0B8093290B80
:10E8100080912A080E94594E80932A0B80914401CE
:10E8200080932B0B20919904822F9927FC01C4E03F
:10E83000EE0FFF1FCA95E1F7E81BF90BE05FF64FFB
:10E84000868580932C0B808180932D0B868180930D
:10E850002E0B838180932F0B87818093300B8581D2
:10E860008093310B2F5F20939904E22FFF27EE0F47
:10E87000FF1FEE0FFF1FE659F74F85851816D4F0DE
:10E880002223C1F0822F992701966DE070E00E944B
:10E89000B0B1AC01282FE82FFF27EE0FFF1FEE0FBE
:10E8A000FF1FE659F74F8585181614F0442351F7DA
:10E8B0004093990410929B04F3C120919A04822FF3
:10E8C000992781309105E9F1823091051CF4892B5B
:10E8D00049F0D0C08230910509F465C0039709F46E
:10E8E00096C0C8C08EE08093130B82E08093260B05
:10E8F0008CE08093270B1092280B8CE48093290BDB
:10E900008091030180932A0B8091500880932B0BF8
:10E910008091400880932C0B8091540880932D0B9C
:10E9200080915C0580932E0B8091010180932F0BC9
:10E930008091F4029091F5029093310B8093300B0B
:10E9400095C08DE08093130B809102018093260B7C
:10E9500080912B088093270B80912C088093280BA3
:10E9600080912D088093290B80912E0880932A0B8B
:10E970008091320880932B0B8091330880932C0B6D
:10E980008091340880932D0B8091370880932E0B53
:10E990008091350880932F0B809136088093300B3F
:10E9A0008091380831C084E18093130B80912C044E
:10E9B00090912D049093270B8093260B80912A042D
:10E9C00090912B049093290B8093280B809128041D
:10E9D0009091290490932B0B80932A0B809110081F
:10E9E00080932C0B8091510880932D0B8091E40A29
:10E9F00080932E0B8091C00A80932F0B80913C084E
:10EA00008093300B80915C088093310B2FC08FE096
:10EA10008093130B809170018093260B80916F017E
:10EA20008093270B80913A088093280B8091A40A49
:10EA30008093290B80915A0880932A0B80910001C2
:10EA400080932B0B80919C0490919D0490932D0BAF
:10EA500080932C0B80919F0380932E0B8091410813
:10EA600080932F0B1092300B1092310B2F5F20935D
:10EA70009A0416C182E18093130B80913604909121
:10EA800037049093270B8093260B80913404909148
:10EA900035049093290B8093280BD0932B0BC093B4
:10EAA0002A0B80911D0880932C0B8091390880934C
:10EAB0002D0B8091000880932E0B80912F0880935E
:10EAC0002F0B809130088093300B80913108809318
:10EAD000310B10929A04E4C0809129088093260B90
:10EAE00080910008863081F08091F002823451F0EC
:10EAF0000E94AF81E82FFF27E052F84E8491809367
:10EB0000F00202C00E94AF818091C9048093270B5C
:10EB100080918A0B90918B0B9093290B8093280BFB
:10EB200080919E0380932A0B8091D60480932B0BB7
:10EB30008091D40480932C0B8091D30480932D0B6F
:10EB40001092D6041092D4041092D30480917A01CA
:10EB5000882329F08091F4039091F50304C08091FB
:10EB6000A10A9091A20A90932F0B80932E0B809173
:10EB7000A7038093300B8091550890C080914D0A77
:10EB80008093260B8091000A8093270B8091020AC4
:10EB90008093280B8091050A8093290B8091DD03D7
:10EBA00080932A0B8091DE0380932B0B8091DF03EF
:10EBB00080932C0B8091E00380932D0B8091E103D7
:10EBC00080932E0B8091E20380932F0B8091E303BF
:10EBD0008093300B8091E40361C08091740585308F
:10EBE00018F01092740585E08093260B8091C00385
:10EBF0009091C10397FD0396959587959595879577
:10EC00008093270B8091D6039091D703A091D803CE
:10EC1000B091D903BC01CD0125E030E040E050E0E7
:10EC20000E94E5B13093290B2093280B8091D203E9
:10EC30009091D303A091D403B091D503BC01CD0131
:10EC400025E030E040E050E00E94E5B130932B0B2E
:10EC500020932A0B8091590580932C0B90915A0593
:10EC600090932D0B8F7780935905907190935A054F
:10EC700080916C0780932E0B8091DC0380932F0B87
:10EC800080919E048093300B8091420790914307BE
:10EC900097FD039695958795959587958093310B6C
:10ECA0008091350B882309F474C16091360B8091F3
:10ECB000A901681719F08AEF8093A7016093A90151
:10ECC00081E0809390014091370B5091380BCA013D
:10ECD00081509E4F8F5F9340B0F42091390B30915B
:10ECE0003A0BC90181509E4F8F5F934060F4809131
:10ECF000E60785FF08C05093850440938404309351
:10ED000083042093820480913D0B90913E0B21E07F
:10ED10008936920724F49093940180939301209173
:10ED2000470B3091480B80912D0390912E03821751
:10ED3000930740F48091FA02882321F430932E0344
:10ED400020932D03862F99278936910509F48BC0CE
:10ED50008A36910544F48736910571F0883691051D
:10ED600009F44CC01EC18A36910509F40FC18B36D7
:10ED7000910509F4D1C015C18091490B8093760BA0
:10ED800080914A0B8093780B80914B0B8093770B8B
:10ED900080914C0B80938F0180914D0B80FF03C0BD
:10EDA00081E080938E0480914E0B8093A801809126
:10EDB0004F0B809396048091500B80938104809137
:10EDC000510B9091520B97FD04C090939201809348
:10EDD000910120918C0430918D048091530B90917E
:10EDE000540B280F391F37FF02C02F5F3F4F359557
:10EDF000279530938D0420938C04D3C08091490BC8
:10EE000080930B0B80914A0B80930C0B80914B0BE2
:10EE100080930D0B80914C0B80930E0B80914D0BCA
:10EE200080930F0B8091320790914E0B892B80932A
:10EE3000320790913307937080914F0B8C70982B11
:10EE4000909333078091500B809393048091510BE2
:10EE5000809399018091520B8093790B8091530B91
:10EE600080938F049EC08091490B8093010B809109
:10EE70004A0B8093020B80914B0B8093030B809184
:10EE80004C0B8093040B80914D0B90914E0B909303
:10EE9000060B8093050B80914F0B9091500B909334
:10EEA000080B8093070B80919504882329F48091A7
:10EEB000510B8158809395048091510B992787FDC0
:10EEC00090959093420A8093410A8091520B8093CF
:10EED000CB038091530B9091540B9C01442737FD39
:10EEE0004095542FDA01C90163E0880F991FAA1FCA
:10EEF000BB1F6A95D1F7820F931FA41FB51F820F06
:10EF0000931FA41FB51F8093CC039093CD03A093B0
:10EF1000CE03B093CF0345C08091490B80939204F8
:10EF200080914A0B8093910480914B0B80939004C5
:10EF300090914C0B992349F08091B001882319F0EE
:10EF40008151833010F49093B00180914F0B9091D8
:10EF5000500B9093CE048093CD0480914D0B809301
:10EF6000D90480914E0B8093D8048091510B8093EB
:10EF7000D7048091520B8093D5048091530B9091CC
:10EF8000540B9093EE0A8093ED0A0BC00E941C82F2
:10EF900008C0109285041092840410928304109289
:10EFA0008204E6E0CDB7DEB70C9428B28091000B66
:10EFB000882319F480E090E00895459881E19BE072
:10EFC00090930A0B8093090B90919404E92FFF27EB
:10EFD000E656FE4F9F5F9093940480818093130BBD
:10EFE0009D3010F0109294041092000B0E94E27277
:10EFF00081E08093100B8091110B8093320B8EBDBA
:10F0000081E090E0089587B18C6087B94298439879
:10F010001092A00480E88093AB0110929F0480932B
:10F02000AA01089580919E04882339F48091410AB1
:10F030009091420A81588093AB048091A50481503D
:10F040008093A5048F3F09F06DC1809123088093C0
:10F05000A704809125088093A80489E08093A504E3
:10F060008091A903992780739070892B41F4809136
:10F070005A0580FD04C08091DC038823E9F4809167
:10F080002708882351F08091A904882319F484E08B
:10F090008093A00481E08093A904809128088823AC
:10F0A00079F08091AA04882319F484E080939F0466
:10F0B00081E08093AA0404C01092A9041092AA04CB
:10F0C0008091A904882309F088C080915908282FCD
:10F0D000332724FF07C08091DB03882319F425FD23
:10F0E00095C096C090912408983F48F08091BB0A43
:10F0F0008D3D28F08091A70488236CF00AC0983FCA
:10F1000078F08091BB0A853059F48091A70487FF7D
:10F1100002C0429A01C0429881E08093AB015AC07C
:10F120008091A00481508093A0048F3F09F071C0AA
:10F1300080915C0885FF35C09091AB04892F86953E
:10F140008093A004992361F490939E048091A70476
:10F1500087FF02C0429A01C042981092AB0159C089
:10F1600081E080939E048091AB019091A704882355
:10F1700059F4809195048093AB0480E48093AB01B3
:10F1800099230CF443C044C0982311F0429A01C063
:10F19000429886958093AB018130D9F51092950401
:10F1A00038C08091BB0A86958093A0048091AB0102
:10F1B000813021F41092AB0480E401C086958093E5
:10F1C000AB018091AB019091A704892311F0429A81
:10F1D00001C0429810929E041CC08091A0048150EE
:10F1E0008093A0048F3FA9F489E08093A0048091CC
:10F1F000AB01813011F480E801C086958093AB01AA
:10F200008091AB0190912708892311F0429A01C0A7
:10F2100042988091AA04882309F043C0909159082C
:10F2200097FF07C08091DB03882319F496FD52C035
:10F2300053C090912608983F48F08091EB0A8D3D8D
:10F2400028F08091A80488236CF00AC0983F78F0D9
:10F250008091EB0A853059F48091A80487FF02C0A1
:10F26000439A01C0439881E08093AA0136C08091FF
:10F270009F04815080939F048F3F79F58091EB0A22
:10F28000869580939F048091AA01813011F480E4D7
:10F2900001C086958093AA018091AA019091A8044B
:10F2A00017C080919F04815080939F048F3FA9F4E1
:10F2B00089E080939F048091AA01813011F480E855
:10F2C00001C086958093AA018091AA019091280897
:10F2D000892311F0439A01C04398429B15C0809145
:10F2E000A60482FD0CC080E880939B0480919C045E
:10F2F00090919D04019690939D0480939C0480912D
:10F30000A80388608093A803439B04C08091A8034E
:10F31000806103C08091A8038F7E8093A80388B189
:10F320008093A60408950F931F93CF93DF93482FE4
:10F33000EB018091DC03E42FFF27843BD8F08F01A1
:10F340000E0F1F1FF801E95FF54F808191819B012E
:10F35000281B390BC90163E070E00E94B0B1CB01FA
:10F36000880F991F860F971F015B154FF801918336
:10F37000808306C0EE0FFF1FE15BF54F1182108204
:10F38000E42FFF27EE0FFF1FE95FF54FD183C08306
:10F39000DF91CF911F910F9108954FB724E130E095
:10F3A000F8948091C9008F778093C9008091C9003B
:10F3B0008F7B8093C9008091C9008F7D8093C900A5
:10F3C000832F99278093CD002093CC008091C80093
:10F3D00082608093C80080E18093C9008091CA0058
:10F3E0008F778093CA008091CA008F7B8093CA0078
:10F3F0008091CA008F7D8093CA008091CA008F7E61
:10F400008093CA008091CA00877F8093CA00809150
:10F41000C9008B7F8093C9008091CA00846080936B
:10F42000CA008091CA0082608093CA008091C8009F
:10F4300087FF03C08091CE00F9CF8091C90080681A
:10F440008093C9004FBF0895EF92FF920F931F93CF
:10F45000CF93DF93482F00E010E08091AC01813022
:10F4600061F41092AC0184E48093AE041092B00475
:10F470001092AF041092B10403C28091AE048823AD
:10F4800019F421E030E001C098019091AF04992374
:10F4900071F4232B11F081E010C084E48093AE045A
:10F4A0009093B0049093AF049093B104D2C1913083
:10F4B00069F4232B09F0C3C182E08093AF048091EB
:10F4C000B0048F5F8093B00483E0C1C19230D1F467
:10F4D000232B09F0B4C183E08093AE044093B104C0
:10F4E0009091B004923039F41092B20447FF03C0F7
:10F4F00081E08093B20483E08093AF049F5F909398
:10F50000B004A7C1933009F09AC1232B09F097C129
:10F510009093AE0482E08093AF048091B0048F5F3B
:10F520008093B0042091B104822F9927782F662709
:10F53000842F9927682B792B80910008813051F412
:10F540007370CB018050924063E070E00E94B0B1D4
:10F55000EB0119C0823069F47770CB018050944080
:10F5600066E070E00E94B0B1EB01269526952695E5
:10F570000CC0EB01D370C856D140CE01D7FD019627
:10F58000EC01D595C79526952695022F11270F706A
:10F5900010700F5F1F4F0D30110508F049C1023088
:10F5A000110519F404E010E005C00430110511F450
:10F5B00002E010E0D801A00FB11FFD01E95FF54F97
:10F5C000808191819E01281B390BC90137FF03C03F
:10F5D000909581959F4F069704F5E0914308EE239F
:10F5E00051F0FF27EE0FFF1FE95FF54F80819181FA
:10F5F0008436910594F48091DC03883C30F480914A
:10F60000DC03865F8093DC0308C088EC8093DC0316
:10F6100080916F008F7D80936F00A95FB54F8D91B2
:10F620009C91BC01660F771F680F791F6C0F7D1FBF
:10F6300077FF02C06D5F7F4F7B01F594E794F594EF
:10F64000E794CE0101968E159F0524F40894E108F5
:10F65000F10808C0CE010197E816F9061CF40894D9
:10F66000E11CF11C0630110509F0CEC0C536D105EC
:10F670000CF4A5C09091AD04E92FFF27E558F44F95
:10F68000E081ED3729F48091AC0480958093AC043F
:10F69000963061F48091AC04882311F0E338B9F01E
:10F6A000882309F088C0ED3791F085C0993009F0C2
:10F6B00082C08091AC04882329F48091840B833824
:10F6C00031F079C08091840B8D3709F074C080913E
:10F6D0007C0B8D3739F480917D0B833899F463E886
:10F6E0007FEF0DC0833871F480917D0B833819F45E
:10F6F00060E070E004C08D3729F46DE770E085E0CC
:10F700000E94937980917E0B992787FD9095BC018B
:10F7100086E00E94937980917F0B992787FD9095D1
:10F72000BC018BE00E9493798091800B992787FD23
:10F730009095BC018CE00E9493798091AD04893052
:10F74000D1F58091820B8D3749F48091170A909101
:10F75000180A0596BC0188E00E9493798091830B7A
:10F760008D3749F48091170A9091180A0597BC01CA
:10F7700088E00E9493798091170A9091180A835823
:10F780009F4F1CF483E89FEF09C08091170A909166
:10F79000180A8E37910534F08DE790E09093180A9F
:10F7A0008093170A8091810B992787FD9095BC0162
:10F7B0008AE00E9493791092AD041092AC04CA3092
:10F7C000D1055CF48091AD048F5F8093AD04E82F88
:10F7D000FF27E558F44F83E880838091AD048A3099
:10F7E00011F41092AD048FEFCC39D8076CF48091EE
:10F7F000AD04E82FFF27E558F44F8DE78083809113
:10F80000AC0480958093AC040530110518F4B70161
:10F81000802F0BC00530110519F4BE0187E005C02B
:10F8200007301105B1F4BE0189E00E94937911C03F
:10F830000231110570F081E08093AC010AC081E0D3
:10F840008093AC011092B0041092B20484E48093CF
:10F85000AE048091B004803198F08091B204882386
:10F8600031F48091AC01882311F48093430110920C
:10F87000B0041092B2041092AF0484E48093AE04FA
:10F88000E6E0CDB7DEB70C9428B2CF93EAE5F0E01E
:10F89000E81BF90BF7FF05C0CFEFF095E195FF4F9F
:10F8A00001C0C1E028E631E0CF01B9010E94B0B14A
:10F8B000FC018B35910554F08B5590408A359105AC
:10F8C00038F484EB90E08E1B9F0BFC0141E00DC0EF
:10F8D000CF01855B90408A35910518F4E45BF040D8
:10F8E00003C02E1B3F0BF9014FEFEE0FFF1FE1543A
:10F8F000F54F259134918C2F992787FD9095289F5E
:10F90000B001299F700D389F700D1124842F992705
:10F9100087FD9095689FA001699F500D789F500DBD
:10F920001124CA01CF910895089508950895089566
:10F930000895089580E00E94FBA385E79BE09F93D4
:10F940008F938EEE93EA9F938F93E0913905F09118
:10F950003A0509950F900F900F900F90089580E051
:10F960000E94FBA386E89BE09F938F938EEE93EA21
:10F970009F938F93E0913905F0913A0509950F9087
:10F980000F900F900F90089580E00E94FBA387E9ED
:10F990009BE09F938F938EEE93EA9F938F93E091DA
:10F9A0003905F0913A0509950F900F900F900F903F
:10F9B0000895FF920F931F93CF93DF93F82E80E06B
:10F9C0000E94FBA387EA9BE09F938F930EEE13EABE
:10F9D0001F930F93E0913905F0913A0509958091B5
:10F9E000A9030F900F900F900F9080FFAAC08091F5
:10F9F0009901803229F08F3219F08D3209F0A1C0BF
:10FA000080911D08882319F486E080931D0880E00A
:10FA10000E94FBA380912404909125049F938F93CF
:10FA200080912604909127049F938F9387EB9BE00E
:10FA30009F938F93CEEED3EA1F930F93E0913905F6
:10FA4000F0913A0509958DB79EB708968DBF8091C4
:10FA5000050A9091060A892B31F48091020A90914F
:10FA6000030A892BF9F080E10E94FBA38091020A2E
:10FA70009091030A9F938F938091050A9091060AB3
:10FA80009F938F9388EC9BE09F938F93DF93CF930B
:10FA9000E0913905F0913A0509958DB79EB7089622
:10FAA0008DBF1CC08091B304882331F080E10E9497
:10FAB000FBA387ED9BE005C080E10E94FBA388EEDD
:10FAC0009BE09F938F93DF93CF93E0913905F09163
:10FAD0003A0509950F900F900F900F909FE2F9163D
:10FAE00031F48091260490912704019608C08FE498
:10FAF000F81681F480912604909127040197909341
:10FB000027048093260482E88093F00281E08093AA
:10FB1000B30464C09FE1F91631F4809124049091FC
:10FB20002504019609C08FE8F81609F057C08091A6
:10FB30002404909125040197909325048093240434
:10FB4000E2CF8091A90380FD37C09FE8F91621F428
:10FB50001092AD011092B3048091B304882331F464
:10FB600080E10E94FBA389EF9BE02BC08130E1F490
:10FB700080E10E94FBA38AE09CE09F938F931F93F8
:10FB80000F93E0913905F0913A0509950F900F9088
:10FB90000F900F908FE1F81609F50E94574382E805
:10FBA0008093F00282E0B3CF8230C1F480E10E9402
:10FBB000FBA38AE19CE005C080E10E94FBA38BE2ED
:10FBC0009CE09F938F931F930F93E0913905F091E1
:10FBD0003A0509950F900F900F900F90E5E0CDB783
:10FBE000DEB70C9429B21F93CF93DF93182F80E0D8
:10FBF0000E94FBA38CE39CE09F938F93CEEED3EA0D
:10FC0000DF93CF93E0913905F0913A0509950F9074
:10FC10000F900F900F908091D504882331F480E1EC
:10FC20000E94FBA388E49CE009C08091030B833011
:10FC300099F080E10E94FBA383E59CE09F938F9362
:10FC4000DF93CF93E0913905F0913A0509950F9034
:10FC50000F900F900F90DBC08091B4048823C1F007
:10FC60008BE00E94FBA38091B40499279F938F930C
:10FC70008EE59CE09F938F93DF93CF93E0913905BE
:10FC8000F0913A0509958DB79EB706968DBF12C0C3
:10FC90008BE00E94FBA382E69CE09F938F93DF930F
:10FCA000CF93E0913905F0913A0509950F900F90A7
:10FCB0000F900F9080E10E94FBA38091D60390915A
:10FCC000D703A091D803B091D903BC01CD0124E69C
:10FCD00030E040E050E00E94E5B13F932F938091E7
:10FCE000ED0A9091EE0A9F938F9385E69CE09F9397
:10FCF0008F93DF93CF93E0913905F0913A05099501
:10FD00008DB79EB708968DBF8091B504882351F0BA
:10FD10008EE00E94FBA386E79CE09F938F93DF9386
:10FD2000CF930BC08EE00E94FBA389E79CE09F93DA
:10FD30008F938EEE93EA9F938F93E0913905F09124
:10FD40003A0509950F900F900F900F901F3251F4C4
:10FD50009091B4048091D5049817D8F49F5F909344
:10FD6000B40409C01F3459F48091B404823088F07F
:10FD700081508093B40481E08093B5040AC01F31A0
:10FD800041F48091B404882321F08093D30410922D
:10FD9000B50480915808E82FFF27EE0FFF1FE95F99
:10FDA000F54F80819181C3978CF082E08093AE0102
:10FDB0008091B6049091B7040E940420882339F101
:10FDC0001092B40481E08093AE0121C080819181C2
:10FDD0008E5C9F4FE4F484EC99E00E94FB1F9093AB
:10FDE000B7048093B6048091AE01823071F4909193
:10FDF000B4048091D504981740F4892F8F5F8093C5
:10FE0000B4048093D3041092B5041092AE01DF9134
:10FE1000CF911F9108951F93CF93DF93182F80E008
:10FE20000E94FBA38CE79CE09F938F93CEEED3EAD6
:10FE3000DF93CF93E0913905F0913A0509950F9042
:10FE40000F900F900F908091D504882399F480E152
:10FE50000E94FBA387E89CE09F938F93DF93CF934F
:10FE6000E0913905F0913A0509950F900F900F90A8
:10FE70000F90EEC08091B8048823C1F08BE00E94FF
:10FE8000FBA38091B80499279F938F9382E99CE00C
:10FE90009F938F93DF93CF93E0913905F0913A05CB
:10FEA00009958DB79EB706968DBF12C08BE00E9454
:10FEB000FBA386E99CE09F938F93DF93CF93E09120
:10FEC0003905F0913A0509950F900F900F900F901A
:10FED0008091D804882359F180E10E94FBA380918E
:10FEE000CC039091CD03A091CE03B091CF03BC0180
:10FEF000CD0124E630E040E050E00E94E5B13F93C0
:10FF00002F938091CD049091CE049F938F9389E994
:10FF10009CE09F938F93DF93CF93E0913905F0910D
:10FF20003A0509958DB79EB708968DBF12C088E136
:10FF30000E94FBA38BEA9CE09F938F93DF93CF9368
:10FF4000E0913905F0913A0509950F900F900F90C7
:10FF50000F908091B904CEEED3EA882331F08EE081
:10FF60000E94FBA38CEB9CE005C08EE00E94FBA3EB
:10FF70008FEB9CE09F938F93DF93CF93E0913905B4
:10FF8000F0913A0509950F900F900F900F901F3246
:10FF900051F49091B8048091D5049817D8F49F5FDC
:10FFA0009093B80409C01F3459F48091B80482308A
:10FFB00088F081508093B80481E08093B9040AC02E
:10FFC0001F3141F48091B804882321F08093D40438
:10FFD0001092B90480915808E82FFF27EE0FFF1FF9
:10FFE000E95FF54F80819181C3978CF082E0809327
:10FFF000AF018091BA049091BB040E940420882331
:020000021000EC
:1000000039F11092B80481E08093AF0121C0808162
:1000100091818E5C9F4FE4F484EC99E00E94FB1F79
:100020009093BB048093BA048091AF01823071F445
:100030009091B8048091D504981740F4892F8F5F70
:100040008093B8048093D4041092B9041092AF0145
:10005000DF91CF911F91089508950895089580E04C
:1000600090E008951092870B1092860B10928B0BE4
:1000700010928A0B1092890B1092880B10928C0BA5
:1000800082E390E00E94FB1F9093BD048093BC0428
:1000900008959927FC0124E0EE0FFF1F2A95E1F750
:1000A000E81BF90BE05FF64F95819F3F19F480E064
:1000B00090E00895993C18F4892F9927089580813C
:1000C00082FF07C08AE0989FC001112488509740A2
:1000D0000895892F99270895A0E0B0E0E2E7F0E8BD
:1000E0000C9409B28091BC049091BD040E9404203C
:1000F000882309F4D6C08091BC049091BD04C296B7
:100100009093BD048093BC04C0E0D0E07E01BB248A
:100110007FEFC72E80918C0B8E3F29F48091A7032F
:1001200081608093A703DB2C00E119E0F801838153
:1001300087FF1CC0B3948581893C30F08D2D0E94CF
:100140004980C80FD91F02C0C80FD11DF801818195
:10015000E80EF11C8681C81610F0C82E07C08F3F2C
:1001600029F48091A7038E7F8093A703D394015F26
:100170001F4FFFE0FD15D0F6C0928C0BEF2869F5FC
:100180002091C2043091C3044091C4045091C5042D
:10019000BB27A52F942F832F9093C1048093C00475
:1001A000AA27BB27281B390B4A0B5B0BCE01AA27BA
:1001B000BB27280F391F4A1F5B1F2093C2043093AF
:1001C000C3044093C4045093C504C5E0D0E08091BB
:1001D000A7038E7F8093A70313C08091C0049091E2
:1001E000C1048C179D0718F4C81BD90B02C0C0E0CE
:1001F000D0E08B2D9927880F991FC80FD91F2596FE
:10020000D093870BC093860BCF3FD10578F48091B4
:100210002701909128018C9F90018D9F300D9C9F0C
:10022000300D1124C90164E670E013C0CE0196952B
:100230008795969587952091270130912801289FD1
:10024000A001299F500D389F500D1124CA0169E16A
:1002500070E00E949CB17093890B6093880B809131
:10026000BE049091BF048C0F9D1F9093BF04809398
:10027000BE0452E0813D9507A0F020918A0B309199
:100280008B0B2F5F3F4F805D9240E2E0813D9E07E8
:10029000C0F79093BF048093BE0430938B0B2093E0
:1002A0008A0BE9E0CDB7DEB70C9425B22091DA04D1
:1002B000822F9927FC0134E0EE0FFF1F3A95E1F7FA
:1002C000E81BF90BE05FF64F97818091DB048917FB
:1002D00028F49093DB042093DD0408C0992331F0C7
:1002E0008091DC04981710F49093DC04822F8F5FC8
:1002F0008093DA048031D0F01092DA048091DC042B
:100300008F3F19F08093CB0402C01092CB048091F0
:10031000DB048093CC048091DD048093CA048FEFCA
:100320008093DC041092DB041092DD04089595E1C3
:10033000899F802D11240E94C7A988E490E19F9392
:100340008F9389E999EA9F938F93E0913905F09112
:100350003A0509950F900F900F900F900895CF9345
:10036000C0E09091B0019093C9048091A90385FFEA
:1003700013C080919F03882331F08091000886305C
:1003800011F4CEE001C0C0E1992301F18091DE04B7
:100390008031E1F4C92F1AC090919304892F8150C4
:1003A0008632B0F48091DB03882349F4E92FFF27DC
:1003B000EE0FFF1FED53F34F8491882349F4E92F8B
:1003C000FF27EE0FFF1FEE53F34FC491CC2351F4E0
:1003D00080915C0886FD03C01092B00105C0C091F9
:1003E000B00102C0C093C9048091DE048C1771F47F
:1003F0008091DF049091E0040E940420882319F486
:1004000080E090E017C080EA9FE002C080ED97E0B6
:100410000E94FB1F9093E0048093DF04CC2331F013
:100420008091B001C81711F41092B001C093DE049E
:100430008C2F9927CF91089520E030E050E08091F3
:10044000540B992789389105E9F08A38910564F4AD
:100450008230910539F1833091051CF40197F9F050
:1004600028C0039719F125C08D389105A1F08E3869
:10047000910524F48A38910541F01BC08E3891050E
:1004800039F017C02FEE3BE008C027EC3CE005C078
:100490002DE83BE002C029EB3BE05CE20AC02EEC19
:1004A00032E002C021EE32E054E003C025EE3BE032
:1004B00059E09091490B40E080914A0B481770F445
:1004C000951760F4D901A90FB11DE42FFF27EA5C4D
:1004D000F44F85898C939F5F4F5FEECF089520E3A3
:1004E00035E7809144018B3211F08D32F9F480911F
:1004F000EB07282F33278091D0039091D103829F5F
:10050000A001839F500D929F500D1124CA0163E0FA
:1005100070E00E94B0B1CB019B01205D3A48C196CA
:10052000C19708F03FC02EEF34E73CC0803229F578
:100530008091A90381FF36C02091C6043091C70481
:10054000205D3A4855E72133350748F085E72439DF
:10055000380718F420E335E702C02456304045E759
:1005600020333407F8F454E72D3C350718F020E326
:1005700035E718C02C593F4F15C08E3549F490917E
:10058000CB038AE0989F90011124205D3A480AC06D
:10059000863741F49091CB038AE0989FC0011124E3
:1005A000281B390BC9010895CF93C0E099278A38D9
:1005B000910509F429C28B38910524F489389105F5
:1005C00051F0E2C38D38910509F415C38E389105B9
:1005D00009F470C2D9C39091C90C8091E1049817B5
:1005E00021F40E94AF818093E1048091D603909121
:1005F000D703A091D803B091D903BC01CD0124E663
:1006000030E040E050E00E94E5B1DA01C9018C50D1
:100610009E4F9093F50B8093F40B8091E104882317
:1006200019F40E946F8202C080E395E79093FB0B60
:100630008093FA0B8091FA0B9091FB0B9093FD0B3A
:100640008093FC0B9093FF0B8093FE0B2091F40B97
:100650003091F50B8091F80B9091F90B2817390721
:1006600024F43093F90B2093F80B8091F60B9091C2
:10067000F70B8217930724F43093F70B2093F60BB4
:100680001092F10B8FEE9BE0909301058093000593
:10069000809144018093150C8091A80380FF02C0D3
:1006A00083E401C080E28093160C209193042223FE
:1006B00009F1822F6AE00E9490B1805D8093000C66
:1006C000822F0E9490B1892F805D8093010C8AE374
:1006D0008093020C81E1289FF0011124A3E0BCE08B
:1006E000E05FF24FCFE084918D93C1503196C7FF08
:1006F000FACF39C180919F03882361F0A0E0BCE06C
:10070000E6E0F0E1C4E184918D93C1503196C7FFDA
:10071000FACF37C38091A90385FF0CC0A0E0BCE0ED
:10072000ECE1F0E1C4E184918D93C1503196C7FFB3
:10073000FACF27C38091C804882379F1A0E0BCE0F8
:10074000E7EAFFE0C6E084918D93C1503196C7FF80
:10075000FACF80910101805D8093040CA7E0BCE09A
:10076000EDE5F8E0CBE081918D93C150C7FFFBCF61
:100770008091A70381FF0BC082E48093110C8FE46A
:100780008093120C81E48093130C84E519C180E2FC
:100790008093120C8093130C13C18091D004882392
:1007A00011F1A0E0BCE0E4ECFFE0C4E184918D93A2
:1007B000C1503196C7FFFACF2091CF042A3020F4E0
:1007C000205D2093120CDDC2822F6AE00E9490B15E
:1007D000805D8093120C822F0E9490B1892F805DE2
:1007E0008093130CCEC28091D204882311F1A0E033
:1007F000BCE0EEEAFFE0C4E184918D93C1503196F4
:10080000C7FFFACF2091D1042A3020F4205D209335
:10081000110CB7C2822F6AE00E9490B1805D809374
:10082000110C822F0E9490B1892F805D8093120C51
:10083000A8C23091D804332309F497C087E5809388
:10084000000C80E58093010C40E24093020C209163
:10085000D904822F6AE00E9490B1805D8093030CDE
:10086000822F0E9490B1892F805D8093040C8FE2CB
:100870008093050C832F0E9490B1805D8093060CBD
:10088000832F0E9490B1892F805D8093070C409345
:10089000080C2091CD043091CE0483E0293E380726
:1008A00080F0C90168EE73E00E949CB1CB01805DCD
:1008B0008093090CC90168EE73E00E949CB19C0111
:1008C00002C04093090C2536310580F0C90164E669
:1008D00070E00E949CB1CB01805D80930A0CC9013D
:1008E00064E670E00E949CB19C0103C080E28093AA
:1008F0000A0CC9016AE070E00E949CB1CB01805DE6
:1009000080930B0CC9016AE070E00E949CB1805D8D
:1009100080930C0C8DE680930D0C80E280930E0C7E
:100920002091D704253660F0822F64E60E9490B1B2
:10093000805D80930F0C822F0E9490B1292F02C0FE
:1009400080930F0C822F6AE00E9490B1805D8093AB
:10095000100C822F0E9490B1892F805D8093110C22
:1009600083E78093120C80E215CF80918F0484FF7F
:100970000CC0A0E0BCE0E0EFFFE0C4E184918D9307
:10098000C1503196C7FFFACFFCC18091C7038823BD
:10099000D1F4A0E0BCE0E4E3F0E1C0E184918D9308
:1009A000C1503196C7FFFACF92E39093100C8EE2BC
:1009B0008093110C81E38093120C9093130C81E6C9
:1009C0008093140CDEC19091A70391FF0CC0A0E0AE
:1009D000BCE0EAEDFFE0C4E184918D93C150319613
:1009E000C7FFFACF0BC0A0E0BCE0E2E3F0E1C4E156
:1009F00084918D93C1503196C7FFFACF90FFC1C14A
:100A000082E58093000CBDC18091D6039091D703FD
:100A1000A091D803B091D903BC01CD0124E630E008
:100A200040E050E00E94E5B1DA01C9018C509E4FD0
:100A30009093DD0C8093DC0C8091E1048093C90CD1
:100A4000882319F40E946F8202C080E395E7909397
:100A5000DF0C8093DE0C88E78093E00C8091020B22
:100A60008093E10C8091010B81FF02C084E407C0F8
:100A70008091030B833011F480E201C081E2809306
:100A8000E20C87EC9CE09093010580930005809137
:100A900099018093EE0C8091E20C8093F00C809190
:100AA000070B9091080B97FD01969595879580937C
:100AB000E30C67C10E9456818091D6039091D703C1
:100AC000A091D803B091D903BC01CD0124E630E058
:100AD00040E050E00E94E5B1DA01C9018C509E4F20
:100AE0009093A80B8093A70B8091270190912801E8
:100AF0009093A20B8093A10B8091270190912801E4
:100B00009093A40B8093A30B8091ED0A9091EE0A31
:100B100097FD0196959587958093930B80939A0BFB
:100B20002091070B3091080B37FF02C02F5F3F4F1A
:100B3000359527952093980B8091050B9091060B86
:100B400064E170E00E949CB16093990B20939F0B2D
:100B50006093A00B8091E104882319F40E946F82B6
:100B600002C080E395E79093B00B8093AF0B88E7CA
:100B70008093B10B80912701909128019093AC0B49
:100B80008093AB0B8091CB048C5E8093A50B8091FE
:100B9000CC048C5E8093A60B80918A0B90918B0B7A
:100BA0006AE070E00E949CB17093AE0B6093AD0B55
:100BB00010928F0B8091860B9091870B9093AA0BCC
:100BC0008093A90B8DE89BE090930105809300052D
:100BD0002091F2023091F302C9016CE370E00E94AF
:100BE0009CB16093B40BC9016CE370E00E949CB1AE
:100BF0008093B50BC6C00E9456818091050B9091E1
:100C0000060B64E670E00E949CB17093CF0B60937A
:100C1000CE0B8091ED0A9091EE0A97FD0196959585
:100C200087958093BF0B809193019091940197FDDC
:100C30000196959587958093C00B80916C07809362
:100C4000C30B8091070B9091080B97FD019695952A
:100C500087958093C40B80910201482F55279A01F4
:100C60002E5F3F4F80912701909128012817390767
:100C700084F48091270190912801841B950B9C019D
:100C8000220F331F280F391F822F86508093CB0BE2
:100C900002C0C093CB0B8091CB0B853618F084E655
:100CA0008093CB0B8091930499279093CD0B8093E5
:100CB000CC0B8091D6039091D703A091D803B0912B
:100CC000D903BC01CD0124E630E040E050E00E94B1
:100CD000E5B1DA01C9018C509E4F9093D10B8093FE
:100CE000D00B80912701909128019093C60B80939F
:100CF000C50B80912701909128019093C80B809398
:100D0000C70B8091E104882319F40E946F8202C00E
:100D100080E395E79093D30B8093D20B8091E1040D
:100D200088588093D40B809127019091280190934B
:100D3000D80B8093D70B8091CB048C5E8093C90B2A
:100D40008091CC048C5E8093CA0B80918A0B909129
:100D50008B0B6AE070E00E949CB17093DA0B609399
:100D6000D90B1092BB0B8091860B9091870B9093BF
:100D7000D60B8093D50B89EB9BE090930105809374
:100D800000052CE230E002C020E030E0C901CF9144
:100D90000895EF92FF920F931F93CF93DF9380916B
:100DA000C6049091C7049C01F3E0220F331FFA950B
:100DB000E1F7281B390B80914B0390914C03280FCE
:100DC000391F37FF02C0295F3F4FE3E03595279574
:100DD000EA95E1F73093C7042093C6048091E304B9
:100DE0009927AA27BB27FC01099710F00C94CD9EE8
:100DF000E459FF4F2091E2040C9437B2822F9927D7
:100E0000AA27BB272F5F2093E204FC01419708F03B
:100E100005C4EB58FF4F0C9437B28091A90385FFAE
:100E20002AC080E00E94C7A98091270190912801E3
:100E30006AE070E00E94B0B19F938F938091270188
:100E4000909128016AE070E00E94B0B17F936F93A7
:100E50008EE590E19F938F938AEB99EA9F938F930E
:100E6000E0913905F0913A0509952DB73EB7285F15
:100E70003F4F2DBF28C080E00E94C7A98091270165
:100E8000909128016AE070E00E94B0B19F938F9327
:100E900080912701909128016AE070E00E94B0B132
:100EA0007F936F938BE690E19F938F9389E999EA03
:100EB0009F938F93E0913905F0913A0509958DB78D
:100EC0009EB708968DBF8091E40A80FF5AC080913A
:100ED000F303882371F18AE00E94C7A9809144013D
:100EE00099279F938F938091D6039091D703A091D8
:100EF000D803B091D903BC01CD0124E630E040E035
:100F000050E00E94E5B13F932F9388E790E19F93D3
:100F10008F9389EA99EA9F938F93E0913905F09135
:100F20003A0509952DB73EB7285F3F4F2DBF0C946A
:100F3000CF9E8AE00E94C7A98091D6039091D703E3
:100F4000A091D803B091D903BC01CD0124E630E0D3
:100F500040E050E00E94E5B13F932F9384E890E198
:100F60009F938F9389E999EA9F938F93E091390535
:100F7000F0913A0509958DB79EB706968DBF0C94F2
:100F8000CF9E8AE00E94C7A98FE890E19F938F933C
:100F900089E999EA9F938F93E0913905F0913A0599
:100FA00009950F900F900F900F900C94CF9E809109
:100FB000A90385FF2AC085E10E94C7A98091F2029A
:100FC0009091F3026CE370E00E949CB19F938F9329
:100FD0008091F2029091F3026CE370E00E949CB168
:100FE0007F936F9389E990E19F938F938AEB99EABE
:100FF0009F938F93E0913905F0913A0509952DB7AC
:101000003EB7285F3F4F2DBF28C085E10E94C7A98A
:101010008091F2029091F3026CE370E00E949CB127
:101020009F938F938091F2029091F3026CE370E0B2
:101030000E949CB17F936F9386EA90E19F938F9378
:1010400089E999EA9F938F93E0913905F0913A05E8
:1010500009958DB79EB708968DBF8FE10E94C7A9ED
:1010600080E690E09F938F938091ED0A9091EE0A35
:101070009F938F9383EB90E19F938F93C9E9D9EA74
:10108000DF93CF93E0913905F0913A05099580916E
:10109000A8032DB73EB7285F3F4F2DBF80FF16C076
:1010A00089E20E94C7A98EEB90E19F938F9389EA12
:1010B00099EA9F938F93E0913905F0913A0509954C
:1010C0000F900F900F900F900C94CF9E89E20E948A
:1010D000C7A980EC90E19F938F93DF93CF93E0912A
:1010E0003905F0913A0509950F900F900F900F90E8
:1010F0000C94CF9E8091A90385FF1BC08AE20E94B9
:10110000C7A980918A0B90918B0B9F938F9382EC50
:1011100090E19F938F938AEB99EA9F938F93E0914D
:101120003905F0913A0509958DB79EB706968DBFA2
:101130001BC08AE20E94C7A980918A0B90918B0BF9
:101140009F938F938AEC90E19F938F9389E999EA1B
:101150009F938F93E0913905F0913A0509952DB74A
:101160003EB72A5F3F4F2DBF86E30E94C7A98091FB
:10117000860B9091870B6AE070E00E949CB19F9370
:101180008F938091860B9091870B6AE070E00E94AC
:101190009CB17F936F9382ED90E19F938F9389E948
:1011A00099EA9F938F93E0913905F0913A0509955B
:1011B0008DB79EB708968DBF0C94CF9E89E00E9494
:1011C000C7A98EED90E19F938F9309E919EA1F93C8
:1011D0000F93E0913905F0913A0509958EE10E944F
:1011E000C7A90F900F900F900F9080EE90E19F9302
:1011F0008F931F930F93E0913905F0913A0509956C
:1012000083E30E94C7A90F900F900F900F9082EE7A
:1012100090E19F938F931F930F93E0913905F09185
:101220003A0509958FE30E94C7A90F900F900F9080
:101230000F9084EE90E19F938F931F930F93E09113
:101240003905F0913A0509958EE70E94C7A90F90DC
:101250000F900F900F908AEF90E19F938F931F93C1
:101260000F93E0913905F0913A0509950F900F9091
:101270000F900F900C94CF9E8091A701882309F4C2
:101280008EC08DE50E94C7A980E191E19F938F9365
:10129000C9E9D9EADF93CF93E0913905F0913A0596
:1012A000099584E50E94C7A90F900F900F900F90A9
:1012B0008091020B99279F938F9382E191E19F93F5
:1012C0008F93DF93CF93E0913905F0913A0509951B
:1012D0008EE50E94C7A92DB73EB72A5F3F4F2DBFAD
:1012E0008091050B9091060B6AE070E00E949CB122
:1012F0007F936F938BE191E19F938F93DF93CF93D4
:10130000E0913905F0913A0509958DB79EB706969B
:101310008DBF8091030B833061F58091010B81FFBC
:1013200014C08BE50E94C7A985E291E19F938F933A
:10133000DF93CF93E0913905F0913A0509950F902D
:101340000F900F900F900C94CF9E8BE50E94C7A931
:1013500088E291E19F938F93DF93CF93E0913905DA
:10136000F0913A0509950F900F900F900F900C9403
:10137000CF9E8BE50E94C7A98BE291E19F938F934B
:101380008AEB99EA9F938F93E0913905F0913A05A2
:1013900009950F900F900F900F900C94CF9E84E0C2
:1013A0000E9497810C94CF9E8091A701882309F415
:1013B0008BC08091E50479E9E72E79EAF72E88233E
:1013C00009F45AC089E60E94C7A98091920499271E
:1013D0009F938F938EE291E19F938F93FF92EF9271
:1013E000E0913905F0913A05099585E70E94C7A972
:1013F0002DB73EB72A5F3F4F2DBF809199019927A6
:101400009F938F9300E610E01F930F938091070B3B
:101410009091080B9F938F9389E391E19F938F9312
:10142000FF92EF92E0913905F0913A05099582E734
:101430000E94C7A98DB79EB70A968DBF8091900470
:1014400099279F938F931F930F93809191049927CE
:101450009F938F9385E491E19F938F93FF92EF92F7
:10146000E0913905F0913A0509952DB73EB7265F11
:101470003F4F2DBF0C94CF9E89E60E94C7A9809153
:10148000990199279F938F9380E690E09F938F9384
:101490008091070B9091080B9F938F938091040B81
:1014A00099279F938F9385E591E19F938F93FF9267
:1014B000EF92E0913905F0913A0509958DB79EB705
:1014C0000C968DBF0C94CF9E85E00E9497810C9462
:1014D000CF9E90919304992309F44EC08091FD040E
:1014E000882309F19732F8F487E00E94978183E915
:1014F0000E94C7A98091930499279F938F938EE6AA
:1015000091E19F938F9389EA99EA9F938F93E0915A
:101510003905F0913A0509952DB73EB72A5F3F4F3F
:101520002DBF0C94CF9E83E90E94C7A989E791E162
:101530009F938F9309E919EA1F930F93E09139055F
:10154000F0913A0509951F921F929091930481E1C1
:10155000989FC0011124805F924F9F938F931F9398
:101560000F93E0913905F0913A0509958DB79EB733
:101570000A968DBF0C94CF9E8091A90369E9E62E4F
:1015800069EAF62E85FF14C084E90E94C7A98FE797
:1015900091E19F938F93FF92EF92E0913905F09143
:1015A0003A0509950F900F900F900F900C94CF9ED5
:1015B00083E90E94C7A982E991E19F938F93FF92EB
:1015C000EF92E0913905F0913A0509950F900F904F
:1015D0000F900F900C94CF9E8091500D823021F48B
:1015E0000E94CCA985E012C0863059F48091E504B0
:1015F000882319F01092E5040DC081E08093E50482
:1016000009C0883039F40E94CCA981E08093E304BA
:101610001092E2041092500D0C94CF9E1092E204AE
:101620000C94CF9E822F9927AA27BB272F5F209348
:10163000E204FC01419708F09CC4EA57FF4F0C9468
:1016400037B28091A90385FF45C080E00E94C7A9F9
:1016500080918A0B90918B0B9F938F9380912701A0
:10166000909128016AE070E00E94B0B19F938F933F
:1016700080912701909128016AE070E00E94B0B14A
:101680007F936F938091F2029091F3026CE370E08C
:101690000E949CB19F938F938091F2029091F302EC
:1016A0006CE370E00E949CB17F936F9388EA91E1B4
:1016B0009F938F938AEB99EA9F938F93E0913905DB
:1016C000F0913A0509952DB73EB7225F3F4F2DBFE8
:1016D0000C94CF9E80E00E94C7A980918A0B9091C4
:1016E0008B0B9F938F9380912701909128016AE043
:1016F00070E00E94B0B19F938F93809127019091E9
:1017000028016AE070E00E94B0B17F936F938091EE
:10171000F2029091F3026CE370E00E949CB19F93FF
:101720008F938091F2029091F3026CE370E00E943B
:101730009CB17F936F9383EC91E19F938F9389E9A1
:1017400099EA9F938F93E0913905F0913A050995B5
:101750008DB79EB70E968DBF0C94CF9E85E10E94EB
:10176000C7A980E690E09F938F938091ED0A9091B6
:10177000EE0A9F938F938EED91E19F938F93C9E92A
:10178000D9EADF93CF93E0913905F0913A050995B5
:101790008091E40A2DB73EB7285F3F4F2DBF80FFF1
:1017A00051C08091F303882339F18FE10E94C7A9CA
:1017B0008091D6039091D703A091D803B091D9031B
:1017C000BC01CD0124E630E040E050E00E94E5B1EC
:1017D0003F932F9388EE91E19F938F9389EA99EA43
:1017E0009F938F93E0913905F0913A0509958DB754
:1017F0009EB706968DBF38C08FE10E94C7A9809121
:10180000D6039091D703A091D803B091D903BC011E
:10181000CD0124E630E040E050E00E94E5B13F9386
:101820002F9381EF91E19F938F93DF93CF93E0917B
:101830003905F0913A0509952DB73EB72A5F3F4F1C
:101840002DBF12C08FE10E94C7A98AEF91E19F933B
:101850008F93DF93CF93E0913905F0913A05099585
:101860000F900F900F900F9089E20E94C7A980916E
:10187000440199279F938F9384E092E19F938F93E4
:10188000DF93CF93E0913905F0913A0509958DB733
:101890009EB706968DBF0C94CF9E8091A70188239A
:1018A00081F18BE20E94C7A98091990199279F93AA
:1018B0008F938091050B9091060B6AE070E00E9477
:1018C0009CB17F936F9380E690E09F938F9380917C
:1018D000070B9091080B9F938F9387E092E19F9362
:1018E0008F9389E999EA9F938F93E0913905F0915D
:1018F0003A0509952DB73EB7245F3F4F2DBF0C9495
:10190000CF9E82E00E9497810C94CF9E8FE30E942D
:10191000C7A98091880B9091890B9F938F93809199
:10192000860B9091870B6AE070E00E949CB19F93B8
:101930008F938091860B9091870B6AE070E00E94F4
:101940009CB17F936F938EE192E19F938F93C9E94E
:10195000D9EADF93CF93E0913905F0913A050995E3
:101960008091A8032DB73EB7265F3F4F2DBF80FF64
:1019700016C082E50E94C7A982E392E19F938F93EC
:1019800089EA99EA9F938F93E0913905F0913A059E
:1019900009950F900F900F900F900C94CF9E82E5B9
:1019A0000E94C7A985E392E19F938F93DF93CF9322
:1019B000E0913905F0913A0509950F900F900F903D
:1019C0000F900C94CF9E8091A70159E9E52E59EA1A
:1019D000F52E882309F459C084E50E94C7A9809197
:1019E000020B99279F938F938091040B99279F93C4
:1019F0008F9388E392E19F938F93E701FF92EF9299
:101A0000E0913905F0913A0509958DB79EB7089692
:101A10008DBF8091030B833051F484E60E94C7A9E7
:101A20008BE492E19F938F93FF92EF920BC084E639
:101A30000E94C7A981E592E19F938F938AEB99EA6F
:101A40009F938F93E0913905F0913A0509950F9096
:101A50000F900F900F908091010B81FD02C00C94AC
:101A6000CF9E84E60E94C7A987E592E19F938F935A
:101A7000DF93CF93E0913905F0913A0509950F90E6
:101A80000F900F900F900C94CF9E84E50E94C7A9F1
:101A90008DE592E19F938F93FF92EF92E09139054C
:101AA000F0913A0509950F900F900F900F900C94BC
:101AB000CF9E8091E40449E9E42E49EAF42E88237C
:101AC00009F45DC089E60E94C7A983E00E944980AD
:101AD0006AE070E00E949CB19F938F9383E00E9424
:101AE00049806AE070E00E949CB17F936F9382E02E
:101AF0000E9449806AE070E00E949CB19F938F939E
:101B000082E00E9449806AE070E00E949CB17F936D
:101B10006F9381E00E9449806AE070E00E949CB16E
:101B20009F938F9381E00E9449806AE070E00E9459
:101B30009CB17F936F9380E00E9449806AE070E0DF
:101B40000E949CB19F938F9380E00E9449806AE03D
:101B500070E00E949CB17F936F9383E792E19F9323
:101B60008F93FF92EF92E0913905F0913A05099534
:101B70002DB73EB72C5E3F4F2DBF0C94CF9E89E60C
:101B80000E94C7A980E690E09F938F9380914409BB
:101B900099279F938F938091350999279F938F93CE
:101BA0008091260999279F938F93809117099927F0
:101BB0009F938F9380E992E19F938F93FF92EF928F
:101BC000E0913905F0913A0509958DB79EB70E96CB
:101BD0008DBF0C94CF9E8091E4049091D807882308
:101BE00009F4B8C0943029F486E00E9497810C94DF
:101BF000CF9E9630D9F58EE70E94C7A985E00E9456
:101C000049806AE070E00E949CB19F938F9385E0C9
